:020000040800F2
:1000000000040020A51F0008F71F0008F71F0008C4
:10001000F71F0008F71F0008F71F00080000000086
:10002000000000000000000000000000F71F0008B2
:10003000F71F000800000000F71F0008B52B02089A
:100040004D2D02084F2D0208512D0208552D020892
:10005000852D0208872D0208892D0208AD2D020882
:10006000D12D0208F52D0208192E02083D2E020896
:100070003F2E0208412E0208432E0208452E020898
:10008000472E0208492E02084B2E0208F71F0008CF
:10009000F71F0008F71F0008F71F00084D2E020881
:1000A000992E02089B2E02089D2E02089F2E020800
:1000B000A12E0208A52E0208D12E0208412F020807
:1000C000432F0208452F0208472F0208492F020834
:1000D0004D2F0208BD300208E52F020881310208C9
:1000E0003D320208013302080333020805330208D7
:1000F00009330208713302087333020875330208AA
:1001000077330208793302087B3302087D33020813
:100110008133020855340208573402085934020862
:100120006535020867350208693502086B35020833
:1001300000000000000000000000000000000000BF
:1001400000000000000000000000000000000000AF
:10015000000000000000000000000000000000009F
:10016000000000000000000000000000000000008F
:10017000000000000000000000000000000000007F
:10018000000000000000000000000000000000006F
:10019000000000000000000000000000000000005F
:1001A000000000000000000000000000000000004F
:1001B000000000000000000000000000000000003F
:1001C000000000000000000000000000000000002F
:1001D000000000000000000000000000000000001F
:0401E0005FF8E0F1F3
:1001E800032A70B404460D4626D941EA000313F0E9
:1001F800030F13D020782B78984208BF294606D0E1
:100208001EE014F8010F11F8013F984218D1012A95
:1002180002F1FF32F5D1002070BC70470B4604464E
:1002280051F8045B50F8046BAE4204D1043A04461A
:10023800032A0B46F2D81D461046002ADAD1EBE70E
:10024800C01AE9E7032A2DE9F00109D82AB10023E9
:10025800CC5CC45401339342FAD1BDE8F001704735
:100268000B468218014603E02478013301F8014B5C
:1002780011F0030F1C46F7D113F003055DD06E4251
:10028800C5F1040CED009B594FEACC0C08E004348E
:10029800A7593B4607FA0CF748EA070741F8047BD9
:1002A800571A23FA05F8032FF1DC03E014F8013B91
:1002B80001F8013B8A42F9D8CFE753F8404C41F89E
:1002C800404C53F83C4C41F83C4C53F8384C41F8FE
:1002D800384C53F8344C41F8344C53F8304C41F80E
:1002E800304C53F82C4C41F82C4C53F8284C41F81E
:1002F800284C53F8244C41F8244C53F8204C41F82E
:10030800204C53F81C4C41F81C4C53F8184C41F83D
:10031800184C53F8144C41F8144C53F8104C41F84D
:10032800104C53F80C4C41F80C4C53F8084C41F85D
:10033800084C53F8044C41F8044C561A1D460C4618
:10034800403340313F2EB8DC2B460FE053F8101CE9
:1003580044F8101C53F80C1C44F80C1C53F8081CE7
:1003680044F8081C53F8041C44F8041C161B2146C6
:100378001D46103410330F2EE8DC2B4602E02468AB
:1003880041F8044B551A1C46032D03F10403F6DC0F
:1003980090E700BF032AC9B270B408D82AB103464F
:1003A800121803F8011B9342FBD170BC70478218E6
:1003B800044601E004F8011B14F0030FFAD14FF0D2
:1003C800013303FB01F31FE044F8403C44F83C3C94
:1003D80044F8383C44F8343C44F8303C44F82C3C6D
:1003E80044F8283C44F8243C44F8203C44F81C3C9D
:1003F80044F8183C44F8143C44F8103C44F80C3CCD
:1004080044F8083C44F8043C161B254640343F2E6B
:10041800DADC2C4607E044F8103C44F80C3C44F87D
:10042800083C44F8043C161B254610340F2EF2DC19
:1004380001E045F8043B541B032CFADC01E005F805
:10044800011B9542FBD3B0E710F0030F38B5044603
:1004580012D10368A3F1013222EA030313F0803FAB
:100468000AD1031D184653F8042BA2F1013525EAD9
:10047800020212F0803FF5D003782BB1431C1846D6
:1004880013F8012B002AFAD100F076F9204638BD7E
:10049800C9B2F0B4002950D010F0030F10D003787F
:1004A800002B79D0994246D0431C05E013F8012B64
:1004B800002A3FD091423ED013F0030F1846F5D1E1
:1004C800036841EA01270646A3F1013247EA0747D4
:1004D80022EA030212F0803F1DD187EA0303A3F149
:1004E800013222EA030313F0803F14D1043002E002
:1004F80012F0803F0FD1064650F8043BA3F10135B6
:1005080087EA030225EA0303A2F1013413F0803FCE
:1005180024EA0202ECD033783046002B3CD09942D2
:1005280009D0731C01E0914205D0184613F8012B3D
:10053800002AF8D11046F0BC704710F0030F0CD019
:100548000378002BF7D0431C03E013F8012B002A93
:10055800F1D013F0030F1846F7D102680346A2F151
:10056800013121EA020212F0803F0AD10430034629
:1005780050F8042BA2F1013121EA020212F0803F67
:10058800F5D01A781846002AD5D00133184613F842
:10059800012B002AFAD1CEE71846CCE780EA0102FF
:1005A80012F0030F3AD110F0030220F0030021F0FB
:1005B800030150F804CB08BF51F8043B0DD082F07A
:1005C80003024FEAC2026FF07F4323FA02F251F8A6
:1005D800043B4CEA020C43EA020300BFACF10132CF
:1005E8009C4501BF22EA0C0212F0803F50F804CB70
:1005F80051F8043BF2D04FEA0C604FEA1C2C01285A
:1006080028BFB0EB036F08BF1B0AF4D003F0FF0349
:100618004FEA1060A0EB0300704700BF10F0030F13
:100628000AD010F8012B11F8013B012A28BF9A4281
:10063800F4D0A2EB030070474DF8045D4DF8044D6B
:100648004FF0010242EA022242EA024201F0030CA0
:1006580021F0030150F8044B51F8045BBCF1020F80
:1006680026D04BD824F07F4CBCEB152FA4EB02030B
:1006780023EA04030DD113EAC21308BF51F8045B3F
:100688000AD18CEA040CBCEB056F0CD150F8044B72
:10069800E8E74FEA15255CE033F07F4352D10D7847
:1006A8004FEA146C55E04FEA146C05F0FF0550E072
:1006B8004FEA044CA4EB02034FEA1C4C23EA040360
:1006C800BCEB154F17D113EAC21308BF51F8045BEE
:1006D80007D18CEA040CBCEB054F08D150F8044B49
:1006E800E6E71B042ED10D884FEA144C31E04FEA9F
:1006F80005454FEA144C4FEA15452AE004F0FF0C73
:10070800BCEB156FA4EB020323EA04030DD113EA33
:10071800C21308BF51F8045B0AD18CEA040CBCEB85
:10072800052F0AD150F8044BE8E74FEA156510E0A9
:1007380014F0FF0F06D051F8045B4FEA142C25F093
:100748007F4506E04FF000005DF8044B5DF8045B60
:1007580070470CF0FF0205F0FF00012828BF904207
:1007680004BF4FEA1C2C2D0AF3D0A2EB00005DF861
:10077800044B5DF8045B704780EA0102844612F07E
:10078800030F4FD111F0030F32D14DF8044D11F082
:10079800040F51F8043B0BD0A3F101329A4312F035
:1007A800803F04BF4CF8043B51F8043B16D100BF0E
:1007B80051F8044BA3F101329A4312F0803FA4F19F
:1007C80001320BD14CF8043BA24312F0803F04BF26
:1007D80051F8043B4CF8044BEAD023460CF8013B93
:1007E80013F0FF0F4FEA3323F8D15DF8044B70473D
:1007F80011F0010F06D011F8012B0CF8012B002A7B
:1008080008BF704711F0020FBFD031F8022B12F069
:10081800FF0F16BF2CF8022B8CF8002012F47F4F24
:10082800B3D1704711F8012B0CF8012B002AF9D12C
:10083800704700BF20F0030110F00300C0F1000072
:1008480051F8043B00F1040C4FEACC0C6FF00002A5
:100858001CBF22FA0CF213434FF0010C4CEA0C2C8B
:100868004CEA0C4CA3EB0C0222EA030212EACC126B
:1008780004BF51F8043B0430F4D013F0FF0F1FBF3E
:10088800013013F47F4F013013F47F0F18BF01308C
:10089800704700BFF0B4002A46D041EA000313F0C5
:1008A80003032CD1032A07460E4643D904680D6872
:1008B800AC423FD1043A37D0A4F1013525EA04040B
:1008C80014F0803F18BF18462CD1041D0D1D0EE0F2
:1008D80054F8043B55F8041BA3F101308B4220EA7D
:1008E800030027D1043A1FD010F0803F1ED1032AFD
:1008F80027462E46ECD820462946002A1DD00478E3
:10090800013A0D78AC420CD172B18CB1002302E0EF
:1009180093420BD064B1013310F8014FCD5CAC4267
:10092800F6D0601BF0BC70471046FBE70020F9E7E3
:100938002046F7E738463146E1E724782D78F0E796
:1009480041EA000313F0030F0B4670B414BF0024F0
:100958000124032A94BF002404F001040546D4B9F5
:10096800BAB10E782B46013A03F8016B56B1AC1CAC
:100978007AB111F8015F2346013A04F8015C0134A9
:10098800002DF5D12AB19A18002103F8011B9342D2
:10099800FBD170BC7047194653F8044BA4F10136DB
:1009A80026EA040616F0803FDAD1043A45F8044BEB
:1009B800032A1946EFD8D3E701232DE9F0071D468E
:1009C80000264FF0FF37AC1900EB070C8C420DD214
:1009D8001CF805C010F80480E0452ED201252646F3
:1009E800E31BAC198C4200EB070CF1D34FF0010963
:1009F80000264D464FF0FF3C1360AC1900EB0C0885
:100A0800A1420ED918F8058010F804A0C2451AD9D9
:100A180001252646CCEB0409AC19A14200EB0C08D1
:100A2800F0D80CF101000137B8423CBF994638466E
:100A3800C2F80090BDE8F00770470BD00123374695
:100A48001D46F618BFE709D04FF00109B4464D46D8
:100A58004E44D2E79D4205D00135B4E74D4505D057
:100A68000135CAE72B4626460125ACE7A9462646A6
:100A78000125C2E72DE9F04FADF5826D81B014462E
:100A8800074610460DF580628B460C3219461D4606
:100A9800FFF792FF03AE04A901F57E72331F0090A1
:100AA80043F8045F9342FBD14DB1681E0023E25C1A
:100AB800C11A013303AEAB4246F82210F7D1DDF874
:100AC8000C142046009A6118FFF78AFB002877D19A
:100AD8000099814605F1FF380646C1F101020192ED
:100AE8005A46AB4609EB0B0501F1FF3AB81800214D
:100AF800AA1A00F0E5F900284FD1002D00F0C080B7
:100B08007B1903A913F8013C51F82330002B4CD171
:100B1800009B9E4228BF334698450FD903EB090135
:100B2800E05C7A18795C884205D038E012F8011F39
:100B3800E05C884233D101339845F7D8009A964251
:100B480080F0A48007EB090214F80A10534612F843
:100B58000A20914204BF0AEB0901791807D095E0F1
:100B680014F802C011F8010D844503D113465A1E2A
:100B7800B342F5D101369E4200F28D80DDF80C6457
:100B88002A46B144C6EB0B0609EB0B05B818002141
:100B9800AA1A00F095F90028AFD0002071E0019A58
:100BA8000026914499442A46EEE7002EFAD0DDF853
:100BB8000C2493423CBFC2EB0B0306469944F2E770
:100BC800009E4FF000080099AB1BB34238BF334674
:100BD800C1F101026E1E019201F1FF3A5A4689469F
:100BE800AB460133CDF80C3408EB0B05B8180021DF
:100BF800AA1A00F065F90028CFD1002D40D07B1942
:100C080003A913F8013C51F82330002B30D1B1452A
:100C180013D208EB090314F80910FA18FB5C99427F
:100C280018BF4B4627D14B4604E012F8011FE05C81
:100C3800884220D10133B342F7D3BAF1FF3F53467C
:100C48002CD007EB080C14F80A101CF80A20914263
:100C58000CD10AEB0802BA1804E0E05C12F8011D96
:100C6800884203D1013BF8D260460AE0DDF80C3433
:100C780098442A46B8E701992A4688449844B3E735
:100C8800284605B00DF5806DBDE8F08F009B013654
:100C98009E427FF673AF07EB0900F2E707EB080CFB
:100CA8006046EEE72DE9F04F8346037885B00C46A1
:100CB800002B00F0F9800A78A2B106460131012024
:100CC80002E011F8012B8AB1934214BF002000F012
:100CD800010016F8013F0D46002BF2D12B782BB1FD
:100CE8004FF0000B584605B0BDE8F08F0028F9D149
:100CF8000BF101002178FFF7CBFB2D1BA5F10102B9
:100D0800534243EB0203002808BF43F001030746A0
:100D180083B90BEB0508404594BFC0EB08084FF0BA
:100D280001081F2D08D9414622462B46FFF7A2FE8F
:100D38008346D7E78346D5E7294603AA2046FFF727
:100D48003BFE03996118814620464A46FFF748FA58
:100D580000284FD109F1FF33C9F10102064601927B
:100D680082464246C84699460AEB050BB818002148
:100D7800C2EB0B0200F0A4F80028B1D1BBF1000FC0
:100D8800B0D046452CBF334643469D420FD903EBAE
:100D98000A01E05C7A18795C884205D075E012F89F
:100DA800011FE05C884270D101339D42F7D1B04504
:100DB8007DD907EB0A0214F809104B4612F80920EE
:100DC800914202BF09EB0A01AC46791806D06EE0E1
:100DD800A55C11F8010D854203D113465A1EB34292
:100DE800F6D1654601369E4267D8039E5A46B244FC
:100DF800AE1BB9E7C9F10101C9EB0503424600265C
:100E080009F1FF3A88464B4538BF4B4601330393F7
:100E180006EB050BB8180021C2EB0B0200F050F8E6
:100E280000287FF45DAFBBF1000F3FF45BAF4D4589
:100E380012D906EB090314F80910FA18FB5C994259
:100E480008BF4B4605D026E012F8011FE05C884237
:100E580022D101339D42F7D1BAF1FF3F534628D042
:100E680007EB060C14F80A101CF80A20914217D157
:100E78000AEB0602BA1804E0E05C12F8011D884289
:100E88000ED1013BF8D2E3462CE7019A00269244A2
:100E98005A469A4468E74B4646445A46F618B7E716
:100EA800039B5A46F618B3E70D46012016E743465A
:100EB80098E707EB060CE34614E707EB0A0B11E784
:100EC80010F0030F034670B4C9B211D0002A22D023
:100ED80003788B421DD0013A013005E0DAB110F8F1
:100EE800014B013A8C4218D010F0030F0346F5D19C
:100EF800032A14D87AB1187888420ED0541E5D1C83
:100F080003E015F8016B8E4203D0013C2846F8D265
:100F1800002070BC70471046FBE71846F9E741EA25
:100F2800012646EA0646184653F8044B86EA0404A6
:100F3800A4F1013525EA040414F0803F03D1043AF2
:100F48001846032AEFD80346D4E700BF0000000084
:100F5800C1F30A5C0246ACF57E7C2DE9F84FACF192
:100F68000704132C0B4606460F468946804627DCA5
:100F7800002C52DB4FF6FF7CC0F20F0C4CFA04FA3F
:100F88000AEA0105054317D037A3D3E9002300F087
:100F980075F80022002300F0B3FC002856D0002F7B
:100FA80005DD4FF4801353FA04F407EB040929EA2A
:100FB8000A0900264B46324610461946BDE8F88F06
:100FC800332C07DDB4F5806FF6D100F057F80246F0
:100FD8000B46F1E74FF0FF3BACF11B0C2BFA0CFB77
:100FE8001BEA000FE8D020A3D3E9002300F046F85D
:100FF8000022002300F084FC40B3002F0ADD142CEB
:1010080006D00126C4F13404A64016EB080601D325
:1010180007F1010926EA0B0619E013A3D3E9002317
:1010280000F02CF80022002300F06AFC78B1002FB1
:1010380013DB46EA07054FF000094D45C3F6F07982
:101048000CBF2E46002608BFA94600E0B9464B460D
:10105800324610461946BDE8F88F00264FF0004981
:10106800F5E700BFAFF300809C7500883CE4377E4D
:1010780081F0004102E000BF83F0004330B54FEA41
:1010880041044FEA430594EA050F08BF90EA020FAE
:101098001FBF54EA000C55EA020C7FEA645C7FEA41
:1010A800655C00F0E2804FEA5454D4EB5555B8BF64
:1010B8006D420CDD2C4480EA020281EA030382EAD5
:1010C800000083EA010180EA020281EA0303362D67
:1010D80088BF30BD11F0004F4FEA01314FF4801C3A
:1010E8004CEA113102D0404261EB410113F0004F4C
:1010F8004FEA03334CEA133302D0524263EB430303
:1011080094EA050F00F0A780A4F10104D5F1200EA0
:101118000DDB02FA0EFC22FA05F2801841F10001FB
:1011280003FA0EF2801843FA05F359410EE0A5F1CF
:1011380020050EF1200E012A03FA0EFC28BF4CF000
:10114800020C43FA05F3C01851EBE37101F00045B6
:1011580007D54FF0000EDCF1000C7EEB00006EEBC3
:101168000101B1F5801F1BD3B1F5001F0CD349084D
:101178005FEA30004FEA3C0C04F101044FEA4452A4
:1011880012F5800F80F09A80BCF1004F08BF5FEA2B
:10119800500C50F1000041EB045141EA050130BD0B
:1011A8005FEA4C0C404141EB010111F4801FA4F1AE
:1011B8000104E9D191F0000F04BF01460020B1FA03
:1011C80081F308BF2033A3F10B03B3F120020CDA3B
:1011D8000C3208DD02F1140CC2F10C0201FA0CF019
:1011E80021FA02F10CE002F11402D8BFC2F1200C7E
:1011F80001FA02F120FA0CFCDCBF41EA0C01904034
:10120800E41AA2BF01EB0451294330BD6FEA04047C
:101218001F3C1CDA0C340EDC04F11404C4F1200267
:1012280020FA04F001FA02F340EA030021FA04F379
:1012380045EA030130BDC4F10C04C4F1200220FAD0
:1012480002F001FA04F340EA0300294630BD21FA0E
:1012580004F0294630BD94F0000F83F4801306BFD4
:1012680081F480110134013D4EE77FEA645C18BFC8
:101278007FEA655C29D094EA050F08BF90EA020F5F
:1012880005D054EA000C04BF1946104630BD91EA57
:10129800030F1EBF0021002030BD5FEA545C05D15A
:1012A8004000494128BF41F0004130BD14F5800499
:1012B8003CBF01F5801130BD01F0004545F0FE410D
:1012C80041F470014FF0000030BD7FEA645C1ABF42
:1012D800194610467FEA655C1CBF0B46024650EA79
:1012E800013406BF52EA033591EA030F41F40021A5
:1012F80030BD00BF90F0000F04BF0021704730B52B
:101308004FF4806404F132044FF000054FF00001FF
:1013180050E700BF90F0000F04BF0021704730B5C0
:101328004FF4806404F1320410F0004548BF404295
:101338004FF000013EE700BF42004FEAE2014FEAEA
:1013480031014FEA02701FBF12F07F4393F07F4FC5
:1013580081F06051704792F0000F14BF93F07F4FF7
:10136800704730B54FF4607401F0004521F000413A
:1013780020E700BF50EA010208BF704730B54FF0C0
:1013880000050AE050EA010208BF704730B511F0C5
:10139800004502D5404261EB41014FF4806404F1FD
:1013A80032045FEA915C3FF4DCAE4FF003025FEA7F
:1013B800DC0C18BF03325FEADC0C18BF033202EB07
:1013C800DC02C2F1200300FA03FC20FA02F001FA61
:1013D80003FE40EA0E0021FA02F11444C1E600BF00
:1013E80070B54FF0FF0C4CF4E06C1CEA11541DBFB3
:1013F8001CEA135594EA0C0F95EA0C0F00F0DEF87E
:101408002C4481EA030621EA4C5123EA4C5350EA62
:10141800013518BF52EA033541F4801143F48013B3
:1014280038D0A0FB02CE4FF00005E1FB02E506F044
:101438000042E0FB03E54FF00006E1FB03569CF099
:10144800000F18BF4EF0010EA4F1FF04B6F5007F9F
:1014580064F5407404D25FEA4E0E6D4146EB060611
:1014680042EAC62141EA55514FEAC52040EA5E509A
:101478004FEACE2EB4F1FD0C88BFBCF5E06F1ED844
:10148800BEF1004F08BF5FEA500E50F1000041EB7B
:10149800045170BD06F0004646EA010140EA020028
:1014A80081EA0301B4EB5C04C2BFD4EB0C0541EA4A
:1014B800045170BD41F480114FF0000E013C00F35F
:1014C800AB8014F1360FDEBF002001F0004170BD83
:1014D800C4F10004203C35DA0C341BDC04F114049C
:1014E800C4F1200500FA05F320FA04F001FA05F228
:1014F80040EA020001F0004221F0004110EBD370F5
:1015080021FA04F642EB06015EEA430E08BF20EA20
:10151800D37070BDC4F10C04C4F1200500FA04F3C3
:1015280020FA05F001FA04F240EA020001F0004155
:1015380010EBD37041F100015EEA430E08BF20EAC8
:10154800D37070BDC4F1200500FA05F24EEA020E10
:1015580020FA04F301FA05F243EA020321FA04F03F
:1015680001F0004121FA04F220EA020000EBD370F6
:101578005EEA430E08BF20EAD37070BD94F0000FF6
:101588000FD101F00046400041EB010111F4801F2A
:1015980008BF013CF7D041EA060195F0000F18BFDB
:1015A800704703F00046520043EB030313F4801F17
:1015B80008BF013DF7D043EA0603704794EA0C0FD1
:1015C8000CEA135518BF95EA0C0F0CD050EA4106E7
:1015D80018BF52EA4306D1D181EA030101F0004164
:1015E8004FF0000070BD50EA410606BF104619468C
:1015F80052EA430619D094EA0C0F02D150EA013698
:1016080013D195EA0C0F05D152EA03361CBF1046D8
:1016180019460AD181EA030101F0004141F0FE4177
:1016280041F470014FF0000070BD41F0FE4141F4FB
:10163800780170BD70B54FF0FF0C4CF4E06C1CEAFB
:1016480011541DBF1CEA135594EA0C0F95EA0C0FB0
:1016580000F0A7F8A4EB050481EA030E52EA03356B
:101668004FEA013100F088804FEA03334FF080558C
:1016780045EA131343EA12634FEA022245EA1115B9
:1016880045EA10654FEA00260EF000419D4208BF6A
:10169800964244F1FD0404F5407402D25B084FEA17
:1016A8003202B61A65EB03055B084FEA32024FF4C3
:1016B80080104FF4002CB6EB020E75EB030E22BF20
:1016C800B61A754640EA0C005B084FEA3202B6EBE0
:1016D800020E75EB030E22BFB61A754640EA5C008F
:1016E8005B084FEA3202B6EB020E75EB030E22BF1F
:1016F800B61A754640EA9C005B084FEA3202B6EB20
:10170800020E75EB030E22BFB61A754640EADC00DE
:1017180055EA060E18D04FEA051545EA16754FEA40
:1017280006164FEAC30343EA52734FEAC2025FEA5E
:101738001C1CC0D111F4801F0BD141EA00014FF0ED
:1017480000004FF0004CB6E711F4801F04BF0143BE
:101758000020B4F1FD0C88BFBCF5E06F3FF6AFAEDA
:10176800B5EB030C04BFB6EB020C5FEA500C50F16A
:10177800000041EB045170BD0EF0004E4EEA1131ED
:1017880014EB5C04C2BFD4EB0C0541EA045170BDF4
:1017980041F480114FF0000E013C90E645EA060E38
:1017A8008DE60CEA135594EA0C0F08BF95EA0C0F66
:1017B8003FF43BAF94EA0C0F0AD150EA01347FF4AE
:1017C80034AF95EA0C0F7FF425AF104619462CE785
:1017D80095EA0C0F06D152EA03353FF4FDAE1046E8
:1017E800194622E750EA410618BF52EA43067FF439
:1017F800C5AE50EA41047FF40DAF52EA43057FF4C9
:10180800EBAE12E74FF0FF3C06E000BF4FF0010CD3
:1018180002E000BF4FF0010C4DF804CD4FEA410C37
:101828007FEA6C5C4FEA430C18BF7FEA6C5C1BD004
:1018380001B050EA410C0CBF52EA430C91EA030F85
:1018480002BF90EA020F0020704710F1000F91EAE2
:10185800030F58BF994208BF90422CBFD8176FEAB0
:10186800E37040F0010070474FEA410C7FEA6C5C7E
:1018780002D150EA013C07D14FEA430C7FEA6C5C85
:10188800D6D152EA033CD3D05DF8040B704700BFB1
:101898008446104662468C461946634600E000BFFF
:1018A80001B5FFF7B7FF002848BF10F1000F01BDD1
:1018B8004DF808EDFFF7F4FF0CBF012000205DF89C
:1018C80008FB00BF4DF808EDFFF7EAFF34BF012021
:1018D80000205DF808FB00BF4DF808EDFFF7E0FFBA
:1018E80094BF012000205DF808FB00BF4DF808ED0B
:1018F800FFF7CEFF94BF012000205DF808FB00BF72
:101908004DF808EDFFF7C4FF34BF012000205DF853
:1019180008FB00BF4FEA4102B2F1E04324BFB3F530
:10192800001CDCF1FE5C0DD901F0004C4FEAC0024E
:101938004CEA5070B2F1004F40EB830008BF20F032
:101948000100704711F0804F21D113F13872BCBFEC
:1019580001F00040704741F480114FEA5252C2F141
:101968001802C2F1200C10FA0CF320FA02F018BF8A
:1019780040F001004FEAC1234FEAD32303FA0CFCDD
:1019880040EA0C0023FA02F34FEA4303CCE77FEA6C
:10199800625307D150EA01331EBF4FF0FE4040F4B6
:1019A8004000704701F0004040F0FE4040F4000065
:1019B800704700BF80F0004002E000BF81F00041A6
:1019C80042001FBF5FEA410392EA030F7FEA226CDD
:1019D8007FEA236C6AD04FEA1262D2EB1363C1BF6D
:1019E800D218414048404140B8BF5B42192B88BFDC
:1019F800704710F0004F40F4000020F07F4018BFFF
:101A0800404211F0004F41F4000121F07F4118BF1E
:101A1800494292EA030F3FD0A2F1010241FA03FCC6
:101A280010EB0C00C3F1200301FA03F100F00043AE
:101A380002D5494260EB4000B0F5000F13D3B0F176
:101A4800807F06D340084FEA310102F10102FE2AE5
:101A580051D2B1F1004F40EBC25008BF20F0010055
:101A680040EA03007047490040EB000010F4000F03
:101A7800A2F10102EDD1B0FA80FCACF1080CB2EB96
:101A88000C0200FA0CF0AABF00EBC25052421843F5
:101A9800BCBFD0401843704792F0000F81F400019A
:101AA80006BF80F400000132013BB5E74FEA41036D
:101AB8007FEA226C18BF7FEA236C21D092EA030FD9
:101AC80004D092F0000F08BF0846704790EA010F53
:101AD8001CBF0020704712F07F4F04D1400028BF80
:101AE80040F00040704712F100723CBF00F5000062
:101AF800704700F0004343F0FE4040F40000704798
:101B08007FEA226216BF08467FEA23630146420243
:101B180006BF5FEA412390EA010F40F48000704756
:101B28004FF0000304E000BF10F0004348BF4042FC
:101B38005FEA000C08BF704743F0964301464FF038
:101B480000001CE050EA010208BF70474FF0000394
:101B58000AE000BF50EA010208BF704711F00043D5
:101B680002D5404261EB41015FEA010C02BF8446A5
:101B78000146002043F0B64308BFA3F18053A3F504
:101B88000003BCFA8CF2083AA3EBC25310DB01FA4B
:101B980002FC634400FA02FCC2F12002BCF1004FCF
:101BA80020FA02F243EB020008BF20F00100704760
:101BB80002F1200201FA02FCC2F1200250EA4C00B4
:101BC80021FA02F243EB020008BF20EADC707047FA
:101BD8004FF0FF0C1CEAD0521EBF1CEAD15392EA08
:101BE8000C0F93EA0C0F6FD01A4480EA010C4002E4
:101BF80018BF5FEA41211ED04FF0006343EA50103E
:101C080043EA5111A0FB01310CF00040B1F5000F7F
:101C18003EBF490041EAD3715B0040EA010062F12E
:101C28007F02FD2A1DD8B3F1004F40EBC25008BF18
:101C380020F00100704790F0000F0CF0004C08BF36
:101C480049024CEA502040EA51207F3AC2BFD2F103
:101C5800FF0340EAC250704740F400004FF0000311
:101C6800013A5DDC12F1190FDCBF00F0004070474B
:101C7800C2F10002410021FA02F1C2F1200200FA89
:101C880002FC5FEA310040F1000053EA4C0308BF50
:101C980020EADC70704792F0000F00F0004C02BFA1
:101CA800400010F4000F013AF9D040EA0C0093F01C
:101CB800000F01F0004C02BF490011F4000F013B76
:101CC800F9D041EA0C018FE70CEAD15392EA0C0FE4
:101CD80018BF93EA0C0F0AD030F0004C18BF31F04F
:101CE800004CD8D180EA010000F00040704790F025
:101CF800000F17BF90F0004F084691F0000F91F0C9
:101D0800004F14D092EA0C0F01D142020FD193EA8E
:101D18000C0F03D14B0218BF084608D180EA010016
:101D280000F0004040F0FE4040F40000704740F0F2
:101D3800FE4040F4400070474FF0FF0C1CEAD052C0
:101D48001EBF1CEAD15392EA0C0F93EA0C0F69D01C
:101D5800A2EB030280EA010C49024FEA402037D087
:101D68004FF0805343EA111143EA10130CF000407E
:101D78008B4238BF5B0042F17D024FF4000C8B426E
:101D880024BF5B1A40EA0C00B3EB510F24BFA3EB4E
:101D9800510340EA5C00B3EB910F24BFA3EB91031E
:101DA80040EA9C00B3EBD10F24BFA3EBD10340EA78
:101DB800DC001B0118BF5FEA1C1CE0D1FD2A3FF6BE
:101DC80050AF8B4240EBC25008BF20F00100704773
:101DD8000CF0004C4CEA50207F32C2BFD2F1FF0316
:101DE80040EAC250704740F400004FF00003013A47
:101DF80037E792F0000F00F0004C02BF400010F4EB
:101E0800000F013AF9D040EA0C0093F0000F01F0FE
:101E1800004C02BF490011F4000F013BF9D041EA20
:101E28000C0195E70CEAD15392EA0C0F08D1420253
:101E38007FF47DAF93EA0C0F7FF470AF084676E726
:101E480093EA0C0F04D14B023FF44CAF08466EE7FF
:101E580030F0004C18BF31F0004CCAD130F00042CD
:101E68007FF45CAF31F000437FF43CAF5FE700BF25
:101E78004FF0FF3C06E000BF4FF0010C02E000BF4E
:101E88004FF0010C4DF804CD4FEA40024FEA4103F0
:101E98007FEA226C18BF7FEA236C11D001B052EAA6
:101EA800530C18BF90EA010F58BFB2EB030088BF6C
:101EB800C81738BF6FEAE17018BF40F001007047DB
:101EC8007FEA226C02D15FEA402C05D17FEA236CBD
:101ED800E4D15FEA412CE1D05DF8040B704700BF04
:101EE800844608466146FFE70FB5FFF7C9FF00289B
:101EF80048BF10F1000F0FBD4DF808EDFFF7F4FFD4
:101F08000CBF012000205DF808FB00BF4DF808ED6C
:101F1800FFF7EAFF34BF012000205DF808FB00BF8F
:101F28004DF808EDFFF7E0FF94BF012000205DF8B1
:101F380008FB00BF4DF808EDFFF7D2FF94BF012062
:101F480000205DF808FB00BF4DF808EDFFF7C8FF5B
:101F580034BF012000205DF808FB00BF42000ED20C
:101F6800B2F1FE4F0BD34FF09E03B3EB126209D4CC
:101F78004FEA002343F0004323FA02F070474FF082
:101F88000000704712F1610F01D1420202D14FF0F7
:101F9800FF3070474FF00000704700BF00F026F890
:101FA8000C4880F30888002103E00B4B5B58435032
:101FB80004310A480A4B42189A42F6D3094A02E009
:101FC800002342F8043B084B9A42F9D318F060FC0E
:101FD8007047000000C000208CA403080000002007
:101FE8006413002064130020846500207047FEE716
:101FF80010B586B0002301244FF46022114801A9CE
:1020080001938DF80930039204938DF808408DF8F8
:10201800144027F03BFD0B48214627F05DFD094899
:1020280027F064FD074827F066FD0028FAD1054827
:1020380027F065FD034827F067FD0028FAD106B0B0
:1020480010BD00BF00240140014610B50D48012213
:10205800032327F067FD0B48012127F059FD7F2056
:1020680028F096FB0748022127F0A6FD0028F6D0A5
:102078000448022127F0A6FD0248BDE8104027F0D9
:1020880098BD00BF002401400C4A0C2303FB012328
:1020980010B59C880CB9588010BD5B8803F11304F7
:1020A800844204DA142B07D9133B834204DC0C2343
:1020B80003FB012102238B8010BD00BF842E00206A
:1020C8000A4B10B500241C7021464FF4E0720848F2
:1020D800FEF760F9074B43F604501C70064B1C7062
:1020E8000FF066FE054B187010BD00BFE415002008
:1020F800B0170020FB190020781900207A19002059
:10210800074B1978013101F01F011970054B1A7836
:102118008A4203D1013202F01F021A70704700BFD1
:1021280078190020FB19002010B50E4A0E2303FB76
:1021380000200D4A014614780C4A03FB042300F1E1
:102148000C0251F8044B914243F8044BF9D10A8828
:1021580000211A800E22FEF71DF9BDE81040FFF796
:10216800CFBF00BFE815002078190020B017002065
:10217800084B1A5C002352FA03F111F0010FD8B290
:1021880002D00130C0B270470133042BF3D10120D3
:10219800704700BFB61A002000F07F0000F57450A9
:1021A8002DE9F84309300C46154698460FF000FE15
:1021B80000284FD043F63C37002638460FF0F8FD8C
:1021C800C0B25FFA86F988B120280FD04FEA5909C2
:1021D8004BF2B77048440FF0EBFDC0B208B10228CB
:1021E80004D10123B340227813432370113743F6F7
:1021F800C43301369F42E0D14BF25E600FF0D8FD48
:10220800C0B280B120280ED02B784BF24D6043F03D
:1022180001032B700FF0CCFDC0B220B1202802D0F2
:10222800012388F800304BF28F600FF0C1FDC0B277
:1022380080B120280ED02B784BF24D6043F002037A
:102248002B700FF0B5FDC0B220B1202802D00123B9
:1022580088F80030BDE8F883034610465A1E10B5CA
:10226800032A1DD8DFE802F00F0F0209124A52783C
:1022780002F00202D2B2A2B111E00F4A527812F073
:1022880001020ED00BE00D4A927802F04002D2B261
:102298003AB10B4A127802F003029A4200D140B1D7
:1022A80000220848105C984203D00132052AF8D170
:1022B8000021084610BD00BF885F0020883A002032
:1022C8004F3E0020A8170020F8B5064643F63C35D7
:1022D800002428460FF06CFDC0B2E7B268B1202890
:1022E8000BD07F084BF2B77038180FF061FD01284A
:1022F80003D1A04033781843307001341135082CCD
:10230800E7D1F8BD03780E2202FB0313084AD3185D
:102318009978002351FA03F010F00100DAB202D0E4
:10232800501CC0B270470133082BF3D1704700BF6F
:10233800B01700202DE9F04101248C40284A294992
:102348000346E4B2107891F800C019E0264F0E2633
:1023580006FB0076F178A9B996F80680B8F1000F67
:1023680010D196F80580B8F1000F0BD196F80480CB
:10237800B8F1000F06D1F67926B9013000F01F0038
:10238800054626E0FBB1012B05D0022B06D10E2114
:1023980001FB007739790C4218D014E0042B04D1E2
:1023A8000E2101FB0077B9790CE0032B04D10E2133
:1023B80001FB0077797905E0052B07D10E2101FB98
:1023C8000077F97911B11570BDE8F081013000F09E
:1023D8001F006045BAD11570FF20BDE8F08100BF2D
:1023E800FB19002078190020B01700202DE9F043D0
:1023F800444D454B2A780E2101FB0232917A85B073
:102408000446984639B101390523594301F56E51FF
:10241800443189B201E043F6C431204604220FF06A
:10242800D8FC2B780E2505FB038393F80B80364EDA
:10243800344FB8F1000F25D131232371073363716D
:102448003B7801A86B430422F15E06F059FB3B7808
:1024580002A805FB03630222997A06F051FB3B7838
:102468000DF10A0005FB03650322697A06F048FBB3
:10247800A01D01A90922FEF763FA4FF00F0984F89D
:10248800108012E0B8F1010F0FD132232371053308
:1024980063713B784FF0080905FB036393F901303A
:1024A800E3713B785D43735BA371002320461A46B2
:1024B80012E010F8011BA1F13005EDB2092D04D886
:1024C800EB183029DBB203D004E037395B1800E0A1
:1024D8000A33DBB20132D2B24A45EAD10F21B3FB4B
:1024E800F1F10801411A5B1AC3F10F03DBB2092BA2
:1024F800A35401D8303300E03733A35405B0BDE806
:10250800F08300BFAE170020B0170020024B1A78E6
:1025180042F001021A7070471D1D002008B50C4BCF
:102528000C4A1B780E2101FB0323D97A21B101291A
:102538000CBF0921002100E0102140221346064863
:1025480006F002F9054B1A7842F002021A7008BD2B
:10255800AE170020B01700207B1900201D1D002099
:10256800034B1A7802F0F8026FF3C3021A7070472F
:102578001D1D0020024B1A7842F004021A707047A1
:102588001D1D0020024B1A7842F008021A7070478D
:102598001D1D002038B5114B1C7814F0010502D11F
:1025A800FFF7B4FF05E004F00405EDB21DB9FFF72D
:1025B800E1FF284638BD04F00805EDB215B9FFF76C
:1025C800E1FFF6E704F00204E4B21CB9FFF7A6FF46
:1025D800204638BDFFF7C4FF012038BD1D1D00206F
:1025E800014B1878704700BFE415002030B51E4B2A
:1025F80085B01B780446002B34D11C4D2B78034141
:1026080013F0010F2ED01A4B1A4A1B780E2101FB2A
:102618000323DA78024112F0010F1CD11B79034120
:1026280013F0010317D110F0010001F1F1014FEA95
:10263800540206D001320091019302926D20FE39B6
:1026480005E001320091019002923C200121032211
:102658000B460FF02BFC012313FA04F42B7823EA22
:1026680004042C7005B030BD7A19002071190020BF
:10267800FB190020B0170020037830B513F0010FC4
:10268800144A4FF00E0419D104FB01210133012231
:1026980012FA03F3CD7825EA0303CB7004780D7999
:1026A800A41812FA04F425EA04040C7103789B18A0
:1026B8009A408B7823EA02028A7030BD04FB01211C
:1026C800013B012212FA03F38A7822EA03038B7092
:1026D80030BD00BFB017002010B5002302785900A4
:1026E80052FA01F404F00304022C05D1013414FA5F
:1026F80001F122EA010202700133042BEED110BD70
:102708002DE9F04F85B00192BDF838201C46734B77
:102718000092DA78054612F020028B4640F0D88005
:102728008DF80E208DF80F208DF80D20DCB99B78E0
:1027380003F04003DBB21BB101238DF80F3020E01A
:10274800674B1B7803F04003DBB21BB101238DF804
:102758000E3016E00DF10F010DF10E020DF10D0313
:10276800FFF71AFD0DE0012C0BD19B7803F0400315
:10277800DBB223B90DF10F00FFF7A6FD01E08DF8DC
:102788000F409DF80F3023B99DF80E00002800F087
:10279800A28044B905F07F01490001F574510DF19B
:1027A8000A00663109E0012C0AD1E90101F51E4150
:1027B800E8310DF10A0001EB4B0102220FF009FB91
:1027C800BDF90A3013B9002C00F08480009B33B99E
:1027D800444B454F93F80080FFF792FC08E0434BC9
:1027E800434F93F8008008F1010202F01F021A70AB
:1027F8000DF10F00FFF770FF002C44D1BDF80A302F
:1028080069B240F6B83212EA210238BF4FF47A7240
:10281800D2180E2303FB08F3ADF80A20FA529DF8EC
:102828000F90224649460120FE18FFF715FD49463C
:10283800F07022460220FFF70FFD86F802903071F3
:102848009DF80E90224649460420FFF705FD4946AB
:10285800B071824622460320FFF7FEFC05F07F0593
:1028680070713572BAF1000F00D128B1214B1B7875
:1028780013B99DF80D3000E00023F37186F809B014
:10288800019AB2721CE0012C1AD10E2303FB08F343
:10289800BDF80A202046FA529DF80F600022314602
:1028A800FD18FFF7D9FC3146E87000220220FFF737
:1028B800D3FC00232871AE70AB716B71EB71AB72F6
:1028C8000E2303FB0877FC72009B0120BB8102E00A
:1028D800002000E0204605B0BDE8F08F883A0020CF
:1028E800885F002078190020B0170020E315002029
:1028F800E8150020021D002073B5154B04461B780F
:102908000E46D3B11348214622F0B1FD0546A0B9C1
:10291800012E04F1010606D12046FFF729FC009597
:102928000246812005E02046FFF722FC009502467A
:10293800982031462B46FFF7E3FE2146054822F052
:1029480080FD0548214602B0BDE8704022F084BDF4
:1029580079190020221C0020191A00202DE9F743BC
:102968007B4B04461B7843B17A4B1B7803F0240356
:10297800042B02D1002900F0E880774B774F1B78B1
:10298800002B00F0C7807648214622F070FD002811
:1029980040F0C08007F5C470214622F068FD8046EB
:1029A800002840F0B7803B1993F880302D2B01D0D8
:1029B800532B3AD16B4E357845B30FF05DFD04F1DA
:1029C8000108054650B12046FFF7D2FB337802468E
:1029D8001E33009393204146002307E02046FFF76B
:1029E800C7FB00950246414693202B46FFF788FE19
:1029F8000FF042FD014628B1337803201E330093BF
:102A0800002101E0009003200A4680E02046FFF7FD
:102A1800AFFB611C02462B4693200095FFF770FE22
:102A28000095032029462A4671E0542B09D12046F7
:102A3800FFF79EFBCDF800800246611C94204346B8
:102A480066E0462B474D20D12E78BEB10FF014FD1D
:102A580004F10109064648B12046FFF789FB2B78A7
:102A680002461E3300939A20494622E02046FFF78B
:102A78007FFB0096024649469A2025E02046FFF74C
:102A880077FB009602469A2039E02E78002E2CD04B
:102A98000FF0F2FC04F11C09064660B12046FFF76E
:102AA80067FB2B7802461E3369F07F000093C0B2A3
:102AB800611C434609E02046FFF75AFB024669F0CD
:102AC8007F000096C0B2611C3346FFF719FE0FF075
:102AD800D3FC21B2024628B12B7803201E33009381
:102AE800002214E00090032011E02046FFF740FB8D
:102AF800024604F11C0060F07F000096C0B2611C21
:102B08003346FFF7FDFD0096032021463246012398
:102B1800FFF7F6FD124821463F1922F092FC97F87C
:102B280080302D2B0AD0532B08D0542B06D0462B9F
:102B380004D00D48214622F09AFC30B10B482146BA
:102B480003B0BDE8F04322F087BC03B0BDE8F083D2
:102B5800E6150020101C002079190020B02C002058
:102B6800221C00207A1C0020382E00201A1C00206D
:102B7800002302780E2101FB0232044901338A182E
:102B88000021062B9170F4D1704700BFB0170020C8
:102B9800064B00201870064B1A78064B1B789A4291
:102BA80002D00146FFF7C6BBFF207047E41500209E
:102BB80078190020FB1900200121814038B5114BFC
:102BC800C9431A78104BC9B202F0030203F5E07446
:102BD800012A04D1DD7801EA0505DD7005E0022A45
:102BE80003D11D7901EA05051D710E33A342EFD10A
:102BF800FFF7FCFC43F604500FF0DAF8034B1870AB
:102C080038BD00BF4F3E0020B01700207A190020C1
:102C18002DE9F743A34D8DF807002B78A24C1BB183
:102C28002378C2B29A4204D043F604500FF0C0F899
:102C380028709DF8073023709C4C2278072A00F2F0
:102C48002D81DFE812F008002400360054005D00F2
:102C580072008D00BA00964A3C211170954A1946B7
:102C6800107800F00300FFF765FB934BFF281870FE
:102C780000F0368121F0F2F8904B002093F8742090
:102C880042F0010283F874208D4B187064E0884B81
:102C98001B78002B00F0248121F0A8FA012840F0CD
:102CA8004D812378142201332370864B01381A7022
:102CB80047E17F4B1B78002B00F01281814E307862
:102CC80008B901234AE021F091FA022804D021F042
:102CD8008DFA032840F0328121F0C0F823780422CD
:102CE800013323701D233370774B1A7026E1704B24
:102CF8003C221A707548FFF779FB2378013323705B
:102D08006B4B1B78002B00F0EB806E4B1D78002D71
:102D180040F014811020FFF73DFC002800F01181DD
:102D280023782846013323700BE1614B1B78002B75
:102D380000F0D68005F072FD002800F00281614B9A
:102D48007D221A705E4B002018705C4B93F874203B
:102D580042F0010283F87420237801332370F0E0F5
:102D6800534B1B78002B00F0BB8021F03FFA012861
:102D7800544E03D021F03AFA03280FD19DF80720CA
:102D8800012111FA02F2524B197821EA02021A7053
:102D980064233370237801332370CFE03078002820
:102DA80040F0CC80484A032323701378013BDBB200
:102DB8001370002B00F09480C3E0404A414E92F813
:102DC8006A201AB13278002A40F0B88000223270A6
:102DD800013212FA03F3DFF8E0803E4F98F8001052
:102DE8004FF00E0909FB0172DB4392F803E0DBB2F6
:102DF80003EA0E0E907882F803E092F804E003EA02
:102E08000E0E0340937082F804E00DF10700FFF7FF
:102E180033FC98F8003009FB0372D278DFF89490FD
:102E28002AB999F8002002F00302012A0AD00E22DA
:102E380002FB03721279B2B999F8002002F003027A
:102E4800022A10D10E2202FB0377BA785AB9224F10
:102E58003A789A4207D11848FFF78AFE3B7801333F
:102E680003F01F033B7099F800009DF8071000F06D
:102E78000300FFF75FFA144B0422FF281A7088F842
:102E88000000164B42D0987800F04000C0B20028ED
:102E98003CD1032323701A33337052E00020207092
:102EA8004FE000BF7A190020E7150020E415002044
:102EB800721900204F3E0020AE170020D43D00209C
:102EC800E5150020E2150020701900207B1900206C
:102ED80071190020B0170020FB190020883A002043
:102EE800FFF73EFB0023237020F0B8FF2B78013B4F
:102EF800DBB22B702BB1144B9B7803F04003DBB291
:102F0800F3B19DF80700FFF757FE19E09B780E4ACA
:102F180003F04003DBB22BB1136843F400031360E2
:102F2800FFF7CEF8FFF71CFB20F098FF0023237073
:102F380043F604500EF03CFF287001E0002000E04A
:102F4800FF20BDE8FE8300BF883A0020044B1A78B2
:102F58000AB1013A1A701B780BB9FFF72DBE7047FA
:102F68007A190020044A054B10781B7803EA5010A0
:102F780000F00100704700BF883A0020E81B0020DD
:102F8800044B054A1B781078C3F3400303EA10107A
:102F9800704700BFE81B0020883A0020034B044A12
:102FA8001B78D078C3F3800318407047E81B0020D3
:102FB800883A0020044B054A1B78D078C3F3C00335
:102FC80003EA5000704700BFE81B0020883A002041
:102FD800044B054A1B78D078C3F3001303EA90002A
:102FE800704700BFE81B0020883A0020044B18787F
:102FF800044BDB785B005BB2DB1103EAD01070474F
:10300800E81B0020883A002008B50E2104481DF06E
:103018005BF9044B5B7803EA000000F0010008BD8F
:10302800041A0020E81B002070B500241BE030467D
:10303800E9B21DF087F980B14FF436636343342257
:1030480002FB05330A4AD3181B7A13F0010F04D088
:10305800084B1878C0F3001070BD0135382DE6D143
:103068000134022C02D0E6B20025E0E7002070BD52
:10307800283F0020E81B002008B51CF07FFA034B0E
:103088001B7800EA931000F0010008BDE81B00203F
:10309800044B054A1B78D078C3F3401303EAD000E9
:1030A800704700BFE81B0020883A00202DE9F74F41
:1030B800FFF758FF8246FFF763FF8346FFF76EFF6F
:1030C8000190FFF777FF8146FFF782FF0446FFF77D
:1030D800ABFF0546FFF7DCFF8046FFF7CDFF07464D
:1030E800FFF784FF0646FFF78FFF019B45EA0404BC
:1030F8009B0043EA4B0343EA0A0343EAC90343EA52
:10310800481343EA871343EAC61343EA0023E0B2AD
:1031180043EA0010BDE8FE8F044B987800F00F00DA
:10312800A0F10203584240EB03007047561A0020F2
:10313800044B987800F00F00A0F10102504240EBD8
:1031480002007047561A0020044B987800F00F00D0
:10315800A0F10301484240EB01007047561A0020D5
:10316800054B987800F00F00A0F1060CDCF1000088
:1031780040EB0C00704700BF561A0020514AF0B5CA
:1031880013781446012B29D003D3022B40F09880E2
:103198005EE04D484D4B047819786FF3C304047012
:1031A80001F0F80158786FF3C301197000F080013D
:1031B800C9B2002900F08480012111709C78062290
:1031C80004F00F04544302464148005D60F30602D0
:1031D8005A701A7861F302021A70F0BD3B494D78B3
:1031E8000B4625F07F00002838D00A7802F0080244
:1031F800D2B222B9344A117841F0080111709A7894
:1032080002F00F02012A04D12F4A117841F001017E
:10321800117015F07F0F53D119789E7801F00700CF
:10322800062206F00F0602FB0606294F5D78BE5DF2
:10323800013066F3060500F007005D7090FBF2F5BB
:1032480002FB150262F30201197002232370F0BD1C
:103258001E494D780B4625F07F0028B98B7860F31E
:1032680003038B701070F0BD174A11786FF3C30118
:103278001170997801F00F01012903D111786FF3CA
:103288000001117015F07F0F1AD119789E7801F09E
:103298000700062206F00F0602FB06060C4F5D78B3
:1032A800BE5D013066F3060500F007005D7090FB17
:1032B800F2F502FB150262F3020119700123237073
:1032C800F0BD00BFA51A0020181A0020561A0020C9
:1032D80038A8020810B51F4A1F4B92F9031009B10C
:1032E800002231E008B1032119701978032930D878
:1032F800DFE801F00209192C1178002929D01548B6
:1033080081700121197092F90200124920B1134B02
:103318001A786FF3861217E0487808B9032213E089
:1033280088700221197092F902100A4889B90B4A6B
:10333800147861F386141470026861F30F22D1B215
:1033480061F31742026001221A7010BD002111605A
:10335800197010BD7C1C0020131A0020B43C0020FA
:1033680070B543F6EF23044643F6F020012A08BF60
:1033780018460D460EF01CFD2678C0B20640164CC5
:103388000CD001201DF0BEF943F6EE200EF010FD22
:10339800236860F307036FF30F2314E02B781842B8
:1033A80012D030461DF0AEF90C4B43F6EE201A88C9
:1033B80066F34D321A800EF0FBFC2368C0B260F34E
:1033C800070360F30F23236094F9003013B1024B15
:1033D8000F22DA7070BD00BF7C1C0020101C00207A
:1033E80008B543F6FB200EF0E3FC014B187008BD4E
:1033F800141A0020014B1870704700BFF21B002000
:103408002DE9F0474FEAD2084BF25F79C14402F048
:1034180007030446012748460D469F4016460EF00E
:10342800C7FCFFB2C1B215B921EA070100E0394370
:1034380008F5D048484608F14E080EF0AFFC404663
:103448000EF0B6FCC1B214B921EA070100E0394315
:1034580040460EF0A3FC254305D106483146BDE899
:10346800F04721F0F9BF03483146BDE8F04721F0A5
:10347800E8BF00BF591A0020024B1A5C6FF3030221
:103488001A547047FF1A002070B50C46C10001F5A8
:10349800D2411B483F3108220EF09BFC00251848FA
:1034A8002946EEB221F0E3FF08B9237823BB154B78
:1034B8002278EB5C1A421FD13046FFF7DDFFF60891
:1034C8004BF25F7030180EF073FC05F00703C0B2C2
:1034D800184110F0010F0FD10B48294621F0C7FF02
:1034E80050B12946084821F0B7FF074B06F5D040F0
:1034F8004E30995D0EF052FC0135402DCFD170BD94
:10350800F41B0020B61A0020591A002038B546F6D8
:10351800960540242046FFF7AFFFA5F5D043094A9A
:10352800563BD15C11F0100F06D06FF30411D15443
:10353800284600210EF032FC0134E4B20135E92CB2
:10354800E8D138BDFF1A00203F287FB5054607D8C7
:1035580000F5E440C1300EF02BFCC3B22BB92AE1D0
:10356800994A1478002C00F02B81984E725D02F075
:103578000F014C1C04F00F0464F303023F2D725535
:1035880033D8002C00F01C8101339C4240F0158197
:103598008F4B5A1992F88020522A725D03D161F339
:1035A8000302725509E16FF30302EC081B19725507
:1035B80093F8902105F0070352FA03F313F0010F73
:1035C80040F0FD802946834821F03BFF814B04F5FC
:1035D800D040195D4E3001240EF0E0FB2D19022376
:1035E8000093019402951820CEE0002C00F0E880AA
:1035F800754B1B7801339C4240F0DF80735D05F505
:10360800D0406FF303035630012173550EF0C6FB0B
:10361800735D43F010037355A5F14003DBB2032B30
:1036280007D8042200920133023201920293192032
:103638002FE0A5F14803DBB2032B07D80422009240
:1036480001330332019202931A2060E0A5F150037E
:10365800DBB2012B07D80422009201330332019216
:1036680002931B2053E0572D07D104230093012414
:10367800033301930294212086E0A5F15B03DBB2BA
:10368800012B09D8042200920133023201920293DD
:1036980022200121033A8AE05D2D06D104230093FC
:1036A8000193043B029328467FE05E2D07D1042353
:1036B800009301330193053B02935E2075E0A5F169
:1036C8005F03DBB26F2B09D80422009201339218F2
:1036D8000192029333200121053A68E005F1310394
:1036E800DBB2032B07D80422009201330332019284
:1036F80002935F200BE005F12903DBB2012B09D807
:1037080004220092013303320192029360200121C6
:10371800043A4CE0DA2D07D1042300930124043B3A
:103728000194029361202FE0D92D07D1042300933F
:10373800023B0193023B0293622036E0DD2D08D163
:10374800042300930322043B019202936320012186
:103758002DE0DB2D06D104230093043B0193029353
:10376800642022E0DC2D06D104230093043B01935E
:103778000293702019E0DE2D0CD10423009301245C
:1037880002330193029468202146032223460EF057
:103798008DFB15E01E35EDB2012D10D804230093E2
:1037A80001350233019302956A20012103220B4659
:1037B8000EF07CFB03E01C4602E0002400E001243C
:1037C800204604B070BD00BF00000020FF1A002092
:1037D800B02C0020591A0020024B185CC0F30010CE
:1037E800704700BFFF1A0020F8B508220E460021D6
:1037F8000746FCF7CFFD46F63F15002433782341F2
:1038080013F0010F08D02946064808220EF0E1FA05
:103818003846044921F0E3FD01340835042CEDD184
:10382800F8BD00BFFE1B0020024846F64E010822E4
:103838000EF0CFBA591A002070B5044600F56A5048
:1038480044300EF0B5FA0B4D06462B7813F0010FF5
:1038580002D1CC2022F030FC2B8843F001032B80CE
:10386800054B1E55054B13F8242042F0010203F8BE
:10387800242070BD101C00203A1A0020291A0020AC
:10388800024B185C084100F001007047B61A00208E
:1038980070B505460024094BE0B2E618E35C4BB16D
:1038A8002946FFF7EDFF28B100233370044821466D
:1038B80021F0D2FD0134402CEDD170BD321C002026
:1038C800461A002038B5054600242846E1B2FFF71D
:1038D800D7FF10B1044BE35C23B90134042CF4D1B5
:1038E800002038BD012038BD3A1A002038B50546F9
:1038F8000EF0C2FDA0B100242846E1B2FFF7C0FFD8
:1039080040B1084B13F8243013F0010F02D0064BD6
:10391800E35C23B10134042CEED1002038BD012032
:1039280038BD00BF291A00203A1A0020F8B51148FE
:1039380000214022FCF72EFD46F63F150024012702
:103948000D4829460822A7400EF043FAFFB2002688
:103958000948314621F08BFD20B1064BF25C47EA5D
:103968000202F2540136402EF2D101340835042CFB
:10397800E5D1F8BDB61A0020FE1B00202DE9FF4155
:1039880000263446B0461A4B1B78234113F0010237
:10399800184B23D0184F1D5D17F82430A84538BFA1
:1039A800A84613F0010F1AD0CDB965F3000307F844
:1039B800243023B20122F71902935B2029462B46B3
:1039C800009201950EF072FA7B78B878F97818436E
:1039D800621C2B460095FEF793FE00E01A55013451
:1039E8000436042CCFD1054B83F80080BDE8FF8155
:1039F800141A00203A1A0020291A0020121A00204E
:103A080010B50C4B1B78A3B10B4B1B788BB1002462
:103A18000A48214621F02BFD40B10948214621F0F2
:103A280026FD18B920460121FEF798FF0134402CE5
:103A3800EED110BD79190020E61500201A1C0020CF
:103A4800AA2300202DE9F043324C334A238800266C
:103A58006FF386136FF3C4032380304B304F85B068
:103A680016701E709146984617F8013B5BB3227892
:103A7800D20052B243EAA2122388402E62F3C40352
:103A880043F0400323801ED000253046E9B2FFF7FB
:103A9800F7FEA8B117F8013C13F0010F06D0012278
:103AA800AA4099F800100A4389F8002013F0020F81
:103AB80006D00123AB4098F80020134388F8003063
:103AC8000135042DE1D10136F6B2412ECCD123784F
:103AD80003F04005EDB2D5B903F02403042B0BD154
:103AE800FFF78EFFFF2300934020294601222B4633
:103AF800019502950EF0DAF9238800226FF3451339
:103B08006FF382036FF3C4032380064B1A7005B06A
:103B1800BDE8F083101C0020503C00206D3C0020C4
:103B2800641A0020F31B002010B500240548214624
:103B380021F09DFC08B9044BE0540134402CF5D128
:103B480010BD00BFEA1B0020641A002010B51278CF
:103B580004469DF80810DAB1D3B111B10D4921F02E
:103B680033FCACB1082246F64E010B480EF031F991
:103B78002146094821F033FC0749082246F64E0041
:103B88000EF021F905480449BDE8104021F03DBC7C
:103B980010BD00BF482E0020FC190020591A002033
:103BA80030B5064B04781D7824EA05040C700178BA
:103BB8001B7823EA0103137030BD00BF141A0020DC
:103BC80038B50A4D002415F8013F2D2B09D0532B89
:103BD80007D0542B05D0462B03D00548214621F0A9
:103BE8003BFC0134402CEED138BD00BF2F2D002006
:103BF8001A1C002010B50F4821F0DEFB00240E48E7
:103C0800214621F034FC80B10C4BE31893F8803046
:103C1800482B06D003D82D2B03D0462B00E0542B7D
:103C280003D10448214621F00CFC0134402CE6D194
:103C380010BD00BFA61A00201A1C0020B02C0020BE
:103C4800094A0A4B117831B1997801F00F01814284
:103C580001D0002111709A7860F303029A705A78A3
:103C680042F080025A707047A51A0020561A0020A8
:103C78002DE9F0431F4685B07C4BDDF830901546A2
:103C880004461A7888460023794911F8231011F060
:103C9800010F05D001219940C1F10F0101EA02028B
:103CA8000133042BF0D1734B1A70002C00F087807D
:103CB80014F0010F0CD00121FF230026009352209D
:103CC8000B460A46019602960EF0F0F86A4B1E70F3
:103CD80014F0020F0DD0FF2301210093FF3B019345
:103CE80002930A460B4653200EF0E0F8624B01227D
:103CF8001A7014F0040F0DD0FF2301210093FF3B2D
:103D0800019302930A460B4654200EF0CFF85A4B03
:103D180002221A7014F0080F0DD0FF23012100931E
:103D2800FF3B019302930A460B4655200EF0BEF85E
:103D3800514B03221A7014F0100F0DD0FF230121EC
:103D48000093FF3B019302930A460B4656200EF060
:103D5800ADF8494B04221A7014F0200F0DD0FF2340
:103D680001210093FF3B019302930A460B4657201B
:103D78000EF09CF8404B05221A7014F0400F0DD03D
:103D8800FF2301210093FF3B019302930A460B4650
:103D980058200EF08BF8384B06221A7014F0800F5A
:103DA8000DD0FF2301210093FF3B019302930A46A4
:103DB8000B4659200EF07AF82F4B07221A70B8F1EB
:103DC800000F1CD02C4B09221A70002438462146BB
:103DD80021F04DFB60B1FF230093FF3B0193631C6F
:103DE8001BB2012102935A200A460B460EF05EF8D8
:103DF80021463846013421F02FFB402CE6D1CDB1C5
:103E080000244846214621F032FB80B1012D0ED115
:103E180004230093631C1BB20826029374202B46CC
:103E28002946032201960EF041F8134B1E70013407
:103E3800702CE6D10F481149114AFFF7B1FE114B1A
:103E480000221A7001320092063201920832029260
:103E58000A490B4A074809F0BDFD0B4B3C2251208B
:103E68001A7005B0BDE8F0430EF0F2BB141A00203A
:103E7800291A0020881D002049640020711E002096
:103E8800641E00204D1D0020391A002037B5FFF7A9
:103E98000DF904460E4821F0BDFAD0F1010538BFEE
:103EA80000250C480E211CF00FFA10B114F4807F85
:103EB80003D124B95DB1224602E0012200E00022CC
:103EC800044B204600932946014BFFF7D1FE3EBD27
:103ED800F71A0020041A0020054B03EBD00393F8CF
:103EE800903100F0070053FA00F000F0010070472D
:103EF800B02C002010B50F4B04461B7813F00103BB
:103F080015D0FFF7DFFC28B90B4B1B1993F880304D
:103F1800462B0DD10EF0B0FA18B92046FFF7DCFF9A
:103F280030B10648214621F08CFA012010BD184610
:103F380010BD00BF101C0020B02C0020F71A002074
:103F4800024B1878003818BF01207047391A002032
:103F580010B5034C04EB830358709970DA7010BDE8
:103F6800291A002010B500240948002100190E2242
:103F78000E34FCF70FFAB4F5E07FF5D1054A0023BB
:103F88001370054A002199520233AA2BF9D110BDAA
:103F9800E8150020E3150020E61E0020044B1878E1
:103FA80000F02400A0F10403584240EB03007047DE
:103FB800101C00207FB5474B04461B780E46AA2BE1
:103FC80078D04548214621F052FA0546002871D19B
:103FD8002046FFF78FFF00286DD14048214621F089
:103FE80046FA50B93E48214621F041FA054620B923
:103FF8002046FFF7A9FA00285DD13A4B1B7823B970
:10400800394B1B7813F0010F09D1384BDB7803F0DB
:104018002003DBB21BB9364B032283F84020012E64
:1040280005D82E48214621F022FA40B142E0022E5E
:1040380007D12B48214621F01AFA10B13AE0274857
:1040480000E02748214621F0FCF92A48214621F0C2
:1040580003FA022E15D10125294603222B46009684
:104068004A206619019502960DF020FF2046FEF7BA
:104078007FF800230246314618200093FEF740FBE4
:1040880019E0012E09D102230093631C02930196C3
:10409800122031460322334609E07EB9012102236A
:1040A8000093631802930191112003220B460DF02F
:1040B800FDFE03E00025284604B070BD2046FEF74B
:1040C80057F8024601200023211800930125FEF726
:1040D80017FBF0E7F21B0020591A0020191A0020DC
:1040E800721C0020141A0020E11E0020883A0020CB
:1040F800641A0020221C00202DE9FF4704460D46C3
:104108007548214621F0B3F98146002840F0DF8048
:104118002146714821F095F97048214621F09CF913
:104128006F4E0DBB01274FF00208E3190293424678
:10413800032039463B46CDF8008001970DF0B6FEC6
:10414800327862B10EF098F9024630B133784046C1
:104158001E33009321462A4604E0009000E00092B6
:10416800404621463B4628E0012D2BD15D4B04F506
:10417800E440C1301F5D0DF01BFE07F00F078742BA
:1041880009DA631C022202930E2029462B4600926C
:1041980001950DF08BFE327892B10EF06DF9024662
:1041A80038B14F4B0D201B7821461E330093002257
:1041B80002E000900D2021460123FEF7A1FA5EE0FF
:1041C8000092F7E7022D0BD101230193E318029324
:1041D800142049462A464B4600950DF067FE4EE0EE
:1041E800032D4CD101272A464FF0020804EB070A99
:1041F8004D2039463B46CDF800800197CDF808A000
:104208000DF054FE35783DB30EF036F9024630B164
:10421800337840461E33009321464A4602E0009018
:10422800214640463B46FEF76BFA0EF025F9671C1F
:10423800054648B12046FDF79BFF337802461E33FA
:1042480000931A2039462CE02046FDF791FF00958F
:10425800024639461A202DE021462A463B4640466A
:104268000095FEF74DFA2046FDF782FF51460246BB
:104278002B461A200095FEF743FA384628E0357891
:10428800EDB10EF0F9F804F11C06054658B12046C8
:10429800FDF76EFF124B02461B7830461E33009323
:1042A800611C002307E02046FDF762FF00950246E7
:1042B8003046611C2B46FEF723FA012008E0204611
:1042C800FDF756FF0095024604F11C00F1E70020B7
:1042D80004B0BDE8F08700BF1A1C0020221C002093
:1042E8007A1C0020FF1A0020064B1B1893F8400187
:1042F800492804D0452814BF032002207047012014
:10430800704700BFB02C00202DE9F041244F002455
:104318003C702448214621F0AAF8E5B2224B002837
:1043280037D01E5D3B789E4200D303B93E70002E05
:1043380030D131461C484022FCF72CF81B4B1C4856
:1043480003EBD50393F8888104F0070348FA03F8D0
:10435800214608F0010821F08AF868B9B8F1000F81
:1043680002D02846022101E028463146FFF7C4FE64
:1043780028460EF06DF90DE0B8F1000F0AD1284675
:10438800FFF7B2FF0B4BDB7803F02003DBB20BB96E
:10439800094B18550134402CBBD1BDE8F08100BF52
:1043A8007A1C0020461A0020321C0020B02C002065
:1043B8001A1C0020883A0020641A00202DE9F04FCA
:1043C800914B8BB01B7813F0010F06D08F4B1A78E6
:1043D8006FF386121A7001F0C2BA8D498D4A0B78B4
:1043E80010788D4D984218BF8C49137018BF0B7008
:1043F8006B7803F00803DBB24BB143F6CF200DF026
:10440800D7FC864B18702B886FF3CB232B80844BFB
:104418001B78AA2B08D18349AA3B0B702B8843F041
:1044280080032B8000F0F4BE6A787B4B02F0100208
:10443800D2B27D4CA2B11A886FF30C321A807B4B32
:104448001B7823B97A4B1B7813F0010F08D1E37856
:1044580003F02003DBB21BB9764B032283F840201C
:104468002368754F6FF3186323603A7802F00202ED
:10447800D2B232B96B494A781AB16B4A43F08073A9
:104488001360E67816F0010648D05D20FFF7A4F91E
:1044980000285AD16B78DFF8808103F00203DBB281
:1044A8002BBB5D30FFF750F8064600BBB8F800306C
:1044B800012143F40073A8F8003004230322009379
:1044C800019302900B460D200DF0F0FC45200EF0F4
:1044D800BFF83146012233460D200096FEF710F949
:1044E80009203146324601230096FEF709F96B7818
:1044F80003F00203DBB243B34C4B1B7823B94C4B9C
:104508001B7813F0010F20D1E37803F02003DBB20E
:10451800DBB9484B032283F8402016E06B7803F0A0
:104528000203DBB26BB13146324601230A20009602
:10453800FEF7E6F88D203146012233460096FEF755
:10454800DFF82B886FF349232B802368354A6FF3F4
:104558005963236093787BB1D37823B93B7813F000
:104568000C0F05D108E03B7803F00C03042B03D0B3
:10457800236843F000732360E17801F00201C9B2B7
:1045880000295BD05E20FFF727F9002865D16B78FA
:10459800214F03F00403DBB2EBB95E30FEF7D4FF22
:1045A8000646C0B93B88012143F480633B8004235D
:1045B800009301330322019302900B4617200DF05C
:1045C80075FC45200EF044F80D2031460122334693
:1045D8000096FEF795F86B7803F00403DBB2002B26
:1045E8003BD0124B1B7823B9114B1B7813F0010FEA
:1045F80033D1E37803F02003DBB273BB0D4B032206
:1046080083F8402029E000BF891D0020B43C002029
:10461800FC1B0020FD1B0020101C00207B1C002020
:10462800F21B002064130020883A0020141A00208E
:10463800E11E0020641A0020AE2C00206B7803F0E5
:104648000403DBB22BB18D2001220B460091FEF74B
:1046580057F82B886FF38A232B8023684FF05F0B62
:104668006FF3DF732360002696E00698F9B21BF01B
:1046780069FE002875D04FF436637343342202FB79
:104688000733A749A8F15E0ACB1803F108021B7A81
:104698005FFA8AFA13F001034DD02368404643F0CD
:1046A800004323600592FFF797F8059A002864D124
:1046B800937813F0040F20D14046FEF745FF059A82
:1046C8008146D0B99378012143F004039370042301
:1046D8000093DB180322019332200B46CDF808A083
:1046E8000DF0E4FB4A200DF0B3FF0C2051460122E7
:1046F8004B46CDF80090FEF703F84FF4366373434A
:10470800342202FB0733864AD3189B7A13F0040F2E
:1047180033D0844B1B7823B9834B1B7813F0010FDC
:104728002BD1E37803F02003DBB233BB7F4B0322AA
:1047380083F8402021E0927812F0040F05D08C20F5
:10474800514601220093FDF7DBFF4FF436637343B4
:10475800342202FB07337249CB189A7A6FF382022C
:104768000AE04FF436637343342202FB07336C4A82
:10477800D3189A7A60F382029A72013708F1010815
:10478800382F5FFA88F87FF470AF01360BF1380BD9
:10479800022E5FFA8BFB04D0F3B20693D8460027AB
:1047A80063E72368624923F080636FF39E73236095
:1047B8000B79002B00F0EF835E4ADFF87CB106929C
:1047C8004FF0CF0800271BF8011F3E46013700298C
:1047D80052D0236808F1710A43F080635FFA8AFABD
:1047E80023605046FEF7F8FF00285CD12923734365
:1047F800DFF8489119F8032012F0100F23D1504622
:104808000593FEF7A1FE059B8246E0B919F803203F
:10481800012142F0100209F8032004230093023317
:1048280001933BB2032202930F200B460DF03EFB8F
:1048380045200DF00DFF0D20514601225346CDF8BD
:1048480000A0FDF75DFF2923734319F8033013F027
:10485800100F28D0334B1B7823B9334B1B7813F038
:10486800010F20D1E37803F02003DBB2DBB92F4B33
:10487800032283F8402016E029237343DFF8BC9015
:1048880019F8033013F0100F05D08D2001220B46C4
:104898000091FDF735FF2923734319F803206FF3BF
:1048A800041209F80320069A12F8011F069200293B
:1048B80046D02368404643F080432360FEF78CFFD0
:1048C800002854D14FF0290909FB06F9DFF86CA03C
:1048D8001AF8093013F0200F49D14046FEF734FE8C
:1048E8000646002843D11AF80930012143F0200375
:1048F8000AF8093004230093033301933BB20322DF
:1049080002934B200B460DF0D1FA50200DF0A0FE7B
:1049180019203146012233460096FDF7F1FE26E0C4
:10492800283F0020141A0020E11E0020641A0020ED
:1049380064130020763B00209B3B0020A53B002011
:1049480029237343DFF80C9319F8033013F0200F71
:1049580005D0992001220B460091FDF7D1FE2923AD
:104968005E4319F806306FF3451309F8063008F16D
:104978000108042F5FFA88F87FF425AFAE4ADFF804
:10498800D8B206924FF05008043F1BF8011F3E466C
:104998000137002952D02368A8F16E0A43F08063DA
:1049A8005FFA8AFA23605046FEF716FF00285CD1AA
:1049B80022237343DFF8A49219F8032012F0400F62
:1049C80023D150460593FEF7BFFD059B8246E0B90B
:1049D80019F80320012142F0400209F803200423BA
:1049E8000093023301933BB20322029369200B46E2
:1049F8000DF05CFA45200DF02BFE0D2051460122EA
:104A08005346CDF800A0FDF77BFE2223734319F827
:104A1800033013F0400F28D0884B1B7823B9884BFC
:104A28001B7813F0010F20D1E37803F02003DBB2E9
:104A3800DBB9844B032283F8402016E0222373431A
:104A4800DFF8189219F8033013F0400F05D08D20C5
:104A580001220B460091FDF753FE2223734319F8F8
:104A680003206FF3861209F80320069A12F8011F33
:104A78000692002935D02368404643F080432360DE
:104A8800FEF7AAFE002843D14FF0220909FB06F9D8
:104A9800DFF8C8A11AF8093013F0200F38D14046C2
:104AA800FEF752FD064698BB1AF80930012143F07B
:104AB80020030AF8093004230093033301933BB21F
:104AC8000322029310200B460DF0F0F950200DF050
:104AD800BFFD19203146012233460096FDF710FE2E
:104AE80016E022237343DFF8749119F8033013F0AA
:104AF800200F05D0992001220B460091FDF700FEFA
:104B080022235E4319F806306FF3451309F806307F
:104B180008F10108022F5FFA88F87FF436AF4A4B94
:104B28001978002946D02368DE2043F0806323608B
:104B3800FEF752FE00284CD1444B1A78984612F0E2
:104B4800400F20D1DE30FEF7FFFC0746D8B998F8B1
:104B58000030012643F0400388F800300423009316
:104B680002333146032201936720334602960DF043
:104B78009DF945200DF06CFD0D20394632463B4627
:104B88000097FDF7BDFD98F8003013F0400F20D0D6
:104B98002A4B1B7823B92A4B1B7813F0010F18D125
:104BA800E37803F02003DBB29BB9264B032283F89A
:104BB80040200EE0254E337813F0400F05D08D20AD
:104BC80001220B460091FDF79BFD33786FF38613A6
:104BD80033701F4B1978002942D02368572043F0BF
:104BE80080432360FEF7F8FD002848D1174E33783C
:104BF80013F0200F43D15730FEF7A6FC07460028D4
:104C08003DD13378032243F0200333700423012677
:104C180000930333314601931F20334602960DF06B
:104C280045F950200DF014FD1920394632463B460F
:104C38000097FDF765FD22E08B3A0020141A00204A
:104C4800E11E0020641A0020D83A0020F13A002022
:104C5800DD3A0020A53B0020693B0020263B0020D0
:104C6800834E337813F0200F05D0992001220B468C
:104C78000091FDF745FD33786FF3451333704FF01E
:104C880000084FF05B094FF0D70A4646794B08F108
:104C98000108F15C784F002949D02368484643F061
:104CA80080632360FEF798FD002852D124237343C4
:104CB800FA5C12F0200F22D148460593FEF744FC17
:104CC800059B8346D8B9FA5C012142F02002FA54C8
:104CD80004230093023301930FFA88F3032202930B
:104CE80020200B460DF0E2F845200DF0B1FC0D2018
:104CF800594601225B46CDF800B0FDF701FD24239B
:104D08007343FB5C13F0200F23D05C4B1B7823B953
:104D18005B4B1B7813F0010F1BD1E37803F02003E2
:104D2800DBB2B3B9574B032283F8402011E02423A8
:104D38007343FB5C13F0200F05D08D2001220B4636
:104D48000091FDF7DDFC24237343FA5C6FF34512F1
:104D5800FA544D4BF15C002933D02368504643F098
:104D680080432360FEF738FD00283ED1242303FB4F
:104D780006735A7812F0200F37D150460593FEF784
:104D8800E3FB059B834680BB5A78012142F0200251
:104D98005A7004230093033301930FFA88F3032214
:104DA80002934C200B460DF081F850200DF050FC7A
:104DB8001920594601225B46CDF800B0FDF7A0FC4A
:104DC80013E0242303FB06735B7813F0200F05D050
:104DD800992001220B460091FDF792FC242303FB46
:104DE80006735A786FF345125A70284B2422F35CE5
:104DF800002B4FD07243BB5CC3F3801BBBF1000F89
:104E08001DD123490978D1B143F04003BB54042391
:104E18000093DB18012101930FFA88F30322029310
:104E28002F200B460DF042F847200DF011FC092009
:104E3800414601225B46CDF800B0FDF761FC242312
:104E48007343FB5C13F0400F35D00C4B1B7823B930
:104E58000B4B1B7813F0010F2DD1E37803F02003DF
:104E6800DBB243BB074B032283F8402023E000BF9B
:104E7800F13A0020743B0020903A0020141A0020D8
:104E8800E11E0020641A00206C3B0020DF3A00205D
:104E9800E63A00207243BA5C12F0400F05D0892030
:104EA800414601220093FDF72BFC24237343FA5C4F
:104EB8006FF38612FA5401360AF1010A09F1010961
:104EC800022E5FFA8AFA5FFA89F97FF4DFAEDFF81B
:104ED80054A24827023E1AF8013FB04601362BB9C2
:104EE800894BF31813F8011C002937D0236838467A
:104EF80043F080432360FEF76FFC002847D14FF052
:104F0800370909FB08F9DFF820B21BF8093013F05C
:104F1800200F3CD13846FEF717FB8046002836D1D3
:104F28001BF80930012143F020030BF80930042352
:104F380000930333019333B20322029313200B46E9
:104F48000CF0B4FF50200DF083FB192041460122DC
:104F58004346CDF80080FDF7D3FB18E0372303FB69
:104F680008F3DFF8C49119F8033013F0200F05D0C7
:104F7800992001220B460091FDF7C2FB372303FB62
:104F880008F819F808306FF3451309F808300137A5
:104F9800042EFFB29FD1A67806F00806F6B2002EBE
:104FA80040F03681594A06925FFA86F8B8F1000F48
:104FB8000CBF4023702347F69B510993089149F68B
:104FC8009E69002447464FF4E07A0AFB06FA4F4AE6
:104FD8002146524410465FFA84F8079220F047FAB7
:104FE80048B94A480AF1700A5044214620F03FFA6D
:104FF800002800F0FA80454B4FF4E07A0AFB063AA5
:105008000AF1E00A5046214620F031FA002840F023
:10501800EC805046214620F014FADFF810A10FB9B1
:10502800484600E008980CF0C3FE8AF800009AF899
:105038000000DFF8F8B0002800F0D7800138C0B2CF
:105048008BF800000BF08AFA002840F0CE809BF81D
:10505800000000F56A507C300CF0AAFE2C49C0B262
:1050680008701FB92B4B19F803A003E0069A13190F
:1050780093F850A100EA0A0ABAF1000F00F0B580CF
:105088000798214620F0F3F9DFF894B000B31F4BDE
:105098004FF4E07000FB06302146703020F0E7F94D
:1050A800B0B91D49012F0B784AEA030A8BF800A012
:1050B80058D13823B8FBF3F203FB12834FF436615F
:1050C8004A43DBB2342101FB0323144AD31843E0DB
:1050D8000E4B4FF4E07000FB06302146703020F094
:1050E800C6F938B10798214620F0C1F910B90A4924
:1050F8000B7804E0084A13781AEA030F18D023EA59
:105108000A0A8BF800A02DE0193B0020282900206E
:10511800221E0020D28EFF1F141A0020283F0020D4
:10512800881D0020213B0020E03C0020F61A0020CA
:105138004AEA030A012F8BF800A013D13823B8FBE1
:10514800F3F203FB12834FF436614A43DBB2342196
:1051580001FB03239249CB1893F8302042F0200238
:1051680083F830208F489049904AFEF719FD8E4BFE
:105178001B781BB1FDF79AFF002836D18A488C4965
:1051880013F0BCF868B10DF077F970BB884808F0E7
:1051980095FC50BB012386488649834A0093FEF755
:1051A800D5FC00230093844A0133019313787D488A
:1051B80002937D497D4A7F4B08F00CFC012F14D1E6
:1051C8003823B8FBF3F203FB12884FF436635A43D3
:1051D8005FFA88F8342303FB08237149CB1893F846
:1051E800312042F0010283F831200134089A0999EC
:1051F800E3B205328B4209F101090892FFF4E3AEEC
:10520800069A013602F5E072022E06927FF4CCAEC1
:105218006A4E73786FF3C71373702B7803F08002AC
:10522800D2B2002A00F0EE8065490C78002C40F0DC
:10523800E98003F02403042B0BD1FEF7E1FBFF23E5
:1052480000934020214601222346019402940CF049
:105258002DFE2B8800246FF3C7136FF3820364F3CA
:10526800451364F3410364F30003564A64F3492386
:1052780064F38A2314702B80534B1A7842F0C002CF
:105288001A705A7864F3C3025A70FEF799FC4F48B3
:1052980020F092F84E4820F08FF84E4820F08CF815
:1052A80041224D482146FBF775F84C4B1A7802F01D
:1052B800DF0264F304121A7093F8292002F0DF0267
:1052C80064F3041283F8292093F8522002F0DF02D5
:1052D80064F3041283F8522093F87B2002F0DF0273
:1052E80064F3041283F87B203D4B1A7802F0DF0246
:1052F80064F386121A7093F8222002F0DF0264F336
:10530800861283F82220374B1A7864F345121A70F4
:1053180093F8372064F3451283F8372093F86E200A
:1053280064F3451283F86E2093F8A52064F34512C0
:1053380083F8A5202C4B1A7802F0DF0264F386125A
:105348001A702A4B5A7864F345125A701A7802F088
:10535800BF0264F345121A7093F8252064F34512CE
:1053680083F8252093F8242002F0BF0264F3451245
:1053780083F8242011E04FF436626243342101FBA4
:1053880003221B49013352189178382B6FF382019D
:105398009170F0D10134022C2CD00023EBE700BF30
:1053A800283F0020881D0020711E0020641E002058
:1053B800211A00204D1D0020221E0020561A002010
:1053C80064130020F31B0020B43C0020721C002052
:1053D800191A0020461A0020641A0020A53B002054
:1053E800263B0020E03C0020F13A0020903A0020C3
:1053F800303F0020042273480021FAF7CBFF724B9C
:1054080000221A70714C2378002B4DD12978704AEC
:1054180001F00201C9B201B36E49487863F3820012
:1054280048706D481188477863F34D3163F3C307BB
:1054380041F0800147701180CA2020F03DFEC6204F
:1054480020F03AFE20F086FE644A13780BB90DF07E
:105458008BF9FEF75BF8FEF785FD614A2B8811781A
:105468006FF341036FF300016FF3000311705D48A0
:10547800002140222B80FAF78DFF5B481FF09CFF2C
:105488005A481FF099FF5A481FF096FF59481FF0D5
:1054980097FF04224B480021FAF77CFF4A4A002371
:1054A8001370554A13706AE02F7807F00203DBB2D5
:1054B80093B917F001070FD14B481FF07DFF2378F0
:1054C800F8B23B4113F0010F03D0FEF7B5F90CF029
:1054D800C9FF0137042FF2D12B783D4F13F0010F8C
:1054E80025D0FEF7D3FC3B8843F002033B80FEF750
:1054F80045FA354B93F80080B8F1000F14D1CA2053
:1055080020F0DAFDCD2020F0D7FD3B883B4868F33A
:1055180000033B80324B1A7842F001021A701FF0E8
:105528004BFFFDF7F3FF02E00120FEF789FB2B7824
:1055380003F00202D2B212B32F4A12782AB113F042
:10554800010F02D10220FEF77BFBFEF7DDFE2C499E
:1055580026481FF04FFF254925481FF035FFFEF765
:1055680049FB224927481FF02FFF274925481FF0EC
:1055780036FFFEF7D9FA1F481C491FF046FF20499D
:1055880022481FF021FF15490B780BB9FEF75AFA8C
:10559800737803F08003DBB2002B3FD1FEF7FEFCEB
:1055A80030B143F6EC200CF003FC08B1062033E0E0
:1055B800FEF7C6FC08B105202EE00DF0BFF938B3A0
:1055C800032029E03A1A0020121A0020141A002099
:1055D800101C0020CB3C0020B43C002064130020A9
:1055E800181A0020321C0020F5310020EA1B002088
:1055F800461A00202A1C00207A1C0020F71A0020D6
:10560800591A00201A1C0020A61A00203E1A002051
:1056180001F06EF810B10420FEF712FB6C4B1B78FA
:105628001BB173786FF3C71373706A4A137813B199
:10563800694B1B78CBB12B78684E03F04403402BA1
:1056480013D10021BF3300933F200B460222019162
:1056580002910CF02BFC338843F6CE2043F0040370
:1056680033800CF0A5FB5E4B18705A495D4E0B78E1
:105678009BB1594B197881B92A78584B02F04002EE
:10568800D2B252B11A8861F382021A80337823B9F0
:1056980043F6CE200CF08CFB30702A78DFF83C8182
:1056A80002F00400C0B2504B00287FD002F0200066
:1056B800C0B24B4F90B11A78002042F0C0021A7065
:1056C800FDF708FE3B78002B76D1B8F8002063F38D
:1056D800820263F34512A8F800206DE0D20052B2AE
:1056E80019789211D2B241F0C00112F0010F19706D
:1056F80003D0C9B260F3C711197012F0020F03D0BA
:105708001A786FF386121A701B78374A03F0400331
:10571800DBB273B9537843F008035370237843B16D
:105728002B8843F400532B80304B5A7842F0040204
:105738005A700120FDF7CEFD43F6CD200CF038FB62
:10574800C0B20128307002D1264B02221A703C7870
:10575800002C31D1FEF754F9FF2301220093402099
:1057680021462346019402940CF0A0FB2B8843F6B3
:10577800CD2043F020032B800CF01AFB184B1C4A59
:105788001870154B14701A780AB1013A1A70197802
:1057980091B9104A13787BB1FF230093412002226C
:1057A8000B46019102910CF081FB05E01A7842F05A
:1057B800C0021A70FDF78EFD0DF070F80D481FF04D
:1057C80029FE0D4BD0B91A7860F3820219E000BFA8
:1057D8006E590020FC1B00207B1C0020101C0020A0
:1057E800F31B0020631A0020B43C0020CB3C0020AF
:1057F80064130020AE1A0020181A00201A7842F00C
:1058080004021A706A78574812F001011A780CBF1E
:1058180061F3410242F002021A7053491FF0F5FD8C
:10582800524950481FF0DBFD4E4851491FF0D7FD43
:105838003378012B40F093802B8800246FF34923A1
:105848006FF38A232B804B4B41221C7021464A4818
:10585800FAF7A0FD49481FF0AFFDFEF7B1F943483C
:105868001FF0AAFD42481FF0A7FD454B1A7802F029
:10587800DF0264F304121A7093F8292002F0DF02A1
:1058880064F3041283F8292093F8522002F0DF020F
:1058980064F3041283F8522093F87B2002F0DF02AD
:1058A80064F3041283F87B20364B1A7802F0DF0287
:1058B80064F386121A7093F8222002F0DF0264F370
:1058C800861283F82220304B1A7864F345121A7036
:1058D80093F8372064F3451283F8372093F86E2045
:1058E80064F3451283F86E2093F8A52064F34512FB
:1058F80083F8A520254B1A7802F0DF0264F386129C
:105908001A70234B5A7864F345125A701A7802F0C9
:10591800BF0264F345121A7093F8252064F3451208
:1059280083F8252093F8242002F0BF0264F345127F
:1059380083F8242011E04FF436626243342101FBDE
:1059480003221449013352189178382B6FF38201DE
:105958009170F0D10134022C01D00023EBE70BB099
:10596800BDE8F08F7A3600201A1C0020191A002092
:10597800721C0020631A0020641A0020461A0020B6
:10598800A53B0020263B0020E03C0020F13A002007
:10599800903A0020303F00202DE9FF4104460D4693
:1059A8000CF0A6FFA04B1A1992F880709F4A9846EF
:1059B8001278AA2A0AD1A7F14F03DAB20B2A00F209
:1059C800AD819B4A5BB29A4040F1A881994B0C2269
:1059D80002FB04335A7A0833AA42C0F09F81FF2A97
:1059E80000F09C81FF229A70934808EBD40321466B
:1059F80093F888511FF03BFD0646002840F08E8141
:105A080004F007031D41502F05F0010500F0268121
:105A180014D8462F00F0F28009D8412F00F09E805C
:105A2800452F00F01B812D2F40F0768134E0482F60
:105A380000F0C5804F2F40F06F810EE0542F67D0E3
:105A480006D8522F00F08A80532F40F065811CE061
:105A5800A7F15903012B00F25F81784821461FF016
:105A680006FD0646002840F059815A2F01D1744896
:105A780002E0592F04D1734821461FF0E2FC54E19B
:105A880021466F481FF0DDFCF5E76F4821461FF0FF
:105A9800EEFC002800F042816C4821461FF0E7FC2C
:105AA8008046002840F03A81214668481FF0C9FC2A
:105AB800674821461FF0D0FC0227012655B1A419DA
:105AC800142041463A4643460097019602940CF04A
:105AD800EDF92AE129463A46334604F101080A203D
:105AE80000970196CDF808800CF0E0F92046FCF705
:105AF8003FFB414602462B4613200095FCF700FE6B
:105B0800384629462A4633460095FCF7F9FD0CE14C
:105B18004E4821461FF0ABFC0746002840F005819F
:105B28000126022231463346A5193E2000920196ED
:105B380002950CF0BBF92046FCF71AFB29460246F1
:105B48003B4614200097FCF7DBFD21463F481FF039
:105B580078FC21463E481FF07FFCE6E03A482146A3
:105B68001FF085FC0646002800F0DF8037482146F4
:105B78001FF07DFC064628B92046FDF7E5FC002805
:105B880040F0D380002D40F08E802046FEF7B2F919
:105B9800002840F0C5802046FEF7A6FB2D4BDB7899
:105BA80003F02003DBB20BB92B4B1855412F00F043
:105BB8008880522F40F0B0802046012183E023489E
:105BC80021461FF054FC28B92046FDF7BDFC0028EB
:105BD80040F0A480002D66D12046FEF78BF90028FE
:105BE80040F09E801B4BDB7803F02003DBB2002BD8
:105BF80067D1194B032283F8402062E013482146FD
:105C08001FF035FC064628B92046FDF79DFC002804
:105C180040F08B802046FEF76DF900287ED1002DDC
:105C280041D1204603214EE0B02C0020F21B002079
:105C380000003080842E0020591A0020082A0020F5
:105C48002829002098290020EA1B00201A1C00207F
:105C5800221C0020883A0020641A0020354821467A
:105C68001FF005FC064600285FD02046FDF73EFEE3
:105C780020B1214630481FF0E4FB4FE0502F28D1D7
:105C88002E4B1B782BBB2046FDF71CFE08BB2C486F
:105C980021461FF0ECFB064620B92046FDF754FCD0
:105CA800002842D115B1204602210CE02046FEF71B
:105CB8001BFB244BDB7803F02003DBB20BB9224B30
:105CC800185520460021FEF717FA061E18BF0126B0
:105CD8002BE02046FDF7F6FD0546F8B91B4821469E
:105CE8001FF0C5FB0646D8B92046FDF72DFC074630
:105CF800D8B9164821461FF0A4FB154A135D8BB985
:105D080010494E7806F02006F6B26EB908EB040387
:105D180093F80031135508E0012606E0002604E058
:105D28002E4602E03E4600E01E46304604B0BDE87E
:105D3800F08100BFEA1B0020F71A00207A1C00201F
:105D48001A1C0020883A0020641A0020461A0020F5
:105D5800321C0020032210B505490648FAF7F0FD69
:105D6800054806490222BDE81040FAF7E9BD00BF20
:105D7800832600200402002009020020812600203A
:105D880070B5834B1B7813F0010F0AD00CF07CFB25
:105D980038B100207F4902F08DFE7F4B7F4819788B
:105DA80047E07F4D2B78002B48D00CF073FB002880
:105DB80044D07C4B1B7863B97B4B5B7813F0010FA5
:105DC80007D00CF059FB20B9FEF7E8F808B103201A
:105DD800BEE0764C207870B10020754902F06AFE6A
:105DE80021780122734802F08BFE00201021621CEA
:105DF80007F0D8FA02E0704902F05CFE6F4C684880
:105E080007F0F6FA2378002B00F018810CF03CFB21
:105E1800002800F013816A496A481022FAF790FDB9
:105E280068485B21FAF734FB002800F007812178E5
:105E380001308322BDE8704002F062BE624C2378D4
:105E480003F00503012B5DD10020604902F032FE0A
:105E5800202110225E48FAF79DFA601D5D49032251
:105E6800FAF718FD40BBE01C5B490222FAF712FD65
:105E780030B95A48FAF7DEFC5849024654480BE054
:105E8800E01C57490222FAF705FD40B95548FAF7D0
:105E9800D1FC544902464E48FAF752FD0EE0E01C88
:105EA80051490222FAF7F6FC30B95048FAF7C2FC19
:105EB8004E4902464648EFE7FFF74CFF6278303A12
:105EC800D3B2092B00F2BA803F4B9B78303BDBB250
:105ED800092B00F2B3800A2101FB0231C9B2002963
:105EE80000F0AC80374BFF220C291A7740F2A680CD
:105EF80010295A7740F2A28013299A7740F29E809F
:105F0800DA7770BD3A4C237803F00203DBB213B1A1
:105F1800002038498EE0234E3378EBB9224B5B786A
:105F280013F0010F18D00CF0A7FAA8B932481FF0E7
:105F380071FA60B12268314B02EA03033BB919F0E8
:105F48001DFB20B9E37803F04003DBB223B1002046
:105F5800BDE8704009F0D6BD337863B90CF08CFA0F
:105F680048B1274B1B7803F00603042B03D02B788A
:105F78000BB90120ECE7FDF7E3FF10B10020214940
:105F880058E0214B1D78002D42D0204952E000BF37
:105F9800101C0020593E0308121A0020000200209D
:105FA800141A0020201E0020E11E00206A1D002077
:105FB8006C130308050200202A1303087A1C00202A
:105FC8004B130308F40100207E26002073180308F1
:105FD8000402002094A1030898A10308D618030816
:105FE8009BA10308B51803089EA103089418030889
:105FF800883A0020CA270308AE1A00203000000F94
:10600800181A0020FC250308691300208D130308C3
:106018000B4802F0FEFC0A4802F0F2FC094802F0C4
:10602800EFFC1DF099FEE37803F02003DBB22BB1FF
:1060380005492846BDE8704002F03CBD70BD00BF70
:10604800741E0020941D002085120308054B1B7840
:10605800D8019B015BB2DB1140B243EAE070C0B2E9
:10606800704700BF101C002070B50E4686B0410076
:106078000122054601F5E97105A80BF0AAFE0021E9
:10608800012E8DF815104FF0FF0205F1010305D11F
:106098000092019102930920FB3A04E000920191D9
:1060A80002931E2004220B460BF000FF05A83D4971
:1060B800FAF774FA50B105A83B49FAF76FFA28B114
:1060C80005A83A49FAF76AFA002867D105A83749B6
:1060D800FAF764FA364B0446F8B95A78214642F082
:1060E80010025A70FF23022200930190FE3B029097
:1060F8003D200BF0DBFE4D200CF0AAFA691C0122B2
:10610800234612200094FCF7FBFA1220214622466F
:1061180001230094FCF7F4FA03E05A786FF30412B1
:106128005A700024E0B2552116F09EFA38B128467C
:10613800214616F03AFC10B1204616F025FC013431
:10614800082CEFD13EBB1B481B491C4AFDF728FD14
:1061580019481B4912F0D2F868B10CF08DF950B902
:10616800174807F0ABFC30B9012315481549124A06
:106178000093FDF7EBFC144B0F491D7000230093AF
:1061880005330193114B0D4A1B780A4802930D4BB6
:1061980007F020FC02E00E4B00221A7005A806B09A
:1061A80070BD00BF25A20308A1A1030831A40308FC
:1061B800B43C0020881D0020711E0020641E0020B1
:1061C800211A00204D1D0020CF3C0020221E002057
:1061D800391A002007B54100012201A801F5E9712B
:1061E8000BF0F7FD002301A804498DF80530FAF7F4
:1061F800D5F9D0F1010038BF00200EBD25A2030853
:1062080007B54100012201A801F5E9710BF0E1FD94
:10621800002301A804498DF80530FAF7BFF9D0F139
:10622800010038BF00200EBDEEA3030870B5154B62
:1062380004461B1893F88050B1B1134821461FF04B
:1062480016F988B9114821461FF0FBF8A5F1590342
:10625800DBB2012B0CD94F2D0AD0542D08D0214682
:106268000B481FF0EEF807E0084821461FF0F4F845
:10627800074821461FF0F0F804480649BDE8704079
:106288001FF0A2B8B02C0020591A0020AE1A002026
:106298004E1A00202A1C0020024B1878C0F38000F8
:1062A800704700BF181A0020024B1A8860F30822B2
:1062B8001A807047101C0020034B5878C00140B268
:1062C800C011C0B2704700BF101C0020014B1878E5
:1062D800704700BF141A002030B54578002300210C
:1062E800C218917055FA03F111F0010F08D0064950
:1062F80059188C7C017804EA0101A14208BF917009
:106308000133042BEBD130BD6A1D002046F629511C
:1063180004220BF05EBD000070B5104C054611223A
:1063280020460021FAF736F8002004F8010C2A78F4
:10633800103414F8011FC3B291420BD152B108496D
:10634800013301F8013B112246F67973BDE870402C
:1063580002F0FCBA01300428EBD170BD6B1D00209F
:106368006A1D00201FB520B1134B1A8842F48052D1
:106378001A80124B00245A78214642F010025A70B3
:10638800FF23022200933D20FE3B019402940BF070
:106398008DFD4D200CF05CF92021012223461220AE
:1063A8000094FCF7ADF912202146224601230094FF
:1063B800FCF7A6F91FBD00BF101C0020B43C00204C
:1063C8002DE9F3412D4C0722E37849F6346702FBA7
:1063D8000030C0B200F51E4055300BF0E9FC2579BD
:1063E80064795FFA80F8002648FA06F313F0010F83
:1063F8003AD03946042201A80BF0EBFC9DF80400C2
:106408009DF805309DF806109DF8072000282BD030
:10641800002929D0002B27D0002A25D0934204D167
:106428009C4221D185421FD30FE09A4210D99C4249
:106438001AD3944218D89C4201D994421AD39C4248
:1064480001D1854216D294420ED18D420CD811E06A
:106458009C4201D185420DD2944201D18D4209D985
:106468009C4207D8944205D301360437082EBBD185
:10647800002000E00120BDE8FC8100BFDC560020C0
:1064880010B5044649F68D6000EBD4000BF090FC83
:1064980004F00704C0B2204100F0010010BD70B53F
:1064A800C30849F68D655D19044628460E460BF06B
:1064B8007FFC04F00704C0B2012126B9A14040EADC
:1064C8000101C9B202E0A14020EA01012846BDE865
:1064D80070400BF063BC0000F0B57D4B8DB0DD78EB
:1064E800042200EBC505EDB2E90001F50A4104A854
:1064F800BC310BF06EFC774B774E1A78002304A959
:10650800C95C312905D13039994041EA0202D2B239
:1065180005E0302903D12F39994022EA01020133DD
:10652800042BECD132706C486C496D4AFDF738FB8E
:106538006A4B1B7813B96A4B1B78F3B167486949F2
:1065480011F0DCFE68B10BF097FF50B9654807F011
:10655800B5FA30B9012363486349604A0093FDF7EF
:10656800F5FA0023009302330193FD3302935A484E
:106578005A495B4A5C4B07F02DFA05EB05110024DC
:1065880001F50C41347004A87C3108220BF021FC81
:106598002646E0B2542116F067F8002838D004AB3C
:1065A8001B5D312B03D1204616F0F4F838B104AB4B
:1065B8001B5D302B2CD1204616F0ECF840B34EB9B9
:1065C800FF23009334203146042233460196029675
:1065D8000BF06CFC04AE305D2146303816F0E8F85C
:1065E800335D0126312B4FF0030306D10093A31925
:1065F8001BB201960293352005E00093631C1BB281
:10660800019602933620002104220B460BF04EFC23
:106618000134082CBDD1A90101F5104104A8343179
:1066280020220BF0D6FB083C04AD274615F8013BA9
:10663800E6B20134302B03D13046FFF721FF38B1E1
:1066480015F8013C312B2CD13046FFF719FF40B328
:106658004FB9FF2300933420394604223B46019763
:1066680002970BF023FC15F8011C30463039C9B2EB
:10667800FFF715FF15F8013C0021302B4FF0FF0301
:1066880005D1009323B201910293372004E00093CF
:1066980023B201910293382004220B460BF006FC2A
:1066A8000127202CC2D1114D6B7803F00403DBB213
:1066B80063B1203C2046FFF7E3FE38B90134E4B269
:1066C800202CF7D16B7860F382036B700DB0F0BDAE
:1066D800DC560020141A0020881D0020711E00209E
:1066E800641E0020211A00204D1D0020B43C00200B
:1066F800014B1878704700BF691300202DE9F04F4F
:106708004E4B00221A704E4A85B01678002E40F083
:1067180091804C4B4FF4B468DA78997808FB02F210
:106728004FF03C0808FB01285A78474F90441FFA5D
:1067380088F8BA466CE03AF815303C24DAB254438B
:1067480004EB13244C44A4B2042CEEB207D842F252
:106758005A73984503D904F51C546034A4B24445CF
:1067680011D949F654600BF023FBC8EB04038342AC
:1067780009DC364B1A787B1993F83830934302D0EA
:106788002E4901230B702F4AD378B34232D142F2FB
:106798006073B4FBF3F203FB12439BB2434523D16E
:1067A8002B4B9B7813F0090F44D12A4B5B7803F0ED
:1067B8008003DBB2002B3DD1274B5B7803F002034B
:1067C800DBB2002B36D1254B1A781BEA020F11D108
:1067D8000199009841EA02021A70FFF7F1FD48B9E1
:1067E8000098FFF779FE05E01C4B02991A7801EA38
:1067F80002021A70013509F5B469072D1FFA89F9E3
:1068080099D1039E07370136042E0AF10E0A11D0DA
:106818004FF0010B0BFA06FB5FFA8BF301936FEA5B
:106828000B03F2B2DBB24FF00009009202934D461F
:10683800039680E705B0BDE8F08F00BF691300201C
:10684800811C0020DC560020821C0020141A002025
:10685800883A0020C33C002072340020801C0020AD
:1068680073B50C4601EBC001C9B2C90001F50A4174
:106878000546042201A8BC310BF0ABFA104B0020EE
:1068880003EBC402121B521982F8380001AA125CE9
:10689800312A0AD10121814003EBC402121B52198B
:1068A80092F83860314382F8381001300428EDD16D
:1068B80001A9312230231EF0E2FDC0B27CBD00BF29
:1068C800821C002000B501EBC001C9B2890189B062
:1068D80001F510413431202268460BF07AFA202065
:1068E8006946312230231EF0CAFDC0B209B000BD8E
:1068F80007B501EBC001C9B201EB011101F50C416B
:106908007C31082268460BF064FA08206946312277
:1069180030231EF0B4FDC0B20EBD00002DE9F843CF
:10692800002634462BE021462846FFF799FF2146EA
:1069380081462846FFF7C6FF214640EA090928464E
:10694800FFF7D6FF5FFA89F949EA000010F0FF0F58
:1069580005D04046394602220BF03BFA03E04FF0DF
:10696800FF33A8F800300135EDB20237072D08F1E2
:106978000208D8D10134E4B20E3E042C07D0054BEE
:10698800C6F50A47C6EB03084C370025CBE7BDE838
:10699800F88300BF821C002010B523F08DFA4FF455
:1069A800803023F0A9FA23F0C1FB0128044628D13E
:1069B800102023F0A3F9022023F094F9002023F0FB
:1069C800DBFA002023F0ECFA4FF4806023F0DEFAC3
:1069D8004FF4404023F0EEFA4FF480304FF4E011CA
:1069E80023F0A6FA204623F0AFFA392023F08AFBD9
:1069F8000028FAD0022023F0ADFA23F0B5FA0828CF
:106A0800FBD17C20012123F047FB46F60120012120
:106A180023F042FB0C48012123F04AFB0B480121DB
:106A280023F046FB0420012123F042FB7E2023F0C3
:106A380069FB38B123F090FB054B04211A7861F308
:106A480044021A7010BD00BF034006002008081851
:106A58005159002010B50C46014620B110220C48AF
:106A6800F9F76EFF04E00A4820211022F9F792FC9A
:106A780034B1084821461022BDE81040F9F760BF3C
:106A8800044820211022BDE81040F9F783BC00BF5C
:106A9800F40100200402002010B5FF2B1446029ACE
:106AA80003D0421802F8013C08E06FF07F439A4295
:106AB80004D01314437013128370C2701CF060F872
:106AC80002E07F2023F064FE1CF046F80028F8D18D
:106AD800ACB10B4890F82010163001F00F011CF0F3
:106AE8004FF802E07F2023F053FE1CF035F8002811
:106AF800F8D1044B93F8693013F0010FE9D110BDB8
:106B0800900C00206C58002010B50A4B002203EBB3
:106B1800C003013B1046084951184C7813F8011F6F
:106B28008C4205D10130C0B20C320828F3D1F730BD
:106B380010BD00BF62A80208842E002070B50D4C5D
:106B480005460E464FF4007200212046F9F722FC54
:106B58002A46314604F50070F9F774FB642024F8DE
:106B6800035C1DF0CBFB0023A4F82D33024B6422F9
:106B78001A6070BDD55900208826002010B5054C34
:106B8800002120464FF40072F9F704FC0023A4F812
:106B98002D3310BDD5590020164B2DE9F0415D8AE3
:106BA80007462846FAF7BCFF1349FBF7C5F8134B0D
:106BB800134E1860D723B5FBF3F5EDB282222946B0
:106BC8000446F01901F09CFF2846FAF7ADFF01468C
:106BD8002046FAF7F3FE0B49FAF7FAFFFBF7BEF97E
:106BE8000337BE19C1B281223046BDE8F04101F039
:106BF80087BF00BFC031002000005743D81C0020C9
:106C0800F40100200000204170B54B4D2868FAF7C8
:106C180093FB45A3D3E90023FAF72EFAFAF77AFE95
:106C2800FAF78AFB42A3D3E90023FAF7D9FB3EA37C
:106C3800D3E90023FAF7FEFCFAF76CFEFAF77CFBBF
:106C4800FAF786F9FAF766FE3C4906462860FBF72C
:106C580067F920B13046FBF781F9C4B25EE03046EF
:106C68003649FBF771F950B130463549FBF758F909
:106C780028B13046FBF772F9C0B2441C4EE03046EA
:106C88002F49FBF761F950B130462E49FBF748F917
:106C980028B13046FBF762F9C0B2841C3EE03046AA
:106CA8002849FBF751F950B130462749FBF738F925
:106CB80028B13046FBF752F9C0B2C41C2EE030466A
:106CC8002149FBF741F950B130462049FBF728F933
:106CD80028B13046FBF742F9C0B2041D1EE0304629
:106CE8001A49FBF731F950B130461949FBF718F941
:106CF80028B13046FBF732F9C0B2441D0EE03046E9
:106D08001349FBF721F948B130461249FBF708F956
:106D180020B13046FBF722F9C0B2841D0A20214673
:106D2800BDE870400BF03AB8736891ED7CFF7F4086
:106D38000000000080842E41DC1C0020000010416F
:106D48000000F0410000484200008E420000B842B6
:106D58000000E0420000F2422DE9F04FA1B01BF024
:106D6800A5FE09201DF066FC1DF04CFA4FF46140A9
:106D78001DF09CFC09201DF019FD0022A3484FF4CA
:106D8800804123F020F8A248002123F0E9FBA14923
:106D980004224B78DFF8A0E26FF300034B709E4BA0
:106DA8009E4C1A705A715A709A70DA701A719A71E8
:106DB800DA719B4B033A1A709A4B00201F328EF8F7
:106DC800000020705A7105900546069006467F20FF
:106DD80023F0DEFC23780E2B01F2B681DFE813F0F6
:106DE8000F004F009500E0007902DE0330048504AF
:106DF800EA06DC07EF075808B108D00882098A4E6E
:106E08008A48317801F00F01013149014118FFF733
:106E180021FE337813F00F0308D1854A92F8012335
:106E2800012A41F09181834A138024E0012B03D188
:106E38007F4B93F819330BE0022B04D17C4B93F86A
:106E48000D33032B05E0032B06D1794B93F80D3353
:106E5800012B41F079810EE0774901220A707748C9
:106E68004FF4007122F0AFFF754BC8221A603378D7
:106E78006FF30303BFE333785A1C01F05FB8704B1C
:106E88001A6822B96D484FF4007122F09CFFDFF8B0
:106E980098816C4898F8001001F00F010131490100
:106EA8004118FFF7D7FD36B198F800305A1C62F345
:106EB800030388F800305F4B00221A8098F800100E
:106EC80001F00F02022A03D11A7842F010020AE0F8
:106ED800042A03D11A7842F0040204E0052A05D1F5
:106EE8001A7842F040021A7001F02EB9062A04D12D
:106EF8004D4B6FF3030119707EE301F00F0101227E
:106F080012FA01F1198001F01FB9474E4E48317845
:106F180001F00F01013149014118FFF79BFD96F877
:106F2800008008F00F08B8F1070F27DC18F0010FF0
:106F3800464B02D00020588002E04FF0FF315980C4
:106F48004FEA6809062209F1010902FB09394FF0E5
:106F5800FF32A9F802204046FFF7D6FDFF2806D0E9
:106F68003B4B03EB40005823437401F0EDB800237A
:106F7800A9F8023008F1010801F08AB800211022AE
:106F88001BA8F9F707FA17A800211022F9F702FA47
:106F980023780133237033786FF3030301F07BB850
:106FA800DFF884A09AF8008018F00F0840F03F81BD
:106FB800284E337803F04003DBB2F3B926486FF06C
:106FC8007F43817A0122009301F00F01FF23FFF72D
:106FD80063FD224B93F8692012F0400F08D093F814
:106FE8006C3013F0040F03D0337843F04003337050
:106FF8007378142262F3C7037370737813F0F80F71
:1070080030D0174800F12001A7E300BF0018014065
:10701800002C0140E2310020B02C0020E21C0020AE
:1070280067130020A53B0020E11C0020A2A802084D
:10703800842E0020B43C0020B8260020000C01401B
:107048008826002042A9020822AA02086E3C0020D5
:10705800F4010020733A0020900C00206C580020A6
:1070680042AB0208BC4B1B7803F04003DBB2002B99
:1070780000F0D980DFF80483DFF8049398F8003033
:1070880013F00C0B30D1B54E6FF07F4396F82B10F0
:1070980006F12100009301F00F0101220523FFF7FB
:1070A800FBFC96F84C104FF4860A06F1420001F0FA
:1070B8000F010122FF23CDF800A0FFF7EDFC96F8A1
:1070C8004110FF2306F1370001F00F015A46CDF8B1
:1070D80000A0FFF7E1FC042389F8003098F800309D
:1070E80043F0080301F02EB803F00803DBB2002BCD
:1070F80039D099F800A0BAF1000F03D0984800F1F0
:10710800400138E0954E6FF07F4B717D06F10B0022
:1071180001F00F010122FF23CDF800B0FFF7BCFCFE
:1071280096F82B1006F1210001F00F010122072328
:10713800CDF800B0FFF7B0FC96F836104FF4860390
:10714800009306F12C00FF2301F00F015246FFF7D0
:10715800A3FC98F800306AF3C303DBB243F00403DE
:1071680088F800305AE099F800C0BCF1000F08D048
:107178007B4800F16001FFF76DFC99F80020303280
:1071880008E2764E6FF07F40717DFF23009001F09A
:107198000F0106F10B000122CDF80CC0FFF77CFCB3
:1071A8009AF80030DFF8C4B103F0100A5FFA8AFADF
:1071B800DDF80CC0BAF1000F0CD098F800206CF381
:1071C800820288F800205A1C62F303038BF800300F
:1071D80000F0BABF96F82B106FF07F42009206F1CC
:1071E800210001F00F0101220C23FFF755FC96F84E
:1071F80036104FF4860300935246FF2306F12C0005
:1072080001F00F01FFF748FC9BF8003083F01002F3
:10721800C2F3001262F304138BF80030042389F8D8
:10722800003000F091BF4E4800F1800195E2B8F1BE
:10723800010F3CD14A4800F1A001FFF70BFC002EDA
:1072480000F082879AF80030444E5A1C62F3030318
:107258008AF8003096F82B106FF07F4906F121006C
:1072680042460F2301F00F01CDF80090FFF714FC00
:1072780096F82B1006F1210042460E2301F00F016B
:10728800CDF80090FFF708FC96F82B1006F12100C6
:10729800424601F00F010F23CDF80090FFF7FCFBE9
:1072A80030488021424622F08EFD00F04DBF2C4828
:1072B80000F1C001FFF7CEFB002E00F045872A4BF6
:1072C80096221A609AF800306FF303038AF80030A8
:1072D80092E1264E317811F00F0A16D1244800F1B8
:1072E8002001FFF7B7FB204B1B68002B40F02C87D1
:1072F8001BA8F9F79FFA4022134601461BA801F084
:1073080023FA3378012200F019BEBAF1010F39D1FE
:1073180012486FF07F4390F8201000220093163037
:1073280001F00F01FF23FFF7B7FB01F077FA002800
:1073380000F00A873378022262F3030333700D4B9F
:107348001A7842F080021A700B4B5A7842F0020207
:107358005A7000F0F9BE00BF733A0020900C00206C
:1073680042AB02080010014088260020E11C0020E2
:1073780022AC0208783A00204A3E0020F05F002044
:107388007761002001F00F0101F10E0303F00F03F4
:10739800012B44D89B4849014118FFF75BFB9A48E9
:1073A8006FF07F4390F8201000221630009301F010
:1073B8000F01FF23FFF770FB1CF06CFD337803F01F
:1073C8000F03022B13D118F0A5F8002800F0BC8693
:1073D8008E4B1A7842F040026FF304121A705A78F2
:1073E8006FF345125A703378032200F0A7BD18F0E6
:1073F8007BF878B118F01AF917F0D2FF844B002007
:107408001A7858816FF3C7121A703378042262F31E
:10741800030333707F4B1A786FF3000263E5BAF108
:10742800040F4DD1DFF8DC914901DFF8108249449F
:107438004846FFF70FFB98F80010774B01F004025D
:10744800D2B27AB941F004016F4883F800A088F8F5
:10745800001090F836104FF4860300932C3001F09A
:107468000F01EEE293F800A0BAF1000F40F06C862D
:1074780065486FF07F45417D01220B3001F00F0117
:10748800FF230095FFF708FB64480122817AFF2358
:1074980001F00F010095FFF7FFFA98F80030052278
:1074A8006AF3820388F800303378484662F30303AE
:1074B800337009F1A001FFF7CDFA554600F044BE3C
:1074C800DFF84481FF2398F8201000226FF07F49ED
:1074D80008F1160001F00F01CDF80090FFF7DCFA73
:1074E8002BB2072B18D1337808F121006FF303036F
:1074F8003370237801220133237098F82B100E2360
:1075080001F00F01CDF80090FFF7C6FA444880213A
:10751800002222F058FC0025424E96F86B3013F0FA
:10752800040F00F0118698F857106FF07F4300227F
:1075380000933D48FF2301F00F01FFF7ADFA96F8DD
:107548006B303A4A03F00F03012B137003D1002D5F
:1075580008BF01250CE0022B04D12BB2012B08BF78
:10756800032505E0032B03D12BB2032B08BF072506
:10757800ABB213F0010F02D02D4A3121517713F02D
:10758800020F02D02A4A3221917713F0040F00F03B
:10759800DB853322264BDA7700F0D6BD1948254E15
:1075A80000F1C001FFF756FA96F80090DFF85C800A
:1075B80019F00F090CD117F00DFE98F8003069F397
:1075C800000388F8003033785A1C62F303033370E1
:1075D80017F092FE98F8003013F0010F00F0B48510
:1075E80000221548802122F0EEFB0A4B00225A7037
:1075F800337862F30303337023780133237000F088
:10760800A3BD00BF22AC0208900C00204A3E002017
:10761800783A0020C23D0020776100200100002058
:10762800001001406C580020DD0C0020723A002048
:10763800F4010020E11C002000180140F05F002048
:107648008648874E00F1E001FFF704FA17A8F9F71A
:10765800F1F817A902468348F9F772F90021824820
:10766800B18090F8C5106FF07F4300220093BB30C3
:10767800FF2301F00F01FFF70FFA7C4A92F86B1015
:1076880092F86C30327843EA012312F0010FB3808C
:1076980010D0A3F1EB0292B20A2A04D9A3F5E6733B
:1076A8009BB2282B02D8F3880133F38033786FF329
:1076B800000333707378002B40F04685684AD288FF
:1076C8007AB16B4A1FA8117863F30301117022780D
:1076D8008DF87F300132227028228DF87C2022F02C
:1076E80091FB0022F28000F02FBD624EDFF8ACA1C2
:1076F800337803F004085FFA88F8B8F1000F15D161
:1077080011A841461522F8F745FE5B4BCAF80080E0
:107718001B684546CDF847303368474643F00403B5
:107728003360564BA3F8368300F00EBD03F0800398
:10773800DBB2002B67D1DAF80010002940F004858D
:107748004F48FFF787F94F484FF4805122F031FB3B
:10775800012806D04A4800F1A001FFF77BF900F0A4
:10776800F3BC4649B1F83623002A43D009314648CC
:10777800013AF9F7E5F8444B03F1100113F8012B2E
:107788000D2A01D00A2A02D1202203F8012C8B42AB
:10779800F4D13E4B4FF03C0808FB073808F11E08AF
:1077A8004046F9F747F8414602463948F9F772F872
:1077B800D8B9022F03D1336843F0100304E0032F34
:1077C80003D1336843F040033360327853005BB22F
:1077D80003EAC263DB173268DBB263F3C7123260B5
:1077E8001BB1FFF7CBF900F0AFBC0137FFB2042F94
:1077F80008BF0227254B3C2606FB07363046F9F71B
:1078080019F8314626E0DAF80080B8F1000F40F0A8
:107818009B84737803F02002D2B2002A40D11D4B1A
:1078280011A81A889B781C498DF84630ADF8442079
:10783800F8F70AFE114B5B7A302B07D1FFF79EF958
:10784800336843F40053336000F07EBC11A8F8F7A6
:10785800F1FF11A9FFF772F900F076BC22AC02081B
:10786800C23D002008020020900C00206C58002027
:10787800E11C00208C260020A3A10308CC5900207D
:1078880022AD020800080140040200200C0000207C
:10789800D5590020A8A10308ACA103088826002018
:1078A80003F04003DBB2002B40F08980B14800F1BF
:1078B8006001FFF7CFF8B048F8F7BCFF8046AE4943
:1078C800AE484246F8F7E6FF002873D1AC4B434474
:1078D8005B7A302B6ED1FFF751F93368DFF8D0921D
:1078E80043F48043336099F82B106FF07F43009383
:1078F80009F12100082301F00F010122FFF7CCF85C
:107908006423CAF800307F2022F042FFDAF8003002
:10791800002BF8D1984699F88E10D633994E89F8ED
:1079280086304B3B6FF07F4A89F88730964801F0E4
:107938000F0142467433CDF800A0FFF7ADF896F872
:10794800B91106F5D670033001F00F014246FF2346
:10795800CDF800A0FFF7A0F896F8C41106F5DD7081
:1079680001F00F014246FF23CDF800A0FFF794F87D
:1079780096F8CF1106F5E270013001F00F0142468A
:10798800FF23CDF800A0FFF787F896F8DA1106F57F
:10799800E87001F00F014246FF23CDF800A0FFF781
:1079A8007BF899F899107948CDF800A001F00F01FB
:1079B800424646E07648F8F73DFF75494AE796F8AB
:1079C80002B0DFF8EC910BF0020B5FFA8BFBBBF116
:1079D800000F3AD199F82010FF236FF07F4809F182
:1079E800160001F00F015A46CDF80080FFF754F851
:1079F800684B93F86B3003F00803DBB2002B00F000
:107A0800A38399F82B10012209F1210001F00F013D
:107A18000323CDF80080FFF73FF83368554843F457
:107A2800003300F180013360FFF714F855485A46D7
:107A380090F8E51100F5EC70CDF80080033001F006
:107A48000F01FF23FFF728F87EE3CAF8008099F8B2
:107A580020106FF07F4300934246FF2309F1160080
:107A680001F00F01FFF718F82AB241F211139A42F8
:107A78001DD1434B5B7A302B13D1FFF77FF8336866
:107A8800454668F3514368F38E3368F34D333360EA
:107A9800414B1A7868F303021A7023780133237074
:107AA80052E33E48F8F7C6FE3C49FFF747F8394E1F
:107AB80096F86B3013F0040F00F0468325B9384868
:107AC80020211022F8F766FC7F2022F061FE99F849
:107AD80057106FF07F43002200933248FF2301F0D4
:107AE8000F01FEF7D9FF96F86B202F4B02F00F021B
:107AF8000D2A1A7005D125B92C4A412191754FF4E8
:107B080080551A78062A08D12AB2B2F5805F04D1C6
:107B1800264A3621D1754FF488551A78082A08D193
:107B28002AB2B2F5885F04D1204A3821117641F291
:107B380010151B780B2B09D12AB241F210139A4267
:107B480004D11A4B2A225A7641F211150D486FF0CA
:107B58007F4390F8F0110022009300F5F370FF23A3
:107B680001F00F01FEF798FF96F86B3013F0010F44
:107B7800AAD0E9E222AD02081A010020D559002056
:107B8800CC59002001000020140D00201F0D0020FA
:107B9800FC0000206C580020E11C00203801002067
:107BA80004020020DD0C0020723A0020F4010020BD
:107BB800900C0020A34B1A7842B300221A700F20B1
:107BC800FAF742FA06460A20FAF73EFA9E4B9F4910
:107BD80058824A7812F0010F18D06436301A588348
:107BE8009B4B1A78642A01D19B321A701B78984EE5
:107BF800FF2B0BD00A21B3FBF1F1964B19311980F9
:107C0800954822F0ADFC337801333370DFF8648295
:107C180098F8003013F00F0612D18E4B19228B48BA
:107C28001A804378192143F0010343708A4822F0EF
:107C380097FC8A4800F12001FEF70CFF04967CE2CD
:107C4800012E68D1804B5A8BA2F1690189B21129A2
:107C580008D8049911F0010F04D141F00101C9B20B
:107C680004910592049A12F0020F0DD15B8A7C4AA6
:107C78001380A3F5C263023B9BB2D72B04D80498A8
:107C880040F00203DBB204931B20FEF785FF059941
:107C9800744B0AB2632A05DD642192FBF1F230329B
:107CA8001A7401E0092A0CDD059A11B2642291FBCD
:107CB800F2F002FB10120A2012B292FBF0F23032FC
:107CC8005A74059802B2642092FBF0F100FB11216E
:107CD8000A2209B291FBF2F002FB101230329A74B8
:107CE8005B4B1B78FF2B08D158495B484B786FF3E7
:107CF80000034B70002122F033FC049A032A40F061
:107D080023825248002143786FF30003437052489E
:107D180022F026FC11E2022E03D1534BC8221A602E
:107D28000BE2032E16D1504B1B68002B40F00C823F
:107D38004A4800F14001FEF78DFE1B20FEF72CFF9C
:107D4800414B5B8AA3F51E630F3B9BB2542B00F299
:107D5800FB81F2E1042E0CD13B4B988A0FF080FE98
:107D6800002840F0F1813D4800F16001FEF772FE05
:107D7800E3E1052E07D1344B988A0FF071FE0328F2
:107D880040F0E281D9E1062E40F0D78122786FF3E6
:107D9800030301322270D5E1344800F12001FEF7D7
:107DA80059FE334B1B78002B00F0CE81237801332A
:107DB8002370304B1A786FF30302FFF794B82D4EF7
:107DC800DFF8A480337813F00F021AD12A4800F1A3
:107DD8002001FEF73FFE2948F8F72CFD2749024607
:107DE8002748F8F72FFA2548F8F724FD254BA3F87C
:107DF800160233785A1C62F3030333701CF000FD3B
:107E080091E0012A16D1D8F80030002B40F09C816F
:107E18001CF022FD012840F097811B48F8F70AFD65
:107E2800194902461948F8F735FD002840F08C81B9
:107E380011486FE0D8F80020002A40F085810B2116
:107E48007BE000BF6A130020C0310020E23100202F
:107E5800F01C00208C0C0020002C0140E2AD020830
:107E6800E41C0020F40100208826002062AE0208ED
:107E7800E01C0020E11C0020A2AE020874010020D2
:107E880060380020705D002092010020715D0020A4
:107E9800874E337813F00F080CD186484146FEF719
:107EA800D9FD33785A1C62F303033370824BA3F86D
:107EB800028049E1B8F1010F18D18048042121F06E
:107EC80078FF002800F040817A4800F12001FEF791
:107ED800C1FD33784FF0FF315A1C62F3030333704E
:107EE800774B64221A60744B59802DE1B8F1020F68
:107EF800DFF8CC811BD1D8F80030002B40F024816A
:107F08006E48042121F055FF002840F01D816A4B7E
:107F18005880684800F14001FEF79CFD33785A1CF0
:107F280062F3030333706423C8F800300CE1D8F817
:107F38000020002A40F008810C21217062F303031D
:107F4800A9E0604910234FF40052CB700D3B8B70B1
:107F58000A805D4821F0DEFE0A2200215B48F8F71E
:107F680019FA802021F03AFE237801332370504B10
:107F78001A786FF303021A70514BC8221A60E3E0B3
:107F88005348DFF848A100F12001FEF763FD9AF895
:107F98000030002B00F0D8804E48DAF80020444E1C
:107FA8000260BAF8042082809AF80620827131783B
:107FB80011F00F0159D1DFF80881D8F80010002915
:107FC80040F0C2809AF80410A2F5A6524FF0640B54
:107FD800103A0BFB01229AF805004FF00A0909FB39
:107FE80000200393F9F79CFD3B49F9F7A5FE0246EB
:107FF8009AF80200039BA0F5A65010380BFB030B60
:108008009AF80100354B09FB00B018600392F9F7A4
:1080180087FD039A01461046F9F7D2FC304B1860E9
:10802800F9F78AF91EA3D3E9002382468B46F9F7AC
:108038005DFC002800F08880504659461AA3D3E911
:108048000023F9F749FC00287ED0FEF7DDFD3378E0
:1080580048465A1C62F303033370C823C8F800303B
:1080680009F0A6FEC0B207906EE001296CD10D3070
:108078000799832200F044FD114BD3F80080B8F132
:10808800000F61D1404621F0A9FD23780133237008
:10809800337868F30303337056E000BFAFF3008012
:1080A800736891ED7CFF7F400AD7A3703D00804044
:1080B800E11C002002AF02086E3C0020000C0140C9
:1080C80088260020DE31002000100140F81C002026
:1080D80062AF02080402002000007A44F41C002069
:1080E800DC1C00208448854E00F12001FEF7B2FC1C
:1080F800F37913F0010F27D0DFF8488298F8009041
:1081080019F00F0920D17E4B0A22597818781039B6
:1081180002FB0011B1701979D878103902FB0011EF
:108128007170D9799B79103902FB0312327019F0FA
:10813800B1FCF37969F30003F37198F800305A1C25
:1081480062F3030388F80030DFF8FC9199F80060C7
:1081580016F001063EF43BAE6A4B01221A701BF082
:108168000FFB2378092B01D00D2B28D1012066495C
:1081780012F044FD654B664A5B7803F01F03D35C3D
:10818800644A522B137002D1634B01221A70634B5D
:10819800634A03F1200153F8040B8B4242F8040BA5
:1081A800F9D1002109A812F067FD09A80D211CF0DA
:1081B800C3FA5C4B1A78013202F003021A7099F87C
:1081C800006006F00206F6B2002E00F08B800FF079
:1081D800F5FE14F077FA06980322431C93FBF2F29B
:1081E80002EB42029B1ADBB20693002B79D1DFF82F
:1081F800488198F84960C246002E4DD0022E03D11E
:1082080098F80130312B49D023780E2B13D14648EA
:1082180046490522F8F73EFB8246002840D1B21FA6
:1082280037484349F8F78CFB344B5646DA7942F025
:108238000102DA7135E00D2B03D13E483A49072295
:1082480027E0032B22D13C4B002713F8012F2C2ABF
:1082580003D00137FFB2B742F7D11BA832493A46DB
:10826800F8F76EFB7B1C07E00AEB03025278303A02
:10827800D2B2092A03D80133DBB2B342F4D30AEBF2
:108288000701FA4317A80231D21802E0264911A8BB
:10829800721EF8F755FB03E0069E02E0012600E097
:1082A80000261E4B204A03F1100153F8040B8B42A1
:1082B80042F8040BF9D1214B214A03F1100153F87C
:1082C800040B8B4242F8040BF9D1402388F8113093
:1082D8001C3B88F82230023B88F84B301BF0B4FF77
:1082E80000E0002699F8003003F0F5036FF300036F
:1082F80089F80030FEF76BBDA2AF0208DC560020FB
:10830800E61C00206A1300200D5D00200C5D002093
:10831800ACE50208163B0020E01C0020F401002018
:108328007C3B00208F3A00207B590020AFA1030836
:1083380080590020F81C00207A59002004020020EF
:108348008C590020E11C002054590020AFF3008014
:1083580010B5044640181146F8F70EFA2046F8F70B
:1083680069FAC0B210BD42540131C8B2704700006A
:1083780010B50D4B0D4A1B780C460E2101FB03234B
:10838800997A39B101390523594301F56E514431C0
:1083980089B201E043F6C4310019042209F019FD3D
:1083A800201DC0B210BD00BF915F0020B017002093
:1083B80010B5054B0C46197800190131042200F05C
:1083C8009FFB201DC0B210BD915F002000F5364014
:1083D80008B54B3009F0ECFC10F0FF0F14BF00207B
:1083E800012008BD10B50A4600210446FFF7B0FF7A
:1083F80001462046FFF7DCFF114A01462046FFF7F9
:10840800A7FF232201462046FFF7ADFF014620467D
:10841800FFF7AEFF5B2201462046FFF7A4FF2322A9
:1084280001462046FFF79FFF01462046FFF7A0FFC1
:108438007C2201462046BDE81040FFF794BF00BFEC
:10844800B5A1030810B55D220446FFF78CFF0D2285
:1084580001462046FFF787FF0023235410BD38B597
:108468001D460C4640182C1911461A4600F048FBC8
:10847800E0B238BD2DE9F04118490446FFF7B2FFD4
:10848800174F0E263B78174D73430146EA5A20468C
:108498000423FFF7E4FF202201462046FFF763FF8D
:1084A8003B78014606FB035320469A7A0223FFF7DE
:1084B800D6FF202201462046FFF755FF3B780146AC
:1084C80006FB035520466A7A0323FFF7C8FF0146D7
:1084D8002046BDE8F041FFF7B5BF00BFB8A10308CB
:1084E800915F0020B01700202DE9F047264E0E229C
:1084F8003378264F534337F90380FA1824494FF449
:108508007A73044698FBF3F8157AFFF76BFF4E224F
:1085180001462046FFF727FF1E4B1C2202FB0535AC
:108528005FFA88F8B8F1030F01460CBF05F1120293
:1085380005F108022046FFF70BFFA14680460025FB
:1085480019E019F8013BA32B07D133780E2202FB5F
:108558000373204629465A7A08E0242B09D1337838
:108568000E2202FB03739A7A204629460223FFF75C
:1085780076FF0135EDB24545E3D120462946BDE8F1
:10858800F047FFF75FBF00BF915F0020B0170020E2
:10859800C2A10308CCE50208074B187800F00400D4
:1085A800C0B240B11A686FF382021A60034B00220E
:1085B8001A70034B18787047883A00201C1D002059
:1085C800041D0020054B00211970054B05481A6849
:1085D80061F382021A601222F7F7DCBE1C1D00202C
:1085E800883A0020041D002038B5084C0849227834
:1085F8000546F7F727FE23780021E954054B1A684A
:1086080061F382021A60207838BD00BF1C1D00206B
:10861800041D0020883A0020064A07491378112BC8
:10862800C85401D801331370044A136843F0040393
:10863800136070471C1D0020041D0020883A00208C
:10864800054B1B7813F0010F05D1044B181810F8CF
:10865800010CFFF7E1BF70471D1D0020E2AF0208C3
:108668002DE9F041334C002314F8101094F82A2017
:1086780001F00F0161F3030284F82A2004EB4000A3
:1086880084F8293084F828304378DFF8B88063F319
:108698000712638C4FF4D277E38498F800302A26C7
:1086A8007B4306FB0133244D2448E95A84F82A20E9
:1086B80021F054FF98F8003094F82A207B4302F008
:1086C8000F0206FB0233EB1859881C48013989B29E
:1086D80021F048FF01210A46184821F00FFF012127
:1086E800164821F0FCFE98F8003094F82A207B43C5
:1086F800120906FB02331248E95A21F02FFF98F8B5
:10870800002094F82A3057431B0906FB0376AD195D
:1087180069880B48013989B221F022FF01210A46F4
:10872800074821F0EBFE06480121BDE8F04121F0A1
:10873800D6BE00BF1E1D0020EEAF02080008004094
:10874800003401404A1D002030B5164C94F82B50D7
:10875800A38445F00105002384F82B50628484F833
:10876800211084F8203019E0C55CA5F13002D2B29E
:10877800092A08D9A5F14102D2B2052A9ABFA5F162
:108788003702D2B22A46084D013305EB420292F86D
:10879800495392F84823257062700234DAB28A424B
:1087A800E2D330BD1E1D0020EEAF0208124B10B5FB
:1087B8009A8C0024DA8483F8294083F828402246DA
:1087C80001210E4821F09AFE64210C4821F0C6FED2
:1087D80032210A4821F0C6FE01212246084821F02C
:1087E8008DFE6421064821F0B9FE05483221BDE816
:1087F800104021F0B5BE00BF1E1D0020000800403B
:108808000034014010B500212C220348F7F7C2FDBF
:10881800BDE81040FFF7CABF1E1D002070B5214CEF
:108828002378042B39D8DFE803F0030D152A30002C
:108838001D4B012093F82B3013F0010F30D020701E
:10884800013870BD184B93F82000FFF709FF022389
:10885800237022E0144DEE8CFEB9FFF7A7FF95F8C0
:10886800203095F821200133DBB29A4285F8203078
:1088780001D8042300E003232370304670BD0A4B5F
:10888800D88C50B90123237070BD074BDD8C35B9E6
:10889800FFF7B8FF2570012070BD002070BD0020D3
:1088A80070BD00BF4B1D00201E1D0020044B002280
:1088B8005A701A709A7842F001029A70704700BF95
:1088C800741E0020202102480A46F7F763BD00BF46
:1088D800F401002038B5044608460D46F7F7AAFF0C
:1088E80098B10319202B094BC8BFC4F120001C19EB
:1088F800002308E014F8012BE02A14BFEA5C2022C8
:1089080004F8012C01338342F4DB38BDF401002064
:108918000D4B46F6E9421B689B6893420FD043F61D
:10892800FC2293420BD0122B09D0B3F5E97F08D073
:1089380046F68D501B1A584240EB03007047012041
:1089480070470120704700BF841D0020F0B51F4606
:1089580087B006460C46084600211546F7F71AFD6B
:10896800244B07B19F80B3F9041005A801EB8601D9
:10897800042209F02EFA002605AB9B5D013BDBB211
:10898800B92B34D81D2B4FEA031208D8D31803F596
:1089980028416846FE31112209F01BFA0BE01649FE
:1089A800D3185B186A4603F110071868596808332A
:1089B800BB4203C2F9D12046F7F73CFFC7B268466D
:1089C800F7F738FF3818A84203D8E0196946F7F7CF
:1089D800D3FE6846F7F72EFF7B1C1B18AB4203D269
:1089E800E0190649F7F730FD0136042EC4D107B067
:1089F800F0BD00BF741E0020F07C0308DAA1030854
:108A080010B500216C220446F7F7C4FC0123A370BB
:108A180010BD002343700370837843F00103837013
:108A2800704700002DE9F0419378804613F0010F5C
:108A38000D4614463AD06FF3000393701BF0DCFB2D
:108A48006378002B32D123780BB90A336370A3788B
:108A5800174F6FF30003A3701BF0CEFB217807EBD1
:108A680008066118073130462A46F7F769FF30468D
:108A7800F7F7E0FEC6B2AE420DD80AD20023237043
:108A880006EB08000A33637038182021AA1BF7F791
:108A980081FCAE420AD12278A3181B7A1BB101329D
:108AA8002270BDE8F08123700A236370BDE8F0816D
:108AB800F4010020054B1A780AB100221A701B78BD
:108AC80046F68A4202FB0311FFF704BF671D002028
:108AD800F8B505460C460818002109F05FF9013C75
:108AE800E4B26719384609F063F9C6B2202E03D8F4
:108AF8003846002109F052F90CB1202EEFD9F8BD03
:108B080002F00F03032B22F07F0230B5D2B20CD94A
:108B18004FF47A7491FBF4F42025E4B2057002B1A5
:108B280014B13034047000220130B1F57A7F05DBCE
:108B38004FF47A7491FBF4F504FB1511022B0BD951
:108B4800642491FBF4F42025E4B2057002B114B159
:108B58003034047000220130632904DD642491FB61
:108B6800F4F504FB1511012B0AD90A2391FBF3F341
:108B78002024DBB2047002B10BB130330370013032
:108B8800092904DD0A2391FBF3F203FB12113031AA
:108B9800017030BD13B5104B01461B689A899C7B48
:108BA80012F0100214BF0220012034B10B4C9B7C40
:108BB8002478634303FB001109B23AB10DF10600B2
:108BC800022209F006F9BDF8060002E0084609F09D
:108BD800EFF800B21CBD00BF841D0020131E00204A
:108BE80010B50F4B1B689A899C7B12F0100214BFBA
:108BF8000221012134B10B4C9B7C2478634303FB95
:108C0800010000B22AB108490222BDE8104009F06B
:108C1800DAB8054B1968BDE8104009F0BFB800BFC5
:108C2800841D0020131E00202C1E00203038C0B2E6
:108C3800092894BFFF20002070470000024B1A78D3
:108C48006FF300021A707047631E002070B5FFF7BB
:108C5800F5FF884B1A781E2A01D91E221A70864CF5
:108C68002678254606F0F006202E72D109F004FC7D
:108C780000286ED1814B1B7833B92378C3F30312D4
:108C8800013262F307135EE07D4B1B7803F080032B
:108C9800DBB2002B59D07B48F7F7CCFDC5B27A4C34
:108CA800BDB1204679493246F7F74AFE0A2D0BD85E
:108CB8002A4620467349F7F743FE60193146C5F145
:108CC8000A02F7F767FB04E020466E490A22F7F725
:108CD80037FE6F4B1B7813F0010F01D0472300E0DC
:108CE8002023E372684C042204F10C00A521F7F755
:108CF80051FB684B1A7852B1FF23012A237306D916
:108D0800022A637303D0032AA37318BFE373624C68
:108D1800257815F0600502D194F8A33013B95F489F
:108D28005F4902E05D4804F1A3010622F7F708FE57
:108D38005C4B1B78452B40F08D81002D40F08A81DB
:108D4800237843F08003237070BD4F48564932465C
:108D580075E12C7804F0F004102C3FD109F08CFB5D
:108D680000283BD1202251494748F7F7E9FD4648FA
:108D78004E492246F7F7E4FD4D4B1B7813F0010FDF
:108D880006D04C48F7F756FD4A4902464A4805E0DE
:108D98004A48F7F74FFD494902464748F7F7D0FDDB
:108DA800364B1B781BB946484649102247E14448D0
:108DB80045491022F7F7C4FD314B1B7803F08003B7
:108DC800DBB22BB13B48F7F735FD02463F484FE091
:108DD8003A48F7F72FFD02463C4842E02B7803F06B
:108DE800F003302B7ED109F047FB00287AD1264CBE
:108DF800202237492046F7F7A3FDA521052204F1D3
:108E08000B00F7F7C7FA334B1B78042B02D9FF2363
:108E1800E37300E002D1FF23A37301E0032B02D127
:108E2800FF23637301E0022B02D1FF23237300E0C9
:108E38000BB1FF23E372284B5B7813F0600F05D06A
:108E48003F23E37223736373A373E373234B1B788A
:108E580003F02003DBB233B11848F7F7EBFC024606
:108E68001F481649EBE01348F7F7E4FC02461C4894
:108E78001049E4E06F1E0020631E0020B826002081
:108E88008C26002090260020F4010020DC420308F4
:108E9800885F002086270020C12600200E020020BF
:108EA800F71803084C1D00209A420308DF780308CE
:108EB8004A3E0020297A0308010200204A7A030862
:108EC80004020020AC7E0308007903081102002088
:108ED8009C190308AF2C0020E8310020883A0020B4
:108EE8000F0200202B7813F0F0030CD120225A49EE
:108EF8005A48F7F725FD5A4B584819888322BDE888
:108F08007040FFF7FDBD602B1ED109F0B5FAD8B946
:108F1800544920225148F7F713FD5348F7F78AFCC4
:108F2800514902465148F7F70BFD5148F7F782FCC3
:108F38004F4902464F48F7F703FD4F48F7F77AFCC9
:108F48004D4902464D487AE02B7803F0F003102B88
:108F580006D109F091FA18B14048494920226EE03B
:108F68002B7803F0F002402A02D0502A6BD10AE095
:108F7800444920223948F7F7E3FC0FF09DFD0446E9
:108F88000FF0B8FD09E0404920223448F7F7D8FC33
:108F98000CF070F904460CF091F9FF2806D13B4813
:108FA800F7F748FC39490246394817E0FD2806D149
:108FB8003848F7F73FFC3749024635480EE00228A3
:108FC80006D13548F7F736FC33490246304805E004
:108FD8003248F7F72FFC314902462D48F7F7B0FC25
:108FE800202107222E48F7F7D5F9FE2C06D127486D
:108FF800F7F720FC25490246294820E0012C06D134
:109008002848F7F717FC27490246254817E0022C9D
:1090180006D12548F7F70EFC2349024620480EE002
:10902800042C06D12148F7F705FC204902461C48C4
:1090380005E01F48F7F7FEFB1D4902461848BDE842
:109048007040F7F77DBC1B4A6FF3071313701A4B78
:1090580000221A6070BD00BF39190308F40100200E
:10906800621D00201819030818120308F8010020CF
:1090780022120308080200201D1203080F02002014
:109088007B19030821790308427903086B7A0308DE
:10909800FD0100208C7A0308E7790308297A030880
:1090A8000D0200206379030884790308A579030871
:1090B800C6790308631E0020841D0020204B70B56C
:1090C800F022204D1A702B7813F0010F0BD01E4C94
:1090D800207810F0010006D11C49FFF7EBFC23783B
:1090E80043F0010323701A4E3378532B0ED1164CDC
:1090F800237813F0010F07D000201649FFF7DAFC98
:1091080023786FF300032370FFF798FD3378232B40
:1091180014D10D4B1B7813F0010F0FD1FFF78EFD03
:109128002B780D4A43F006032B701378013BDBB212
:1091380013700A4A52F82320094B1A6070BD00BF09
:109148006F1E0020631E0020891D0020B06E0308DA
:109158004C1D00208F6E0308431E0020501E002067
:10916800841D00202DE9F0415C4BF0225C4D1A7003
:109178002A7802F01003DBB2002B2DD1594963F392
:1091880047120B601C462A70574A9A5C2D2A01D058
:109198000134E4B20133082BF6D1544E3A2130465B
:1091A800F7F776F938B1801BC0B201303018214684
:1091B8000222FFF7A5FC4E4B1B78452B40F08B8015
:1091C80000242046013413F0D5FA082CF9D12B7865
:1091D80043F010032B7038E0464C237813F0010F4E
:1091E80017D1404E4448FFF70BFC404F31683846D2
:1091F80001310222FFF784FC2D23BB70307846F63C
:1092080015733E496522FFF7A1FB237843F001035C
:10921800237003200D21384AFFF704FC2D78304EC7
:1092280015F0E00541D110203549FFF743FC304BDC
:109238001B78442B0DD12B4A136801332A4903F0BC
:109248000703C95C2D29F8D01360BDE8F041FFF78A
:10925800F5BC532B0DD132784E3B63F34712327075
:10926800204A28491268062000FB02125380BDE8F4
:10927800F081232B2FD11B4B1D60337803F0EF03B4
:1092880065F347133370FFF7D9FC23781E4A43F080
:10929800060323701378013BDBB213701B4A52F8A4
:1092A80023201B4B1A60BDE8F081104C102019498F
:1092B800FFF700FC04F110002821F7F7E9F850B196
:1092C800001B3178C0B20130201849098022BDE85E
:1092D800F041FFF715BCBDE8F08100BF6F1E00200C
:1092E800891D00202C1E0020513C0020F401002084
:1092F8004C1D0020631E0020741E00207B1E0020D1
:109308002C6E03086E3C0020431E0020501E0020D7
:10931800841D00204D6E0308454B2DE9F041F022D5
:10932800444E1A703378444D43F0010333702B6870
:10933800424C9B7C022B06D1414B1B7803F0400327
:10934800DBB23BB10FE0012B0DD13E4B1B7813F084
:10935800010F08D109F008FA236800206FF355536C
:109368002360394944E0A378344F03F02003DBB28B
:10937800C3B909F0F9F9F87800F02000C0B288B94B
:109388002968324B897C1A7861F301021A703B68AC
:109398002D4943F400133B60FFF78CFB2C4B8022D4
:1093A80083F843200DF00CFF804678B12B689B7C36
:1093B800012B08D1234B5B7803F01003DBB213B108
:1093C8000020244914E00020234911E00DF028FF73
:1093D800074610B1404621490AE00DF069FF10B177
:1093E80038461F4904E01A4B93F8433013B91D4916
:1093F800FFF760FB1C4B1B78232B16D1FFF71EFCD5
:10940800337843F00603337009F0AEF923686FF33D
:10941800555323600CF08EFD144A1378013BDBB2E0
:109428001370134A52F823302B60BDE8F08100BF57
:109438006F1E0020631E0020841D0020883A002033
:109448008C2600204A3E0020D16E03084F3E0020A3
:109458000D220020136F0308F26E0308556F0308EE
:10946800346F0308766F03084C1D0020431E00204C
:10947800501E00202DE9F341704B714DF0221A70F7
:109488002B68704C9B7C1BB9637843F0020302E0A5
:10949800637843F001036C4E6370337843F0010343
:1094A8003370238823F4FF739B059B0DB3F5007F6E
:1094B80007D0664B1B787BB1624B5B7813F0010FCA
:1094C8000AD0237800206FF3861361492370FFF7D1
:1094D800F1FAF8F7F5FD84E023785A4F03F04003DA
:1094E800DBB2FBB9BB78EBB95A4B93F8008018F0A4
:1094F800010817D1F8F7E4FD3B7843F040033B70CF
:109508002B68B3F91030022B3B780CBF43F0800373
:1095180068F3C71300213B70082001220B46009115
:10952800F9F7EEF8A378474A032B28D003D8012B84
:109538000BD00DD806E0052B2DD0117825D3FF2BA5
:1095480032D12BE00020424949E00020424946E060
:109558004248F7F76FF9DFF83C81C7B23F4908F195
:1095680010003A46F7F7ECF90F2F3AD807F1100038
:1095780040442021C7F11002F6F70CFF31E0384BC8
:10958800187800282DD1374929E06FF3861111701A
:109598000020354923E00020344920E06FF386118C
:1095A8001170002032491AE0053BDBB26FF38611D7
:1095B800022B117002D100202E4910E0012B02D19C
:1095C80000202D490BE0032B02D100202B4906E097
:1095D800052B02D100202A4901E02A490020FFF783
:1095E80069FA237803F04003DBB20BB9F8F768FD9A
:1095F800254B1B78232B1ED1FFF720FB33782278CD
:10960800617843F00603337001F0FE01002302F095
:10961800BF0263F3C71263F34101A3702270617044
:10962800F8F74EFD194A1378013BDBB21370184A5C
:1096380052F823302B60BDE8FC8100BF6F1E00206C
:10964800841D0020885F0020631E002082360020D1
:10965800D16E03088E5F0020146B0308975F00200B
:109668008C5F0020356B0308D96F0308B96B0308BA
:109678001C6C0308566B0308776B0308986B030888
:10968800DA6B0308FB6B03084C1D0020431E002007
:10969800501E0020F40100207B4B2DE9F341F022FD
:1096A8007A4E1A7033787A4D43F0010333702B6881
:1096B800784C9B7C022B11D1774B1B7803F040032D
:1096C800DBB293B1754B1B7803F02003DBB2BBB15F
:1096D800A37803F04003DBB23BB111E0012B0FD1BB
:1096E8006F4B1B7813F0010F0AD1F8F7E9FC2368D8
:1096F800002023F480036FF3D753236069498FE078
:10970800A778DFF8908107F04003DFB2002F34D14B
:10971800F8F7D6FC2968644B897C1A78384661F3D7
:1097280001021A70D8F800305E4943F4800367F3E9
:10973800D753C8F80030FFF7BDF92B68198A21B94B
:109748000091082001220B4615E00BB2022B0CD128
:1097580001223B46082039460097F8F7D1FF534BC2
:109768001A7842F008021A7007E0012B05D1009719
:109778000E2039463A46F8F7C3FF0DF021FD07469B
:1097880078B12B689B7C012B08D1454B5B7803F0A3
:109798001003DBB213B10020454941E000204549E0
:1097A8003EE0414B3946187800F00300F8F7C2FD57
:1097B800FF280FD13D4B1B7803F01803182B31D02D
:1097C800A07800F08000C0B210B138463A4927E0CE
:1097D8003A4925E00DF024FD8046E0B1334B187876
:1097E80000F008085FFA88F8B8F1000F0AD1F8F716
:1097F800F7FEC0B2022801D840460AE0062811D870
:10980800404604E000F01000C0B210B138462C49C0
:1098180006E02C4904E00DF04BFD18B12A494046FA
:10982800FFF748F9294B1B78232B29D1FFF706FAB4
:10983800337843F006033370F8F742FC236823F4C7
:1098480080036FF3D7532360184B1A786FF3C30262
:109858001A701F4A1378013BDBB213701D4A52F885
:1098680023302B60104B1B7803F00303022B02D12B
:109878000DF07CFC20B102B0BDE8F0410CF05ABB01
:1098880002B0BDE8F08100BF6F1E0020631E0020FB
:10989800841D0020883A00208C260020C126002044
:1098A8004A3E0020D16E03084F3E00209C1F002036
:1098B800136F0308F26E0308D96F0308FA6F0308E1
:1098C800B86F0308976F0308346F03084C1D002016
:1098D800431E0020501E002010B5FFF7AFF90A48BC
:1098E8002523C377094B0A4A1B6824219B7C1C301B
:1098F80001FB03235B781A3903F00F0359438322D2
:10990800BDE81040FFF7FCB8F4010020841D0020DA
:10991800903A00202DE9F047514D524F2B78F02214
:1099280043F001032B70504BDFF878911A703B68B5
:109938009C6847F67313E21A544244EB020424214C
:1099480061434A4A565C5318C6F300065FFA86F824
:109958009246B8F1000F23D140464549FFF7AAF8CF
:1099680099F80030232B79D1FFF768F92B78414A11
:1099780043F006032B701378013BDBB213703E4AA9
:1099880052F823303B603D4B1E703D4B1E703D4BE3
:109998001E703D4BC3F800803C4B1E70BDE8F0873D
:1099A80099F80020232A21D19A786FF300029A703F
:1099B8000EF0B0FBFFF742F92B782E4A43F006036E
:1099C8002B701378013BDBB213702B4A52F823300B
:1099D8002A4A3B6000231370294A1370294A1370DE
:1099E800294A1360294A1370BDE8F087532A13D116
:1099F8009A7812F001010FD172206043244D42F091
:109A080001022E5C61F300062E549A701E4B01224F
:109A18001A60204617F06CFA242303FB04A39B78F2
:109A280013F0010F02D000201A4913E0164B1B68EF
:109A380073B9382102221848FFF762F8204616F059
:109A4800D7FC014615480222BDE8F047FFF758B891
:109A580013490020BDE8F047FFF72CB8BDE8F087B0
:109A6800631E0020841D00206F1E0020903A0020F5
:109A780067270308431E0020501E0020691D002090
:109A8800921D0020131E00202C1E00201E1E0020E8
:109A9800E85500200A720308120200200D02002077
:109AA800E97103084C1D00202DE9F0412D4E2E4F81
:109AB800307800F5E640713008F07AF93B78C4B2A6
:109AC80013F0010F26D0294D2B78552B0AD1EC2CF9
:109AD80001D0013CE4B23078214600F5E64071300F
:109AE80008F05CF92B78442B0DD1A4F11403DBB2F8
:109AF800D72B01D90134E4B23078214600F5E6408D
:109B0800713008F04BF92B78532B03D1FFF796F8F7
:109B18000EF000FB164B1B7803F08003DBB253B149
:109B28003B7813F0010F06D0124820210422BDE82B
:109B3800F041F6F72FBC14F0800F0F4805D12B2306
:109B48000A2103746143113006E02D230374373B67
:109B58005C43113004F520610322BDE8F041FEF7B3
:109B6800CFBF00BF131E0020631E00204C1D002025
:109B7800883A002004020020F40100201FB5204B81
:109B880020491A781AB1087840F00100087009785D
:109B98001C4C11F0010F31D01B490978532901D011
:109BA8000AB103E082B901221A700DE023290BD112
:109BB800002018701549FEF77DFFFFF73FF823785E
:109BC80043F00603237019E01B78012B16D12021DE
:109BD8000A460F48F6F7DEFB0E4B68461B68102254
:109BE800996808F0F6F8002409491DF8040001EB0B
:109BF800440101341BF056FC102CF5D11FBD00BFE9
:109C0800131E0020631E00204C1D0020227503082F
:109C1800F4010020841D0020034B1B78532B01D135
:109C2800FFF70CB8704700BF4C1D0020084BFF28F9
:109C38001A68936807D1917B41B10649927C0978EB
:109C480001FB023302E0927C02FB003318467047A6
:109C5800841D0020131E00204328F8B504460D4635
:109C6800174608D1114B0A261A7891FBF6F66FF3BE
:109C7800C3021A7000E00E462046FEF7D7FF90B1E7
:109C88000A4B303C1A780A2602F00801C9B20029AA
:109C980018BF002506FB05466FF3C30236B21A70DB
:109CA800BE42A8BF3E4630B2F8BD00BF631E0020CA
:109CB800614B2DE9F3411A689846157C977C5F4CF7
:109CC8002DB15F4821780222FEF71AFF00E02570C7
:109CD800FF01237807F51E47E83707EB4307594E7E
:109CE8000BB90DB10FE015B901A8394601E001A87B
:109CF800B91E022208F06DF89DF80430F3759DF83E
:109D08000530337605E006F117003F210222F6F709
:109D180041FB5B23B375023373764B4B1B7813F00F
:109D2800010F5DD0494B1B78A3F13002D2B2092A4A
:109D380031D822780AB9002D3CD1454A1178964687
:109D48009942444A01D00021117043481178A3F187
:109D5800300490F800C004EB840404EB010802A866
:109D680001318444C9B23D48641810F80880005D88
:109D78000CF8048C117008B1032901D90021117065
:109D88008EF800300DB9384600E0B81E01A902224D
:109D980008F019F817E0232B04D12F4B1A7892B941
:109DA800013205E02A2B05D12B4B1A785AB1013A1A
:109DB8001A7008E0532B06D1294A533B1370264AE0
:109DC8001370FFF729FF274B1B7803F08003DBB2E2
:109DD800002B2FD0204B1B78F6182023F37529E091
:109DE80045B31A4B1878A0F13003DBB2092B10D811
:109DF8001B4A137803B92370013303F0010313706E
:109E0800D8F800302178B3F91020FFF725FF20702B
:109E180005E0432803D1124B1B7803B92370114B7B
:109E28001B7803F08003DBB223B10548202102220E
:109E3800F6F7B0FABDE8FC81841D0020931D0020D0
:109E480002020020F4010020631E00204C1D0020A7
:109E5800661D0020921D0020641D00205CB30208CE
:109E68001E1E0020883A0020F7B5384E384D33784A
:109E7800384C6FF34103337019F0B0FFFFF7CCFE95
:109E880002238DF807302B7883B1334AD17941F01A
:109E98000101D171314A207802EBC3035F6B93F85B
:109EA80039203978FFF7D8FE38700DE0337813F091
:109EB800010F06D02378303BDBB2062B9CBF264A25
:109EC800D37003238DF80730337813F0010F12D0C5
:109ED800234B1B7803F08003DBB263B129781F4B57
:109EE800204803EBC10393F838309DF80720C018C9
:109EF8002021F6F74FFA2378232B09D11A4A2B7819
:109F08001268927C013A934202DA114A01331370C3
:109F180023782A2B04D12B7813B10D4A013B1370F7
:109F28002378532B0FD117F0B5FD0B4B0021297067
:109F3800DA7961F30002DA71FFF76EFE0B4B9A795A
:109F480042F004029A7100232370FEBD631E0020B4
:109F58001E1E00204C1D0020DC5600205CB30208A9
:109F6800883A0020F4010020841D0020901F002062
:109F78002DE9F74F864E874C3378874D232B874F33
:109F880025D12368986843F6F123984217D1DFF862
:109F98003482296898F8000000F56A50713007F09B
:109FA800FDFE98F80000013000F0010088F800007C
:109FB80000F56A50713007F0FBFE286007E000B238
:109FC800FEF7E8FD28603B7843F008033B703378E0
:109FD800532B40F06E81236849F695629B68934243
:109FE80002D12A686E4B15E04BF23662934202D1D9
:109FF8002A686C4B0EE04BF2B352934202D12A68A6
:10A00800694B07E049F6E662934204D12A68674B38
:10A0180002B101221A7023689A6843F6DD239A4236
:10A028000AD1634B29681A7861F300021A7008F0A4
:10A0380023FA08B108F03EFA236843F6E0229B6849
:10A04800934206D15A4B29681A7861F3C7121A70DD
:10A0580019E043F6EA22934206D1554B29685A780B
:10A0680061F300025A700EE043F6E72293420AD1E8
:10A078002968504B19B11A6842F0005202E01A6878
:10A0880061F35D721A6023689A684BF2CC639A4256
:10A098000AD12968484B19B11A7842F0040202E043
:10A0A8001A7861F382021A7023689A684BF259731E
:10A0B8009A4202D128781AF0F9FB236843F6DA228B
:10A0C8009B68934202D12A683C4B05E043F6DE22A6
:10A0D800934203D12A683A4B1A7008E049F69E6207
:10A0E800934204D12B6813B92B4B01221A602368C1
:10A0F8009A684BF25A739A420BD1324A2B681278FB
:10A108003149032B8B5404D1304B5A7942F0100259
:10A118005A71236849F6DE629B68934202D1296826
:10A128002B4A05E049F6E162934203D12968294A9E
:10A13800117016E049F6E262934203D12968264A73
:10A14800117015E049F6E462934203D12968234A65
:10A1580011704DE049F6E562934202D12A68204B1E
:10A1680013E043F60852934202D12A681D4B0CE0D3
:10A178004AF6EC02934202D12A681B4B05E04BF2E7
:10A188004A62934234D12A68184B1A703BE000BFE8
:10A198004C1D0020841D00202C1E0020631E002062
:10A1A800B8260020703A0020673400204A1D00209D
:10A1B800E11E0020883A0020885F00206A590020AC
:10A1C800E63A0020131E0020A81700206026002071
:10A1D8001C3F00201A3F00204D3E0020C13D0020BA
:10A1E80010200020E6150020811C0020021D002000
:10A1F80049F69662934206D12A68A04B01201A704C
:10A2080001460EF0C1FD2368986843F6F123984291
:10A218000DD1DFF87482296898F8000000F56A50BB
:10A22800713007F0BBFD002388F8003002E000B26F
:10A23800FEF7D6FC23689A6843F698139A4236D1FB
:10A248002968DFF840B2DFF848A20BEBC1031B799D
:10A25800DFF83482C3F34113012BDFF8389221DD94
:10A2680098F8000000F56650203007F097FD98F840
:10A278000030DAF8001009EB030211720BEBC1028F
:10A288001279C2F34112032A0CD17D4A12689068F0
:10A298001030C01807F082FD98F80030DAF8002076
:10A2A8004B441A7498F800302A6809F80320FFF71D
:10A2B800B3FC3B78DFF8E08113F0010F00F0EE808B
:10A2C800216843F698128B68934240F081806D4A6A
:10A2D8002B68914602EBC3010979C1F341110129A9
:10A2E80006DD694A1278072A02D9FEF7A7FCE1E0E1
:10A2F8003278442A36D15FFA83F82DE008F1010854
:10A30800604B5FFA88F803EBC8031B79C3F341136A
:10A31800012B06DD5D4B1B7823BB5B4B1B78072BA2
:10A3280020D8DFF864A19AF800301F2B08D808F06D
:10A33800A3F870B109EBC8031B7913F0100F08D10B
:10A348009AF800301F2B07D909EBC8031B79DB09E2
:10A3580002D0C5F8008005E009EBC8031B7913F0AB
:10A36800080FCBD03378552B40F0A4802E782CE002
:10A37800013EF6B209EBC6031B79C3F34113012B67
:10A3880009DD424B1B78002B40F094803E4B1B7834
:10A39800082B00F28F80DFF8F08098F800301F2B30
:10A3A80008D808F069F870B109EBC6031B7913F0F7
:10A3B800100F08D198F800301F2B06D909EBC603F7
:10A3C8001B79DB0901D02E6074E0002ED0D171E03A
:10A3D8004BF25A7293420AD005DCA3F536424A3A48
:10A3E800012A0ED803E04BF2B772934209D13378B1
:10A3F8002F2B5FD9B1F91020303293425ADC303B11
:10A4080030E043F6F122934207D11F4B1B7823B16A
:10A418003078B5F900103B222CE008F02DF818B37D
:10A42800236843F6C4219A688A4203D047F28121FF
:10A438008A4204D13078B5F900102D221AE0A2F52D
:10A448006A516139052903D943F6E9218A4201D1C4
:10A45800012307E043F6E0218A4202D00A318A420A
:10A4680003D100232B6025E023683078B5F900106C
:10A47800B3F91020FFF7F0FB28601BE0C23C002076
:10A48800841D002014040020131E0020820D0020CB
:10A498002C1E0020B02C0020631E00202368B3F976
:10A4A8000800FEF777FB286098F8003043F00803AF
:10A4B80088F80030FFF7B0FB236843F6D22298688B
:10A4C80090420BD12B6813B99C489D4901E09B48E9
:10A4D8009C490222F6F734FA0226B0E14BF2B77231
:10A4E80090420AD12B6813B99748984913E0012B79
:10A4F80095480CBF964997490DE04BF25A72904225
:10A5080018D12B68012B02D18F48934903E0022B05
:10A5180005D18D4891491022F6F712FA8EE1032BE6
:10A5280002D189488E49F6E7042B87480CBF8D492C
:10A538008D49F0E74BF24A6290420AD12B6813B971
:10A5480081488A49E7E7022B7F480CBF8849894937
:10A55800E1E74BF24B6290420AD12B6813B97A4873
:10A568008549D8E7012B40F0698177488349D2E7CC
:10A5780049F6E362904203D043F6EE2290420ED1B0
:10A5880028680A21B0FBF1F201FB12017C4B303143
:10A59800D97730322E2199775A7703264FE143F63F
:10A5A800F12290423ED1774B1B78E3B90222296809
:10A5B8007548FEF7A5FA43F6F220FEF7EBFA0222F9
:10A5C80001465E48FEF79CFA3B7813F0010F00F055
:10A5D80086816E4B1B7803F08003DBB2002B00F002
:10A5E8007E81694819E0FEF7D5FA022201466648DD
:10A5F800FEF786FA022251482968FEF781FA3B786D
:10A6080013F0010F00F06B81604B1B7803F080039F
:10A61800DBB2002B00F06381484820210222F5F7C5
:10A62800B9FE5CE143F69812904240F0F5802B6841
:10A63800574EDFF8508156F8331010224248F6F78B
:10A648007FF90DF1060298F800000DF1070110F0EE
:10A6580071FC4246334620B316784E49895D03297A
:10A668001FD0296803EBC1010979C1F34111012900
:10A6780017D1072E15D948490B224848F6F760F933
:10A688004748711C0222FEF73BFA9DF8071045481F
:10A6980001310222FEF734FA9DF8061042480131D2
:10A6A80018E02E68157803EBC601097903EBC60696
:10A6B8003679C1F34111012906F00706C8BF05F034
:10A6C8000705012E0ADC394934480B22F6F738F918
:10A6D8003348691C0222FEF713FAAFE0022E0BD1B1
:10A6E80033490B222D48F6F72BF932462C48691CC2
:10A6F800FEF706FA0E36A2E0032E0BD12D490B22E7
:10A708002648F6F71DF92648691C0222FEF7F8F9D3
:10A718000D3694E0042E51D127490B221F48F6F735
:10A728000FF91F48691C0222FEF7EAF91D4805F1D6
:10A7380009010222FEF7E4F90C3680E0120200203B
:10A74800C0B30208C2B3020804020020066103086D
:10A758004861030827610308DD5F0308FE5F0308FB
:10A768001F60030840600308BC5F0308AB6103086F
:10A77800ED610308CC6103082F62030850620308E7
:10A78800F4010020131E00200F020020883A002048
:10A7980014040020B02C0020947B0308F901002049
:10A7A800FA010020FE01002001020020527B03086C
:10A7B800AD7A0308317B0308EF7A0308052E11D11F
:10A7C80048490B224848F6F7BBF84848691C02225A
:10A7D800FEF796F9464805F109010222FEF790F9BD
:10A7E8000B362CE0062E29D142490B223E48F6F7BB
:10A7F800A7F83E48691C0222FEF782F93C4805F199
:10A8080009010222FEF77CF93B4805F111010222F9
:10A81800FEF776F90A3612E0B3F91060092E04DD66
:10A82800632ECCBF0326022600E0012633482968A0
:10A83800801B46F08002FEF763F900E010263B78A3
:10A8480013F0010F0BD02E4B1B7803F08003DBB203
:10A858002BB12A482021801B3246F5F79BFD294E53
:10A86800B37803F00203DBB2002B38D0FEF750F8C0
:10A87800254D034628B92878F11D6522FEF766F8AC
:10A8880008E0B2792978B388F01D01FB023109B2DA
:10A8980007F09FFA236847F281229B68934213D0FE
:10A8A80006DC43F6C42293420ED043F69E5209E0DA
:10A8B80047F20132934207D049F69E62934203D091
:10A8C80047F2C12293420AD105200B210D4AFEF717
:10A8D800A9F829780D4801310222FEF711F9BDE8DF
:10A8E800FE8F00BFCE7A0308F9010020FA0100208C
:10A8F800FE010020107B0308020200201402002041
:10A90800883A0020741E0020131E0020F501002044
:10A91800F0B5114B1F78114B303F1E680DE0D6F88B
:10A9280014C01CF803C00133644501D112E00023B0
:10A93800DAB28242F3D301350D70094B0622094978
:10A9480002FB07330D785B1993F86840002CEED1B1
:10A958000C70F9321046F0BD4C1D0020841D0020FB
:10A968005CB30208921D00202DE9F74F974C984ED2
:10A9780023689A6843F609539A4203D133780BB98E
:10A98800013333702368934F9968B3F910303A78DC
:10A99800B3F1010848BF03F106084FEAE808337825
:10A9A80008F1010812F0010F03FB08188A4D00F0A6
:10A9B800AD808A4B1A789946432A4DD128780FFAE8
:10A9C80088FA0AEBD00007F0F3F92268844B916803
:10A9D80046F648029142186001D12A783AB12A789D
:10A9E800012102F0070211FA02F25040186028789B
:10A9F80019780AEBD00007F0D1F9236847F26132E1
:10AA08009B68934209D1744B1A78764B03EBD203B7
:10AA1800734A126883F8A0211EE046F62952934231
:10AA280005D13178002001310EF028FD14E046F6FA
:10AA38003F1A4FF0000B23689B68534504D101204F
:10AA48000BEB00010EF01AFD0AF1080A46F65F1337
:10AA58009A450BF1010BEED199F80030232B10D158
:10AA680022682B78927C013A93420ADA5A4A0133D7
:10AA780013705D4B9B7803F00203DBB20BB1FDF75B
:10AA880015FF99F800302A2B0CD12B7853B1524A74
:10AA9800013B1370544B9B7803F00203DBB20BB1FC
:10AAA800FDF704FF99F80030552B14D12368997CE1
:10AAB8000F2910D92A7808398A42474B01DA083217
:10AAC80000E000221A70484B9B7803F00203DBB2C7
:10AAD8000BB1FDF7EBFE99F80030442B42D1236807
:10AAE8009A7C0F2A3ED929783B4B072902D9083985
:10AAF800197001E0083A1A703B4B9B7803F0020387
:10AB0800DBB2002B2ED0FDF7D1FE2BE049F65563C2
:10AB180099420ED1314B1B78A3F13101C9B20329F7
:10AB280007D842F006023A7007225343284A573B97
:10AB3800137023689A6843F609539A4212D13378FE
:10AB48001B2B08D9284B46F615629A809A7842F052
:10AB580002029A7006E05901C918244B0020C9184E
:10AB6800FDF7A8FFFFF758F8214A2B78117893468C
:10AB7800994288BF137012780F32934202DD1C4A43
:10AB88000F3B137023684FF0000A93F81290B9F145
:10AB98000F0F9ABFC9F120095FFA89F94FF0100920
:10ABA8009BF800004FFA8AF318180FFA88F202EBA4
:10ABB800E000019307F0FCF89BF80020019B5FFA86
:10ABC80080FC9B1803F007032BE000BF841D0020C6
:10ABD800131E0020631E00201E1E00204C1D002096
:10ABE8002C1E0020B02C0020741E00206064030876
:10ABF800151E00204CFA03F06549013300F00100EE
:10AC080000280CBFA520DB20DBB201F809000AF1FF
:10AC1800010A09F10109082B5FFA8AFA5FFA89F932
:10AC280003D0B9F1200FE5D109E0B9F1200F06D022
:10AC380023684FFA8AF19B7C89189942B0DB3B78EC
:10AC480013F0010F15D0236852499B7C09780F2B0C
:10AC580001F0800198BFC3F11003C9B294BFDBB201
:10AC6800002331B1297810318A1A4949CB185F215C
:10AC78009954DFF8288198F80230474603F0020318
:10AC8800DBB2002B64D0FDF743FE034600BB22680D
:10AC980046F6295192688A4206D024318A4203D066
:10ACA80043F6E5118A4204D130783B4965220023F6
:10ACB80009E043F609518A4208D130781C38C0B2FD
:10ACC80008F107016522FDF741FE18E02878F7E74B
:10ACD800236846F6E9429B68934203D043F6FC2278
:10ACE800934202D1BA79317801E0BA792978BB88E0
:10ACF800294801FB0231BA7909B207F06AF82368DA
:10AD08009A7C102A02D905200B211EE09B6846F682
:10AD1800E94293420ED006DC43F6E512934209D08D
:10AD280043F6FC2204E046F62952934202D024322C
:10AD3800934201D1102007E043F60952934202D111
:10AD48000020102101E000200721144AFDF76AFEC7
:10AD5800226846F68D5193688B4216D046F64741D5
:10AD68008B4212D043F6ED218B4202D1084BDB21F6
:10AD78009977937C102B08D9297809480131022248
:10AD880003B0BDE8F04FFDF7BBBE03B0BDE8F08FE0
:10AD9800F4010020883A00207B1E0020741E002049
:10ADA800F5010020114B002270B50D461A7118B13B
:10ADB8001B7803B920234370BDB10D48F5F73AFD60
:10ADC8000446681C5CB10A492246F5F73BFA022C96
:10ADD8000BDC601C28182021C4F1030201E02021AB
:10ADE8000322BDE87040F5F7D5BA70BD001E0020FB
:10ADF800011E002038B50546002408E0601906F059
:10AE0800D7FF3038C0B2092808D80134E4B2044B5F
:10AE18001B78303B9C42F1DB012038BD002038BD57
:10AE2800681D002008B506F0C3FF0023C0B2064A1B
:10AE3800D25C824201D1202804D10133082BF6D1FB
:10AE4800002008BD012008BD00B4020870B5064600
:10AE58000D4600240DB12D232B55A01900210134D6
:10AE680006F09CFF062CF5D170BD00002DE9F04FCF
:10AE7800974C984F206839788368068A9AB201FB04
:10AE880006260D4648F6BC218B4287B0B6B20BD1D8
:10AE9800914B1A785B7802F00702C3F3420303EB85
:10AEA800C20306EBC3062BE048F67C418B4212D165
:10AEB800894B8A481A78597802F0070288235A433E
:10AEC800C1F34201773B03FB012320210822F61836
:10AED800F5F760FA14E049F234018B420BD17E4B4E
:10AEE8001A785B7802F00702C3F3420303EBC2034C
:10AEF8009B01F61804E0B3F5E97F08BF02EB4506AD
:10AF0800774B784D1A78984612F0010F53D1236881
:10AF18009A6847F289139A4204D046F689739A428E
:10AF280040F04481704B1B782A2B3BD16F4B93F830
:10AF3800009009F1010909F0010983F80090B9F1BD
:10AF4800000F1AD046F689739A4208D1684B46F624
:10AF580015629A809A7842F002029A7026E12021BE
:10AF680010226448F5F716FA3B7800205901C918F1
:10AF7800614BC918FDF79EFD18E15D48FDF740FDDE
:10AF8800236848469A6846F689739A420CBF5B491B
:10AF98005B49FDF78FFD39785A4801310222FDF7E8
:10AFA800AFFD03E1552B02D0442B40F0FF804F4BFF
:10AFB80000221A70FAE023685869F5F73BFC4A4BFF
:10AFC800834693F800A09946BAF1450F02D14E4B3B
:10AFD80000221A705046FDF729FE00284DD04B4B31
:10AFE8005FFA8BFB1A7852450ED15846FFF790FC52
:10AFF800FF2804D15846FFF78BFCFF283DD0444B6F
:10B008001A7801321A7015E0DFF804A100228AF8D4
:10B01800002058460593FFF77BFCFF28059B04D0CA
:10B028009AF8002001328AF8002099F80020FF28B9
:10B038001A7022D02168374A4B6910601B5C8868F7
:10B0480047F289118842136092460FD1562B01D0DE
:10B05800542B0BD13B78123BDBB2022B06D82B7852
:10B0680030B2C01806F0A4FECAF800002B7830B23F
:10B07800C018DAF8001006F091FE99F80030552B48
:10B0880017D12368997C0F2913D92A7808398A425D
:10B09800144B01DA083200E000221A70144B9B7836
:10B0A80003F00203DBB20BB1FDF700FC184B0022E2
:10B0B8001A7099F80030442B3BD123689A7C0F2AE8
:10B0C80037D92978074B072926D90839197025E077
:10B0D800841D0020131E0020191E002004020020D9
:10B0E800631E00201E1E00204C1D00206E1E002026
:10B0F800741E0020F4010020835C0308945A03089E
:10B10800D65A0308F5010020641D0020661D0020A2
:10B11800921D00202C1E0020083A1A70964B9B782E
:10B1280003F00203DBB20BB1FDF7C0FB934B002227
:10B138001A7099F80030432B0CD1236830B25B6940
:10B1480019788F4B19602B78C01806F027FE8B4BA7
:10B1580000221A7099F80030232B13D122682B781B
:10B16800927C013A93420DDA864A01331370834B7D
:10B1780000221A70804B9B7803F00203DBB20BB1FC
:10B18800FDF794FB99F800302A2B0FD12B786BB17F
:10B198007C4A013B1370794B00221A70764B9B78DE
:10B1A80003F00203DBB20BB1FDF780FBFEF734FDC1
:10B1B800754A2B7811789246994288BF1370127895
:10B1C8000F32934202DD704A0F3B137023684FF031
:10B1D800000B93F81290B9F10F0F9ABFC9F120092B
:10B1E8005FFA89F94FF010099AF8000033B218187D
:10B1F8005844059306F0DCFD644A02F8090009F199
:10B2080001095FFA89F9B9F11F0F059B05D8216873
:10B218000BF1010B897C8B45E6DB98F8001011F0E7
:10B22800010F16D021685A48897C00780F2900F050
:10B23800800098BFC1F11001C0B294BFC9B200210B
:10B2480038B128789AF8006010305218801B5F21B6
:10B258001154226890684AF6EA0290420AD14D4B8E
:10B268001B78532B2FD106F0A3FD4B4B187006F01B
:10B2780099FE28E0B0F5E97F25D1464A1278532A8D
:10B2880021D11846FFF7CEFD0646E0B93B78DA0033
:10B29800D31A03F11200FFF7ADFD60B1FF2300934D
:10B2A8003E4B01961B7879200133029331460422E4
:10B2B800334606F0FBFD3B780021DA00D31A03F190
:10B2C8001200FFF7C3FD2C4EB37803F00203DBB284
:10B2D800002B6ED0FDF71CFB034680B9226849F2AB
:10B2E800340192688A420AD046F689718A4214BFAC
:10B2F80028783878F11D6522FDF728FB0FE02368D0
:10B30800B2799B682648B3F5E97F0CBF397829786C
:10B31800B38801FB0231B27909B206F05AFD2368FD
:10B328009A7C032A08D99A6848F6BC218A4203D035
:10B3380046F689718A4214D19B6848F6BC2293422A
:10B348000CD198F8003013F0010F01D010202CE038
:10B35800202107221348F5F71DF82AE0B3F5E97F05
:10B3680002D105200B2121E046F6897293421BD1B8
:10B37800002010211AE000BF741E0020921D00203A
:10B388002C1E00201E1E0020151E0020F401002087
:10B39800883A00204C1D0020681D0020131E002044
:10B3A8007B1E00200402002000200721104AFDF720
:10B3B80039FB23689A7C032A16D9B27802F0020274
:10B3C800D2B28AB19B6848F6BC2293420CD046F6AA
:10B3D8008972934208D0297806480131022207B0C1
:10B3E800BDE8F04FFDF78CBB07B0BDE8F08F00BF9C
:10B3F800741E0020F50100202DE9F04F794E8BB026
:10B4080033689D6893F81290122D01D00B2D09D145
:10B41800754A122D92F80090A9F130095FFA89F95E
:10B4280015D01DE04BF267739D4203D028339D422F
:10B4380040F053836D482821F5F72AF88046002804
:10B4480000F04E8301302821F5F722F848E39F7B6E
:10B4580037B9674BB846D879FEF7E8FB044615E0DC
:10B468000027B846FF20FEF7E1FB4BF258539D42F8
:10B4780004460BD14BF2376006F09AFCC0B2099033
:10B4880020B15B4B9B790BB1FDF7D8FB3368594D65
:10B498009A68122A1AD19B7BC3B12B7813F0010F3B
:10B4A80008D12046FFF7A6FC534B10B101221A70B1
:10B4B80000E018704E4B9B7943B12046FFF79AFC89
:10B4C80020B14D4B1B780BB1FDF7B8FB2978DFF89D
:10B4D80044A111F0010100F087819AF80030DFF8EB
:10B4E80038B118460793FDF7A1FB079B002800F029
:10B4F800B5804249002008704148424A90F800C08F
:10B5080013609C45404940F0898033689B8903F06B
:10B518000F03032B1ED13D4BACF1300C18784FF0C4
:10B528000A0E05903A480EFB0C00DDF814E000EB1B
:10B538000E0C0EF1010E5FFA8EFE70449CF8ADC041
:10B5480090F8AD00C2F800C083F800E0002872D17E
:10B55800187070E0082B2CD12C4BACF130001B7804
:10B5680000EB800C0CEB030E294BDFF8A0C013F89E
:10B578000E3008930BB98CF800309CF800E000EB13
:10B588008000059070440EF1010E5FFA8EFE8CF873
:10B5980000E01F4BDDF814C01B5C08900CEB0E009C
:10B5A800DFF86CE013601EF80030002B43D1174819
:10B5B80011E0072B11D1BCF1300F10D113480378DB
:10B5C80023B14FF02B0EC2F800E001E0C2F800C032
:10B5D800013303F0010303702DE0062B2BD10B7808
:10B5E800013327E0841D0020681D0020040200208C
:10B5F800221E0020631E00206B1300206F590020BC
:10B60800661D00202C1E00201E1E0020921D0020FA
:10B618005CB302084C1D0020691D0020DFF898E289
:10B6280003709BF800304FF0010C8EF800C013B186
:10B638000B7863440B7040238BF800300B784B4534
:10B6480003D39B4B09F1FF30187008781168201854
:10B6580006F0A4FB2B7843F004032B709AF8003013
:10B66800232B2FD1924B09F1FF311A788A4229DA1C
:10B6780072B932684BF2677192688A4208D02831F1
:10B688008A4205D02046079306F092FB079BC8B173
:10B6980018780130C0B21870201806F089FB28B954
:10B6A800834B20211878201806F078FB814B402224
:10B6B8001A702B78804A43F004032B7000238BF810
:10B6C800003013709AF800302A2B10D1784B1A7872
:10B6D8006AB1013A1A70774B40221A702B78764A71
:10B6E80043F004032B7000238BF8003013709AF892
:10B6F8000030432B1FD16E4B1878484505D22018CF
:10B708002021079306F04AFB079B9BF800203AB9D3
:10B718001B7809F1FF32934202DA654A013313704C
:10B728002B78644A43F004032B7000231370624A99
:10B738008BF8003013709BF8003013B15F4A013B5F
:10B7480013709BF80030012B0ED1594B1A784A45DB
:10B7580001D201321A70584A002313702A7842F035
:10B7680004022A708BF800302B7803F00402D2B25E
:10B77800002A71D0524A6FF38203137000211122FC
:10B788005048F4F707FE504A494B11781B78994204
:10B7980088BF137011780F318B4202DD4A490F3B85
:10B7A8000B70117847481022611806F012FB4548C3
:10B7B800F5F740F833684BF267719B68C2B28B4269
:10B7C80002D028318B4205D122B94048F5F732F82A
:10B7D800421CD2B20F2A3FD83A4820218018C2F121
:10B7E8001002F4F7D7FD37E0DFF8D8B01122584639
:10B7F800F4F7D0FD33684BF267729B68934202D02E
:10B808002832934209D1214604222E4806F0E1FA53
:10B8180040463946FFF7C6FA1EE021461022584630
:10B8280006F0D7FA5846F5F705F802462021C2F186
:10B8380010025844F4F7AEFD21464A46244806F063
:10B84800C8FA244A1020937882F8069043F002033D
:10B8580093700146FDF7E6F89AF80030532B75D13E
:10B8680033689A684BF258539A4208D1204606F03A
:10B878009FFA20B14BF23760012106F08FFA336846
:10B88800DFF838A09B68122B40D12046FFF7B2FAA8
:10B898008346002830D0104BFF2219780F4BF9B996
:10B8A800009201911B78782001330293FB3A1FE044
:10B8B8001E1E00206F590020921D0020691D0020C7
:10B8C800631E0020001E0020151E0020011E0020FF
:10B8D8009B1D0020941D00206B130020131E0020C8
:10B8E8000021009201911B787A20013302930422EF
:10B8F8000B4606F0DBFA09E08AF800007D4920468D
:10B90800FFF7A4FA7C4B83F800B0EFE020464946E5
:10B91800FDF7DEF8794B0020187033688AF80000CC
:10B928009B684AF6FE02934202D10090013005E07E
:10B938004BF27A52934206D1012300930146024604
:10B9480003460DF0C7FD6E48FDF75AF8FEF764F997
:10B958002B7813F0010F17D033684BF267729B688E
:10B96800934202D02832934204D140463946FFF729
:10B9780019FA09E05F4B634A03F1100153F8040B0D
:10B988008B4242F8040BF9D133689A68122A1ED107
:10B998009B7BE3B12046FFF72DFAC0B12B7813F05B
:10B9A800010F14D1584B9A7922B9DA79574B1B7881
:10B9B8009A420CD0564B1A780023303A05E0554984
:10B9C8002A20C91801330874DBB29342F7DB3268C6
:10B9D80093680B2B01D0122B0AD14A4B991D13F8EF
:10B9E800010B202802D10D3003F8010C8B42F6D14F
:10B9F80092684BF258539A4214D1434B9B798BB1BE
:10BA0800099878B14FF0000909EB040006F0D0F965
:10BA180018B1404B2A224B441A7409F10109B9F1B3
:10BA2800100FF1D12B7813F0010F25D03A4B1B786A
:10BA380003F08003DBB2FBB133689A684BF267739B
:10BA48009A422D4B03D04BF28F718A420CD11B784E
:10BA580033B9B8F1000F0FD05F3388F801300BE02D
:10BA680057B15F22FA5407E0244A1B781278103342
:10BA78009B1A284A5F21D154284CA37803F002036B
:10BA8800DBB2002B32D0FCF743FF2049034628B92C
:10BA980008786522E11DFCF759FF12E03068B4F917
:10BAA8000430A27984680978122C01FB023105D18F
:10BAB800807B18B91449C97902FB0131184806F08E
:10BAC80088F933689B68122B10D10820134A014665
:10BAD8000BB0BDE8F04FFCF7A5BF0027B84600E063
:10BAE800074609F1FF395FFA89F9BBE40BB0BDE8F5
:10BAF800F08F00BF001E00201E1E0020151E002013
:10BB0800941D002004020020221E0020131E002085
:10BB1800681D0020F4010020883A0020741E0020CF
:10BB28007B1E002024282DE9F041144626D16B4BBA
:10BB380043F63C321B686A4D9B686A4E934206D1B5
:10BB48002B7813F0010F0ED02438674909E04BF227
:10BB58008F7293420AD12B7813F0010F03D06349F7
:10BB68000020FCF7A7FF2978490800E02978301958
:10BB780001310222FCF7C4FF0234AAE0E72809D108
:10BB8800574B58481978801801310322FCF7B8FF41
:10BB980003349EE0A3282AD1514D2B783F2B15D88A
:10BBA80010465349FCF786FF5148F4F743FE2A2113
:10BBB80024184C48E4B2F4F76BFC002800F08A80A3
:10BBC800297802220131FCF79BFF83E05901494D96
:10BBD800C918691801F582411046DF31FCF76AFF80
:10BBE80005F59240FE30F4F725FE241871E0F2289E
:10BBF80021D13B4F3B4D3978072605EB0208B1FBB5
:10BC0800F6F1404601310222FCF77AFF39782D23FC
:10BC1800B1FBF6F688F80230F3009E1B8B1B364FFB
:10BC2800DBB207EB83031988E21CA9529B78A8189A
:10BC3800837006344DE025280BD1304B46F615624B
:10BC48009A8045229A719A78053842F002029A70D1
:10BC58003CE05E280BD1294B46F615729A804522A6
:10BC68009A719A783E3842F002029A702EE07C2847
:10BC78000BD1224B46F248129A8011229A719A7877
:10BC88005C3842F002029A7020E0EC280BD11B4B82
:10BC980046F659729A8045229A719A78CC3842F0C1
:10BCA80002029A7012E0A7280BD1144B46F679725B
:10BCB8009A8045229A719A78873842F002029A70DF
:10BCC80004E0E02801D1541C03E018B1054B1855D5
:10BCD8000134E4B22046BDE8F08100BF841D002095
:10BCE800131E0020F4010020E8540308A65403089A
:10BCF800625C030864120308DD3E0308741E00201A
:10BD080038B50A4B46F68A451B78002405FB03051F
:10BD180007E0074B22461978FFF704FF041B2D198B
:10BD28000446287808B11F2CF3D938BD671D0020B8
:10BD3800131E002070B5002543F62064204606F047
:10BD480037F8064604F1080006F032F816F0FF0F3F
:10BD580006D020F07F0010F0FF0F01D00135ADB202
:10BD680046F23F139C4201D00934E7E7284670BDEC
:10BD780070B5B0F900500E4605EBC50505F57855C8
:10BD88002835284606F014F8C3B213F0800F064C85
:10BD980008D03EB922882846013A03F07F01228064
:10BDA80005F0FCFF208870BD621D0020454B2DE981
:10BDB800F74F1B88444A044689461788DFF80C81E8
:10BDC80023B14FF0000A0AE09A4608E00529FBD1A2
:10BDD80098F8003043F0040388F8003070E098F8D1
:10BDE800003013F0030F0BD013F0010F02D0B4F1A1
:10BDF800FF3F05D103F00203DBB21BB1012C01D0D8
:10BE08003F19BFB23BB2B3F1FF3F04D0B3F57A7F1D
:10BE180008BF002701E040F2E7370FFA87FB0BEB7A
:10BE2800CB0303F5785303F12000019305F0C0FF1D
:10BE380010F0FF0F019B16D0B9F1050F09D103F1DE
:10BE4800280005F0B5FF20F07F0010F0FF0FC6D0E6
:10BE580022E0B9F1000F1FD003F1280005F0A8FF78
:10BE680000F07F0618E00AF1010AB4F1FF3F1FFA5B
:10BE78008AFA04D198F8003043F0010305E0012C58
:10BE880005D198F8003043F0020388F80030BAF57D
:10BE98007A7F0DD03D46A2E74E4505D0B9F1000F97
:10BEA80002D0B9F1050F9AD1BAF1000F05D000E020
:10BEB8003D46054A2DB2156002E0034BC3F800B0B9
:10BEC800BDE8FE8F621D00202C1E0020301E0020C1
:10BED8002DE9F041037890465A1ED2B2792A9AB0D9
:10BEE8000F4600F2CA805E01654AF3189B18654A3E
:10BEF80046F68A461278457806FB0236E721304630
:10BF0800F4F7C6FA0446F0B930467C21F4F7C0FAD3
:10BF18000446C0B930462521F4F7BAFA044690B968
:10BF280030462421F4F7B4FA044660B9304640217B
:10BF3800F4F7AEFA044630B93046F921F4F7A8FA16
:10BF48000446002878D0A41B0FB14F4800E04046B3
:10BF580031462246A619F4F7F3FC3046E721F4F7F8
:10BF680097FA30B128466946652246F65973FCF7B8
:10BF7800EDFC30467C21F4F78BFA50B1691EC9B24A
:10BF880001EB011101F5C24168464831112205F063
:10BF980020FF30462521F4F77BFA38B1681EC0B27D
:10BFA8006946652246F61563FCF7D0FC3046F92150
:10BFB800F4F76EFA38B1681EC0B26946652246F6D3
:10BFC8001573FCF7C3FC30464021F4F761FA50B111
:10BFD800691EC9B201EB011101F5EA416846BB319E
:10BFE800112205F0F6FE30462421F4F751FA58B133
:10BFF80017B12548201801E008EB04002946022261
:10C00800FCF77EFD02340CE017B11F48201801E050
:10C0180008EB04006946F4F7AFFB6846F4F70AFC3E
:10C028000419002F29D0194A9378141943F00203F0
:10C0380093700023E37116E03046F4F7FBFB0546E6
:10C048001FB9404631462A4615E0102810DD2A4619
:10C058000D483146F4F774FC0C4A9378551943F0AF
:10C0680002039370EC7110200146FCF7DBFC04E03E
:10C07800074831461022F4F763FC1AB0BDE8F08196
:10C0880047440308671D00207B1E0020741E002003
:10C09800040200200C4B1A7812F0010302D0002091
:10C0A8000A4905E002F00200C0B218B10849184672
:10C0B800FCF700BD02F00402D2B20AB10549F7E765
:10C0C80005480121FFF704BF301E0020201A03088D
:10C0D800FF190308411A0308651E002070B5124DA8
:10C0E800124C00201249FCF7F5FB2846A1780222E1
:10C0F800FCF706FDE81CE1780222FCF701FD05F1DA
:10C10800080021790222FCF7FBFC05F10B0061799C
:10C118000222FCF7F5FCA17905F10E000222BDE828
:10C128007040FCF7EDBC00BFF4010020651E002044
:10C138006DB402082DE9F341544F554C3B689D7C82
:10C14800237813F0010F33D1022243F61E610DF15B
:10C15800060005F03EFE4F4EBDF806304FF0FF30AA
:10C1680033602946FFF722FE237843F0010323704A
:10C17800494B1B7813F0030F18D1B6F90010474844
:10C1880001EBC10101F578512031092205F021FEAA
:10C19800434B1B883BB1434B30461978C1F34001F0
:10C1A800FFF7E6FD10B90020FAF77EF8FFF796FFD3
:10C1B8003D4E3378552B0DD1DFF8DC803B48FCF73A
:10C1C8001FFC98F800304FF0FF306FF3410388F8F8
:10C1D80000300DE0442B2FD1DFF8BC803348FCF74A
:10C1E8000FFC98F8003001206FF3000388F8003046
:10C1F8002946FFF7DBFD98F8003013F0030F19D13B
:10C20800244D2648B5F90010092201EBC10101F5BA
:10C218007851203105F0DDFD214B1B883BB1214BC6
:10C2280028461978C1F34001FFF7A2FD10B9002094
:10C23800FAF73AF8FFF752FFFFF72CFF3378232B72
:10C2480022D1154B194E1A7802F0FC026FF38202C4
:10C258001A70FCF7F3FCB3786FF34103B370144B17
:10C268001D7835B9FCF722FB3046FCF7C9FB3D6069
:10C278000AE02278013DEDB242F0060222701D70FC
:10C288000C4B53F825303B60BDE8FC81841D002031
:10C29800631E00202C1E0020301E0020651E00207A
:10C2A800621D0020B36400204C1D0020741E002075
:10C2B800431E0020501E00202DE9F0411646104A6A
:10C2C8000F4653780E21C3F342034B43117803F50D
:10C2D8000A434C330B4D01F00701044603EB4101BF
:10C2E800022205F076FDE81921780222FCF708FC05
:10C2F8006178A8190222BDE8F041FCF701BC00BF33
:10C30800191E0020F4010020044B02225978044B26
:10C31800C1F3420118180131FCF7F2BB191E0020C5
:10C32800F401002010B5074B074C1B78074A03F0AF
:10C33800070304EB83031C88111814529B788B7035
:10C3480010BD00BF191E0020DD3E0308F4010020C7
:10C35800084B1B789B0902D0012B06D102E0102064
:10C36800054904E01020054901E005491020FCF7C3
:10C37800A1BB00BF191E0020C2260308E32603083C
:10C38800042703082DE9F041DFF868800F4698F884
:10C398000010174DC1F382010446164605F1080046
:10C3A80001310222FCF7ACFB98F80010042201F0DE
:10C3B8001C0101F51E413431204605F00AFDE8193B
:10C3C80021780222FCF79CFBF81C281861780222CD
:10C3D800FCF796FBA819A1780222FCF791FBF01C48
:10C3E800E17828180222BDE8F041FCF789BB00BFBC
:10C3F800F4010020651D0020064B1B7803F0800324
:10C40800DBB233B1435C04482021C0180222F3F7A1
:10C41800C1BF7047883A0020F40100202DE9F74396
:10C42800654D664C2B6821789B68022203EB41011D
:10C438000DF1060005F0CDFC2B68A9469A6843F675
:10C44800F4239A4208D100205D49FCF733FBBDF87C
:10C4580006804FF4B46303E0BDF806804FF46163CF
:10C46800B8FBF3F103FB11883C221FFA88F8B8FBEC
:10C47800F2F302FB1388CFB2DEB2022251483946EA
:10C48800FCF73EFB5FFA88F802224F483146FCF77A
:10C4980037FB02224D484146FCF732FB4C4B1B78D8
:10C4A80013F0010F6ED04B4B4B4D1878232804D155
:10C4B8002B78012B62D8013305E02A2805D12B7887
:10C4C800002B5BD0013B2B7058E0A0F13003DBB2AE
:10C4D800092B01D943284BD12B7873B9D9F80030EF
:10C4E80039B29A6843F6F4239A4201D10A2200E04D
:10C4F8001122FDF7B1FBC7B216E0012B0ED1D9F816
:10C50800003031B29A6843F6F4239A4201D11722D7
:10C5180000E03B22FDF7A0FBC6B205E041463B2206
:10C52800FDF79AFB5FFA80F8D9F800309A6843F66D
:10C53800F4239A4209D13C235E434FF4B46303FBCE
:10C548000767B844ADF8068006E0384631464246EB
:10C5580010F067FAADF80600D9F8003020789B682B
:10C568000DF1060103EB4000022205F02CFC05E06A
:10C57800532803D100232B70FDF74EFB1748297869
:10C58800FFF73AFFD9F800309A6843F6F4239A4245
:10C5980010D02078124965220023FCF7D7F905202E
:10C5A8000B21104AFCF73EFA21780F48013102228C
:10C5B800FCF7A6FABDE8FE83841D0020131E0020A8
:10C5C800E7580308040200200A0200201202002093
:10C5D800631E00204C1D00201E1E00207EB4020891
:10C5E8007B1E0020741E0020F501002073B59A4BB5
:10C5F8009A4D1A7812F0010F05D12A7812F03802F4
:10C6080004BF2A706A701A78934E42F001021A70B9
:10C618002B78924C13F038023ED19149097855296C
:10C6280004D113F0070F2FD0DA1D0AE044290CD1EA
:10C6380003F0070201323D3992FBF1F1C800411ABB
:10C64800521A62F3020323701EE053290AD1C3F37E
:10C65800C201013161F3C5032370637862F34303B8
:10C66800637011E023290FD1FCF7E8FA33787D4A8B
:10C6780043F0060333701378013BDBB213707A4A38
:10C6880052F82320794B1A6000207949FCF712FAF6
:10C698001C20FFF747FEDDE0082A2ED1754900204F
:10C6A800FCF708FA0620FFF72FFE0C20FFF73AFEEA
:10C6B8001521182201A8FFF7FFFD694B1B78552BA0
:10C6C80006D1637803F0FE03C3F34202013A07E0A0
:10C6D800442B0BD1637803F0FE03C3F3420201320B
:10C6E80002F0030262F343036370B3E0532B28D0D4
:10C6F800232B40F0AF802378A6E0102A51D15D4962
:10C708000020FCF7D7F90620FFF7FEFD0C20FFF705
:10C7180009FE1521182201A8FFF7CEFD61785648B9
:10C7280001F00101FFF768FE4D4B1878232801D06E
:10C738002A2804D16378DA4362F30003D4E7532844
:10C7480004D12378C3F3C202013280E0A0F13003A0
:10C75800DBB2092B01D943287CD16B7802AA03F0FC
:10C7680001033B21D41883F001024B43172606FB33
:10C77800023214F8041CFDF76FFA04F8040C6B7805
:10C788000E22C3F342035343287803F50A434C337C
:10C7980000F0070003EB400001A90C3A05F013FB79
:10C7A80058E0182A4DD133490020FCF783F90620B8
:10C7B800FFF7AAFD0C20FFF7B5FDFFF7C9FD284BD1
:10C7C8001B78552B07D1237813F0C00F42D0C3F341
:10C7D8008112013A06E0442B07D123789A09012AED
:10C7E80038DC013262F3871333E0232B04D123783A
:10C7F800C3F3C202023A2AE0532B2BD1FCF71EFAEC
:10C8080033781E4A43F006033370164B16481978DE
:10C8180040F82120013119702378C3F3C201013196
:10C8280061F3C503C3F381112370104B11B10129C2
:10C8380004D101E01C3202E0114A00E0114A1A60FA
:10C8480008E0114A00211170C3F3C202013A62F3F1
:10C85800C50323707CBD00BF631E0020191E002085
:10C868004C1D0020431E0020501E0020841D002067
:10C8780080260308A126030881B4020884B40208AC
:10C88800BCB40208D8B402081E1E002073B5494B78
:10C89800494D1A7812F0010F04D12A7812F00302D8
:10C8A80008BF2A701A78434E42F001021A702B789A
:10C8B800414C13F003022ED1404A1278552A03D175
:10C8C800C3F38202013A04E0442A06D1C3F3820288
:10C8D800013262F38403237017E0532A03D15A1CF0
:10C8E80062F30103F7E7232A0FD1FCF7A7F933789E
:10C8F800334A43F0060333701378013BDBB21370FD
:10C90800304A52F82320304B1A6001A810211B220C
:10C91800FFF738FD4CE0012A4AD101A810211A324C
:10C92800FFF730FD254B1878232804D12378C3F36B
:10C938004112013205E02A2807D12378C3F34112B6
:10C94800013A62F3461323702CE0532804D123786C
:10C95800DA1C62F30103F6E7A0F13003DBB2092B1E
:10C9680001D943281ED12B7802AAC3F34113D41846
:10C978000C215A1C03F001034B4302F001021F264D
:10C9880014F8041C06FB0232FDF766F904F8040CDF
:10C99800287801A900F01C0000F51E40343004225C
:10C9A80005F011FA29780948C1F34111FFF724FD70
:10C9B8007CBD00BF631E0020651D00204C1D0020AB
:10C9C800431E0020501E0020841D0020F4B40208DD
:10C9D800064B1B7803F08003DBB233B1435C044899
:10C9E8002021C0180322F3F7D5BC7047883A0020ED
:10C9F800F40100204328F8B504460D46174606D131
:10CA0800104B00261A786FF3C3021A7000E00E4626
:10CA18002046FCF70BF990B10A4B303C1A780A26ED
:10CA280002F00801C9B2002918BF002506FB054617
:10CA38006FF3C30236B21A70BE42A8BF3E4630B288
:10CA4800F8BD00BF631E00202DE9F3416E4F6F4E05
:10CA58003B7843F001033B70347844B94BF2AF5054
:10CA680005F0A6F96A4B6B491860204617E0012CBF
:10CA780002D10020684912E0022C02D10020674947
:10CA88000DE0032C02D10020654908E0042C02D1F6
:10CA98000020644903E0052C03D163490020FCF71A
:10CAA80009F83178D9B9614B1B78312B01D10131A3
:10CAB80001E0302B05D1564B4BF2AF50196005F011
:10CAC8006DF95B4B1A785B4B02F08002D2B20AB167
:10CAD800202202E04E4A12683032DA776EE00129ED
:10CAE8000BD002290CD003290DD004290ED04BF20B
:10CAF800AB55052918BF00250AE04BF29B5507E006
:10CB08004BF29F5504E04BF2A35501E04BF2A755B9
:10CB18002946042201A805F05CF9474B474A03F16E
:10CB2800100153F8040B8B4242F8040BF9D103228D
:10CB380043489DF80410FBF7E3FF032241489DF8A2
:10CB48000510FBF7DDFF03223F489DF80610FBF7B1
:10CB5800D7FF3E4803229DF80710FBF7D1FF334B60
:10CB68003B4C1878232804D12378022B22D8013390
:10CB780004E02A2804D12378E3B1013B237019E0AB
:10CB8800A0F13003DBB2092B01D9432812D194F864
:10CB9800008002AA904418F8041CFF22FFF72AFF1D
:10CBA80008F8040C207802AA131813F8041C281893
:10CBB80005F0F4F827482178FFF70AFF1B4B1B788C
:10CBC800532B1FD1224B00221A7033780133DBB26A
:10CBD800062B337004D0012B14D10D4B1B688BB17D
:10CBE800FDF71AF8002333703B781B4A43F006031D
:10CBF8003B701378013BDBB21370184A52F82320BC
:10CC0800174B1A60BDE8FC81631E0020131E00202C
:10CC18002C1E00206D72030896730308B77303086F
:10CC2800D8730308F97303081A7403084C1D00200D
:10CC3800883A0020F4010020CCA103080402002057
:10CC480005020020090200200D0200201102002028
:10CC58001E1E0020F8B40208431E0020501E0020AB
:10CC6800841D002070B5174C0D460646002120464D
:10CC78004FF4C172F3F78EFBFF2D0AD1B10001F515
:10CC8800DC4120461531042205F0A3F823789BB92E
:10CC980070BDFE2D01D1173E02E0FD2D02D10136F7
:10CCA800267009E0B60006F5DC401530401905F09D
:10CCB8007FF8C0B2207020B10248BDE8704019F07A
:10CCC80085B970BD882000202DE9F04119F0B0F930
:10CCD80060B110208F49FBF7EDFE8F4B1B78432B7B
:10CCE80040F0EE81BDE8F04119F0C4B919F0B2F98D
:10CCF800002826D0894C23786BB110208849FBF78F
:10CD0800D9FE88482D211030F3F7C2FB002800F027
:10CD1800D781217810E010208349FBF7CBFE8148AA
:10CD28002D211030F3F7B4FB0446002800F0C88129
:10CD380019F0A8F9014620468222BDE8F041FBF728
:10CD4800DFBE7A4C43F6CC2223689B68934250D0CE
:10CD5800774E744D307803EB800005F029F80322F4
:10CD680001467448FBF7CCFE2368986846F6797349
:10CD780098422BD0203B984228D03378013000EBE2
:10CD8800830005F015F80322014605F11500FBF7AD
:10CD9800B7FE236830789B68023303EB800005F008
:10CDA80007F80322014605F11900FBF7A9FE2368DD
:10CDB80030789B68033303EB800004F0F9FF03220B
:10CDC800014605F11D00FBF79BFE0EE02D21032215
:10CDD8005948F3F7DFFA2D2103225848F3F7DAFA16
:10CDE80057482D210322F3F7D5FA20232B772B76EA
:10CDF8002B75544B1B7813F0010F00F0BD8023688E
:10CE080043F6CC229B68444D934261D04E4E484F26
:10CE180032783878D31803EB800004F0C9FF4B4B05
:10CE28000146186028789846A0F13002D2B2092A43
:10CE380001D943280FD109B2BA22FCF70DFF2368A4
:10CE480032789B680146C8F800003878D31803EB9D
:10CE5800800004F0A3FF2B782A2B04D1337813B178
:10CE6800394A013B13702B78232B0ED13378022BD0
:10CE78000BD8226846F6597192688A4205D020314B
:10CE88008A4202D0304A013313702B78552B01D0D7
:10CE9800442B0FD1236831789B68A3F5DC43B3F1A9
:10CEA800150248BFA3F112023B7803EBA202D0B2ED
:10CEB800FFF7D8FE264B1B7803F08003DBB23BB1AB
:10CEC8003278184B03EB820320225A749A74DA746E
:10CED8002B78532B06D023689A6843F6CC239A42C2
:10CEE80040F0EE80FBF7AAFE236846F615629B68C1
:10CEF800934203D10E4B0220197806E046F6797268
:10CF0800934227D10A4B002019780131BDE8F0413E
:10CF18000CF0B4BA9C5B03084C1D0020E0150020FF
:10CF2800735A0308F4010020BD5B0308841D002028
:10CF3800131E002005020020090200200D02002017
:10CF480011020020631E00201E1E00202C1E00203F
:10CF5800883A002046F65972934204D1594B012071
:10CF680019780918D2E746F61572934240F0A8805E
:10CF7800544B03201978C8E723684AF6FE029B68D9
:10CF880093423ED14F4E10204F49FBF793FD317825
:10CF98004E4D01EB011101F52841FE3110222846C2
:10CFA80004F017FF2B4605F110012A461078474F69
:10CFB80078B94749FBF77EFD3846E721F3F768FA69
:10CFC80078B13178401B381801310322FBF798FDFE
:10CFD80007E013F8010B10B9203003F8010C8B425D
:10CFE800E4D13C4D2B782A2B03D13078FD21FFF773
:10CFF80039FE2B78432B63D1307823680130C0B2D7
:10D0080059E043F6CC229342324E1AD010203249CE
:10D01800FBF750FD33782A2B52D1304B1B689B68A5
:10D02800A3F5DC43B3F1150248BFA3F11202254B67
:10D03800FF211B7803EBA202D0B2BDE8F041FFF755
:10D0480011BE33781F4D552B04D12B78142B01D1E9
:10D05800033B2B703378442B05D12B78122B02D14C
:10D06800184B15221A702B78DFF874805901C918EB
:10D07800414401F5944100201F31FBF71BFD08F5E1
:10D088009241102017312F78FBF714FD3378112FB8
:10D098008CBF032700272A2B05D12878FE21C01B27
:10D0A800C0B2FFF7DFFD3378432B09D12B78173B4C
:10D0B800DF1B2368F8B2997CBDE8F04118F0A0BFE7
:10D0C800BDE8F081131E00207B5B0308F4010020FB
:10D0D8008B3C03084C1D0020395B0308841D00208D
:10D0E8006412030810B50E4B1B78452B17D10D4B56
:10D0F8001A7842F006021A700B4A1378032B0ED8DE
:10D108000A490B4C086844F82300013313708368FC
:10D118000B60FBF7D7FBBDE81040FBF78FBD10BDD8
:10D128004C1D0020631E0020431E0020841D00208B
:10D13800501E002010B50C4B04462146D8790FF03C
:10D1480034FC60B1204655210FF08EFA48B12046D4
:10D158000FF020FBD0F1010038BF002010BD0220E5
:10D1680010BD022010BD00BF221E002008B50FF020
:10D178000BFCC0B208BD00002DE9F047634B644CBE
:10D188001A78994612F0010F624D65D02078FFF7A2
:10D19800D1FF614A2B181178604F93F8A031604E87
:10D1A80044293870336090460AD12D2B08D038B9FD
:10D1B80095F8A11101233B7031602078FFF7D6FF65
:10D1C80098F80030552B10D133682D2B0DD03B78B3
:10D1D8005BB1013B514ADBB21370EB1893F8A01115
:10D1E8004F4B20781960FFF7C1FF98F80030232BC8
:10D1F80019D14C4B20781B689B7C013B984212DA72
:10D20800434B0130C0B21870FFF794FF38702818EC
:10D2180090F8A0313360444B9B7803F00203DBB2F3
:10D228000BB1FBF743FB98F800302A2B14D1207878
:10D2380090B1374B0138C0B21870FFF77BFF3870D8
:10D24800281890F8A0313360374B9B7803F002031D
:10D25800DBB20BB1FBF72AFB344EFCF7DDFC23787D
:10D2680032789A4288BF337032780F32934202DDA7
:10D278002E4A0F3B1370DFF8C48000273078381827
:10D28800C0B2FFF757FF281890F8A0310137102FC8
:10D2980008F8013F07D0254B1A78224BBA181B68AB
:10D2A8009B7C9A42EADB99F8003013F0010F13D007
:10D2B8001F4B1A781F4B02F08002D2B22AB1227893
:10D2C80031781032521A5F2105E022783178103215
:10D2D800521A134909689954134DAB7803F00203A5
:10D2E800DBB25BB12078E91D652246F61573FBF7C2
:10D2F8002DFB05200B212A46FBF794FB21780E48CD
:10D3080001310222BDE8F047FBF7FABB631E00209B
:10D318001E1E00205CB302084C1D0020641D002066
:10D328002C1E0020841D0020741E0020151E0020C5
:10D33800883A0020F4010020F501002003020020B3
:10D348002DE9F041002480460D4616462346012764
:10D3580017FA04F298F80010E0B2914206D146F6A6
:10D36800597329463246FBF7F1FA3B460134042C3F
:10D37800EDD1043C0A4AE0B2A218917898F800204E
:10D388008A4207D132B146F6797329463246FBF70D
:10D39800DDFA01230134042CECD11846BDE8F081F4
:10D3A800221E00202DE9F041074610460D4614467E
:10D3B800F3F740FAC3B28046B3B1AB4214D80B4E70
:10D3C80020212A46F019F2F7E5FF2046F3F732FA52
:10D3D800C8EB05056D08EDB2EF1902462146F019B4
:10D3E800BDE8F041F2F72EBFBDE8F081F40100205E
:10D3F800312200230178194111F0010F02D00449AC
:10D40800C9188A7501330132042BD2B2F2D17047A0
:10D41800F40100202DE9F04F87B09DF84040814687
:10D42800072C0D4605929A4637D1073C27462B789C
:10D43800234113F0010F2CD0012623B24FF000082E
:10D44800029351203146324633460096CDF8048087
:10D4580004F02CFD1B204146A2194346CDF800805C
:10D46800F5F74EF937B9112039463A463346009751
:10D47800F5F746F9534B204613F8242001276FF39C
:10D48800000203F824201199F5F7FEFF2046F6F76D
:10D49800FFF90134042CCAD10DE2012C03780CD118
:10D4A8000BB90B7823B3FF2300930021464B01915E
:10D4B8001B780C200133029316E0022C09D10BB91A
:10D4C8000B78ABB10021FF23009301910291342026
:10D4D8000AE0062C0CD10BB90B784BB10021FF23C5
:10D4E800009301910291652004220B4604F0DEFCB2
:10D4F800BAF1010F99F800302BD13BB1334B002022
:10D50800D979024653460090F5F7FAF82B783BB1E3
:10D518002E4B0120D979002203460092F5F7F0F846
:10D528000020F5F767FF99F80030002B5BD0284BF7
:10D538001978002957D1274B5B78002B53D0FF234C
:10D5480000933A2001220B460191029104F0AEFCAF
:10D5580049E063B1052C4FF0000102D100910F2082
:10D5680001E000910B200A460123F5F7C9F82B7852
:10D5780083B1052C4FF0000106D110200A46012383
:10D588000091F5F7BDF812E00C200A46012300913E
:10D59800F5F7B6F8022C25D0032C01D10E4B02E08A
:10D5A800042C02D10D4B1F781DE0052C01D10C4B2A
:10D5B800F9E7012C01D1044BF5E7062C0CBFFF2736
:10D5C800002710E0291A0020F61A0020221E002049
:10D5D800141A00206B1300203C200020475800201C
:10D5E800CF3C0020FF2799F80030002B00F0B580D1
:10D5F800934B944E1A78984602F02002D2B262B148
:10D60800317811F0010108D1FF230093282001226D
:10D618000B460191029104F049FC98F8003003F0A0
:10D628001003DBB26BB1317801F00201C9B241B924
:10D63800FF230093292001220B460191029104F057
:10D6480035FC98F8033013F0010F0DD0317801F054
:10D658000401C9B241B9FF2300932A2001220B46D5
:10D668000191029104F022FC98F8033003F00203C0
:10D67800DBB26BB1317801F00801C9B241B9FF23BF
:10D6880000932B2001220B460191029104F00EFC1D
:10D6980098F8033003F00403DBB26BB1317801F082
:10D6A8001001C9B241B9FF2300932C2001220B4677
:10D6B8000191029104F0FAFB98F8033003F0080393
:10D6C800DBB26BB1317801F02001C9B241B9FF2357
:10D6D80000932D2001220B460191029104F0E6FBF4
:10D6E80011F04CFF68B1317801F04001C9B241B97D
:10D6F800FF230093492001220B460191029104F077
:10D70800D5FB98F8033003F04003DBB26BB13178F6
:10D7180001F08001C9B241B9FF2300934E200122D4
:10D728000B460191029104F0C1FB767816F00106D0
:10D7380013D14548314617F09AFE58B1FF2300939C
:10D74800731C00211BB20293752001220B46019124
:10D7580004F0ACFB0136702EEBD1119B3B4A1978D3
:10D768003B4B51B199F8001011702A781A702B7838
:10D778000BB1542005E0522003E011702A785320A1
:10D788001A7004F065FF119B00261A78314B1A7045
:10D7980099F80030334113F0010F2DD03146059828
:10D7A80017F065FE0122014628B933B201900092B4
:10D7B8000293104605E0002133B2009201910293D2
:10D7C80024200B4604F072FBBAF1010F05D1224B5D
:10D7D8008020DA790521013208E0022C07F10102E4
:10D7E80002D18020072101E0802006213346F6F788
:10D7F800AFFB3046F6F720F82B78334113F0010FD2
:10D8080055D000214FF0010B33B2029302205A4643
:10D818000B46CDF800B0019104F048FBDA45DFF87B
:10D828003C801DD118F8263013EA0B0332D10A4A7E
:10D838000520D1790093594406EB0B0228E000BF7C
:10D84800883A0020E81B0020041A0020611A0020F2
:10D85800621A0020061C0020221E0020291A00201F
:10D8680018F8263013F0010314D1022C0CD1134BF5
:10D878001B7803F02403042B04BF114B83F800B07A
:10D8880000230093072001E000930620791C721CF6
:10D89800F4F736FF11993046F5F7F6FD3046F5F7FF
:10D8A800F7FF18F826306FF3000308F82630013622
:10D8B800042E7FF46DAF07B0BDE8F08F101C002078
:10D8C800641300202DE9F04180460E46174646F6BF
:10D8D8003F1500243846214617F0C9FD88B129466E
:10D8E80008220B4804F075FA0948414617F06CFD08
:10D8F800074817F08FFD20B90123A340327813435E
:10D90800337001340835042CE4D1BDE8F08100BF40
:10D91800FE1B00202DE9F04387B08046894604A805
:10D9280047F26931082204F054FA0024404621469F
:10D93800E7B217F09CFD002843D03846F4F718FCEE
:10D948000025661C0246314611202B460095F4F747
:10D95800D7FE012321462A460420FF080095F4F744
:10D96800CFFE4BF25F70381804F022FA04F0070378
:10D97800C1B2194111F001014FF002024FF0010349
:10D988000AD00092019336B27720294692182B4686
:10D99800029604F08BFA14E00092019336B2232029
:10D9A80004220B46029604F081FAB9F1000F08D060
:10D9B80004A8214617F05BFD18B10548214617F069
:10D9C80040FD0134402CB1D107B0BDE8F08300BF61
:10D9D8003E1A00202DE9F74F9846137805460C4665
:10D9E80017469DF830909DF834B09DF83800DFF860
:10D9F800C8A073B12A4A51786FF3820151703B78FD
:10DA080000EA03033B7021789AF800208A18D31A99
:10DA18002B70237883B123482146F5F7E5FE224988
:10DA2800204817F0D1FC1F480121FFF773FF1D485C
:10DA380041462246FFF746FF1C4B00261E702978F8
:10DA480043F6FB2004F0AAF9494646F64D0004F0D7
:10DA5800A5F9204639464A46F5F782FC144B42465A
:10DA68009E7039464B462046CDF800B00195FFF729
:10DA7800D1FC2846F8F750FC2B780E480E498AF856
:10DA88000030F5F7B1FE12F0C7FD88F800603E706F
:10DA980026702E7003B0BDE8F04F04F0E3BC00BF61
:10DAA800CB3C0020071C0020591A0020601E0020D3
:10DAB8006B130020EA1B0020141A002010B50B4B32
:10DAC8000B4C024603CB206061600A48114617F0F0
:10DAD8009CFC2146074817F077FC064817F09AFC8B
:10DAE800D0F1010038BF002010BD00BF402E00203B
:10DAF800F41B0020FE1B002010B50A4C637C4BB1C0
:10DB080000200949FAF7D6FF084B1B78432B01D1AF
:10DB1800433B6374607C20B90549BDE81040FAF7BF
:10DB2800C9BF10BD4E1D0020CD3C03084C1D002070
:10DB3800AC3C0308034B1A7801321A7001230370B6
:10DB4800704700BF601E002010B50C48FAF758FF58
:10DB58000B4A002414700B4A0B4B14700B4ADC70F0
:10DB680014700B4A9C7014700A4A1C7114700A4A8B
:10DB78001470FBF763F8094B1C6010BD741E00207D
:10DB8800221E00204D1D00206B130020641E002063
:10DB9800711E0020881D0020601E0020841D0020AA
:10DBA8002DE9F04F984B994E93F800903368DFF8C1
:10DBB800AC829C7C964BF0221A7098F800308BB09F
:10DBC8000D2B354647463FD1924B93F803C0BCF125
:10DBD800010F04D9ED3A5A7100208F492FE01AD16C
:10DBE8000024DC708D4A8E4B8E498F488F4D04700F
:10DBF8001C7014700C70CDF800C001942D7802953B
:10DC0800FFF7E8FEFBF71AF8894834600BB0BDE867
:10DC1800F04FFAF7F5BE87488249F5F7E5FD864BE0
:10DC2800864A03CB864B10601B785160532B5FD11B
:10DC380098F800308349013388F8003000200BB091
:10DC4800BDE8F04FFAF736BF092B0FD17C4B1B7894
:10DC5800532B3DD17C4B00221A700D2388F80030DD
:10DC68007A4B1A7842F006021A7089E20E2B37D1E5
:10DC7800734B1B78532B2BD175496E4817F0A4FBB7
:10DC88006C48FFF71BFF044640B198F800300522A6
:10DC9800013B88F800305F4BDA7071E2082246F6E3
:10DCA8004E01664804F095F864496A4817F0ADFBE0
:10DCB800012300935D4B01941B785B4802935949FB
:10DCC800564A574BFFF786FEFAF7B8FF346057E21B
:10DCD800232B40F055820BB0BDE8F04FFFF734BF5F
:10DCE80033B95D4B1A781AB901321A7012F094FCE4
:10DCF800631E48BFA31DDB10013303FB09F91FFA9C
:10DD080089F909F5D046A9F59049A9F1A1094F4B20
:10DD1800CDF81C901A784E3612F0010F4A4C00F0DC
:10DD28002081474B1A789946432A40F0C9803B78AE
:10DD38000D2B40F0C5803F48217817F098FB00284C
:10DD480000F0BE803D48217817F091FB002840F094
:10DD5800B780079920780FFA81FB0BEBD00004F00D
:10DD680027F823784FF0010A03F007020AFA02FAAB
:10DD7800DFF8EC805FFA8AFA10EA0A0FC8F80000A8
:10DD880027D0244B5B78002B40F09A80274BD8791A
:10DD9800F8F720FA002800F09380D8F80010CAF1AC
:10DDA800FF0A20780AEA0101C8F800100BEBD0003E
:10DDB80003F0F4FF20780FFA86FB0BEBD00003F09A
:10DDC800F7FF00EA0A012078C8F800100BEBD00032
:10DDD80061E032B202EBD300059203F0E9FF10EAEA
:10DDE8000A0FC8F800003DD140EA0A01059B2078D7
:10DDF800C8F8001003EBD00003F0D0FF21781548D5
:10DE080017F01FFB5CE000BF131E0020841D0020DC
:10DE18006F1E00206B130020723D0308641E002053
:10DE28004D1D0020711E0020881D0020221E00208C
:10DE3800741E0020071C0020402E0020FC19002022
:10DE48004C1D0020383E03081E1E0020631E0020C3
:10DE58004E1A0020591A0020B0140020601E00201D
:10DE68002C1E0020924B5B7823B9924BD879F8F797
:10DE7800B1F9B8B92078DDF814C0CAF1FF0A0CEB83
:10DE8800D00003F095FF8C4A00EA0A01059B207830
:10DE9800116003EBD00003F081FF2178874817F069
:10DEA800DBFA0DE020780BEBD00003F081FF40EAAD
:10DEB8000A012078C8F800100BEBD00003F06EFFC1
:10DEC80099F80030232B10D12A682378927C013AE4
:10DED80093420ADA7A4A013313707A4B9B7803F03B
:10DEE8000203DBB20BB1FAF7E1FC99F800302A2BF8
:10DEF8000CD1237853B1724A013B1370714B9B7854
:10DF080003F00203DBB20BB1FAF7D0FC99F800304A
:10DF1800552B12D129682278897C694B08398A42A5
:10DF280001DA083200E000221A70664B9B7803F091
:10DF38000203DBB20BB1FAF7B9FC99F80030442BB5
:10DF48000FD122785E4B072A9CBF2A68927C083A38
:10DF58001A705C4B9B7803F00203DBB20BB1FAF743
:10DF6800A5FCFBF759FE584A237811789246994246
:10DF780088BF137012780F32934202DD524A0F3B6A
:10DF880013702B684FF0000B93F81280CDF818B07F
:10DF9800B8F10F0F9ABFC8F120085FFA88F84FF060
:10DFA800100839784FFA8BF30D2905D19AF800201B
:10DFB8009B18DB10454A04E09AF800209B18444A55
:10DFC800DB10D35C9AF8002005934FFA8BF39A186C
:10DFD8000D2902F007094FEAE20202D13D49895CA6
:10DFE8000691DDF81CC004930FFA8CF0101803F0AA
:10DFF800DFFEC0B2049B08909AF8000032B21818ED
:10E0080002EBE00003F0D4FE39789AF80020049B74
:10E01800C0B209919A1846E0059BDDF824C043FA7E
:10E0280009F12D4B01F0010100290CBFA521DB21CD
:10E03800BCF10D0F03F8081014D128494FEAE20C7F
:10E0480011F80C1041FA09F111F0010F08D0DDF8B0
:10E0580018C04CFA09F111F0010F03D0582110E053
:10E068002D210EE0DDF820C04CFA09F111F0010F66
:10E0780001D0502105E040FA09F111F0010F02D05A
:10E08800542103F8081009F101095FFA89F90BF125
:10E09800010B08F101080132B9F1080F5FFA8BFB97
:10E0A8005FFA88F81CD0B8F1200FB5D125E000BF81
:10E0B8006B130020221E00202C1E0020591A00205D
:10E0C8001E1E0020741E0020151E00204E1A00205F
:10E0D800AE1A0020FC190020F4010020071C0020C3
:10E0E800B8F1200F09D09AF800304FFA8BF2D21805
:10E0F8002B689B7C9A42FFF654AF23490B7813F0A8
:10E10800010F17D02B68214A9B7C12780F2B02F045
:10E11800800298BFC3F11003D2B294BFDBB20023D0
:10E1280042B122789AF800101032521A1849CB18C6
:10E138005F219954174EB37803F00203DBB293B111
:10E14800F11D652246F615632078FAF7FFFB2B6868
:10E158009B7C102B02D905200B2101E00020072110
:10E168003246FAF75FFC2B689B7C102B08D9217884
:10E178000948013102220BB0BDE8F04FFAF7C0BCE4
:10E188000BB0BDE8F08F00BF631E0020883A002066
:10E19800F4010020741E0020F501002088234B4361
:10E1A800054A03EBD003D35C00F0070053FA00F0F4
:10E1B80000F00100704700BF840D002070B50446D0
:10E1C8001646157839B912E00135EDB228462146D0
:10E1D800FFF7E4FF48B9202DF6D970BD013DEDB237
:10E1E80028462146FFF7DAFF08B1356070BD002DDB
:10E1F800F4D170BD064B38211B78032201FB003196
:10E20800044844230370C9B2173BC370FAF778BCBB
:10E218001E1E0020F4010020012802D0022806D189
:10E2280002E01D20044904E01D20044901E00449DE
:10E238001D20FAF73FBC00BF19360308F83503085C
:10E248003A360308037809680F4A03EB03104018AD
:10E2580002EBC00050F8240C0C4988420FD18821E9
:10E2680001FB03239A68A0F59C63063B9A4208D0F9
:10E27800A0F598600538101A18BF012070470020D3
:10E2880070470020704700BF840D0020D735030871
:10E2980003780A6803EB0313D318084A053B02EB1B
:10E2A800C3035968064A914205D1187A09288CBFD8
:10E2B8000020012070470020704700BF840D002017
:10E2C800D73503082DE9F04F984B994FF0221A7073
:10E2D8003B6889B09C6847F67313E11A4C4244EBDB
:10E2E8000104CC3A6243934B9D5C03EB0208C5F3EF
:10E2F8000005EEB23A46002E2CD130468E49FAF788
:10E30800D9FB8E4B1B78232B41F02A8298F80130D9
:10E3180066F3041388F80130FAF790FC884B1A78F2
:10E3280042F006021A70874A1378013BDBB2137079
:10E33800854A52F823303B60844B1D70844B1D7016
:10E34800844B1D70844B1E60844B1D70844B1D7064
:10E3580001F006BA814D95F80090B9F1000F0CD084
:10E368004FF43661614309F1FF30342303FB001396
:10E378007C49CB181B798DF81F307B4B1E787EB1FA
:10E388007A4E2046317811F0DDFF002840F05C8499
:10E3980075493070087007460646804600F05BBC39
:10E3A8006D490B688B46A3F11200032809D9A3F124
:10E3B8001601032909D9A3F11A01032909D93746F6
:10E3C80005E037464FF0010805E037460126B84614
:10E3D80001E00127B04659490978532940F0D58111
:10E3E800B9F1000F3AD1722262436149885C10F09A
:10E3F800020F0AD0002B41F0B381013363F383008D
:10E408008854CBF8003001F0ABB95A4B997989B1EF
:10E4180020464A4611F07EFFFF2801F0A181013015
:10E428002870CBF80090FAF709FC2046FFF7E2FEC7
:10E4380001F096B9DFF8FCC0242202FB04C251782F
:10E44800204669F3041151704B4A022182F800906A
:10E45800039311F005FF0122039BCDE209F1FF317F
:10E468002046C9B211F06EFF002840F08B80DFF81B
:10E4780010B1DFF8EC909BF80020012332B98BF83B
:10E488000030324B89F800201A70E4E305900393BA
:10E49800FAF7D4FB05988BF80000039B89F8003045
:10E4A800364A835C9246A3F13001C9B2092904D9DE
:10E4B800413BDBB2052B01F2538101300A28EFD131
:10E4C8004FF0000847460AEB480017F005F87B08AC
:10E4D8000237FFB20A2F294E0AF8030008F1010893
:10E4E800F1D1304612F034FC002801F03981304671
:10E4F80012F09CF90746002841F032811D4B304646
:10E50800997912F034FC002801F02A8129783379AE
:10E5180001392046C9B202220097019612F07AFC0E
:10E52800022389F8003001F01BB900BF6F1E0020DC
:10E53800841D0020903A0020672703084C1D002006
:10E54800631E0020431E0020501E0020691D00206D
:10E55800921D0020131E00202C1E00201E1E0020CD
:10E56800151E0020283F0020601D0020141E0020DA
:10E57800E85500206B130020621E0020441E002076
:10E588001F1E0020DBF80030DFF80893202B27D06F
:10E59800212B23D14FF43662624329783420013984
:10E5A80000FB0122AC489DF81F3012184FF0000BF9
:10E5B80020460192C9B20322CDF800B012F02AFC1D
:10E5C800FAF73CFB2A78A54B013AA5481A701423A0
:10E5D800C9F800B085F800B003703CE31E2B03D1E6
:10E5E8000133C9F8003019E31F2B18D14FF43662F4
:10E5F800624329783420013900FB012296484FF004
:10E60800000B121801929DF81F302046C9B206224D
:10E61800CDF800B012F0FEFBC9F800B0FEE29A1F78
:10E62800062A0ED88F4B1A7819462AB901321A7061
:10E638008D4B1A788D4B00E3012A40F00C8302239E
:10E64800A1E1A3F10D02042A3AD88949D3B291F87D
:10E6580000C095F800E08048864ABCF1000F1ED043
:10E668004FF0000C81F800C011784FF43662624315
:10E678000EF1FF3E0CF1340C0CFB0E228018C01872
:10E688004174382000FB04EE5FFA8EF000EB800046
:10E6980000F5FA409B30C01803F080FBDBE24FF036
:10E6A800010C81F800C04FF4366161430EF1FF3E62
:10E6B8000CF1330C0CFB0E1E7044C3185B7C59E044
:10E6C800A3F112020B2A4CD86B4A2978107800283B
:10E6D80045D000201070A3F1120938224B1E02FB0E
:10E6E8000433203ADBB2534303F5FE435FFA89F95A
:10E6F800DFF894B1CB3303EB49039BF800101846BD
:10E70800039303F04BFB5D4A4FF4B66C0CFB04FC1F
:10E7180011781A22013902FB01C14F48494400EB24
:10E7280041019BF80000DFF870B18875039B9BF8E6
:10E738000010581C0492CDF814C003F02FFB4F4969
:10E74800049A0B78DDF814C0013B02FB03C2424B6C
:10E758004A4403EB42029BF80030D3757BE2012365
:10E7680008E0DFF8209199F800302BB9012289F8E8
:10E778000020434A13706EE2FAF760FA002389F822
:10E7880000302046FFF736FD65E243294BD1354A74
:10E798001278002A40F05F82354A1278002A40F049
:10E7A8005A82B9F1000F00F05682364A1278002AD0
:10E7B80040F05182212B30D01F2B30D02E4B1978AE
:10E7C800012919D9B8F1000F02D1002F00F04382B6
:10E7D8002D4B02391A7852FA01F010F0010F4FF060
:10E7E800010004D010FA01F122EA010225E210FA30
:10E7F80001F141EA020220E200F02D8209F1FF3125
:10E808002046C9B211F09EFD20B9204B1B78002B81
:10E8180040F0218200232B7000E2202300E01E2319
:10E82800CBF80030FAE1232940F096800D4B1B7895
:10E83800002B40F010820E4B1978002940F00B8213
:10E84800104BB9F1000F50D01A783AB30C480F2A80
:10E8580001700F48017042E1283F0020141E00207B
:10E86800601D0020621E0020121E0020701E002065
:10E878002B1E0020E01E0020171E00201E1E002058
:10E88800691D0020131E0020111E00201F1E0020DD
:10E89800921D00202C1E0020611E002009F1FF316E
:10E8A8002046C9B211F04EFDB0B19A4A13787BB137
:10E8B800B8F1000F01D0042B08D90EB1012B05D9EE
:10E8C800002F00F0C881042B00F2C281013351E708
:10E8D8009DF81F000121F6E08F4B1A78511EC9B22E
:10E8E80008296FD801321A706CE0DFF86CC2242155
:10E8F80001FB04C1487869F30410487002212046DE
:10E908000492039311F0ACFC09F004FCFAF796F9B1
:10E918008249087840F0060008708148017801397A
:10E92800C9B201707F48049A50F8211011607E4ADC
:10E9380082F800907D4A82F80090039BCBF8009003
:10E9480083F800907A4B85F8009083F80690794B0D
:10E9580083F8009000F004BF2A2936D1764B1B7843
:10E96800002B40F07881754B1A78002A40F07381AB
:10E9780073490B784BB16C48012B02706B480270DD
:10E9880040F26981013B0B7065E1B9F1000F00F0BD
:10E99800628109F1FF312046C9B211F0D3FC58B1A8
:10E9A8005C4A137823B1012B40F25581013BE1E623
:10E9B8009DF81F00002186E0574A1378012B01D9E2
:10E9C800013B13700022584B37E1442940F08D80F9
:10E9D800594A1278002A40F03E81B9F1000F0DD152
:10E9E800534B9A79511EC9B2012901D8013203E06B
:10E9F800032A40F03081023A9A712CE1504A127889
:10EA0800002A40F02881444A1278002A40F02381E5
:10EA18004A4A1278002A58D13E4B1B78012B09D953
:10EA2800002E00F01881474B1A78072A00F212814D
:10EA38000132AAE019D1B8F1000F0BD0424A0320E5
:10EA480011789846013191FBF0F000EB4000091A6B
:10EA5800117000E1002E00F0FE803B4A1E4611783E
:10EA6800013101F003011170F5E0314B204699792D
:10EA78004A4611F04FFCFF2800F0ED80DBF800302B
:10EA8800212B00F0E8801F2B00F0E5800130287072
:10EA98002046FFF7AFFB4FF43662624329783423F0
:10EAA800013903FB0123294A9BF80000D31893F886
:10EAB800049049468DF81F90FFF770FB0146002827
:10EAC80040F0AC804846224AA6E00D2B0BD19DF8B9
:10EAD8001F0011F0E9FA30B11E4B1A781F2A00F214
:10EAE800BA800132A9E00120AAE0552940F0B3809C
:10EAF800114A1278002A40F0AE80B9F1000F2DD1EA
:10EB08000B4B9A79012A01D9013A75E740F0A380A5
:10EB1800032271E7171E00201F1E0020631E00201D
:10EB2800431E0020501E0020691D0020921D002059
:10EB38006B130020151E0020621E00202B1E0020D3
:10EB4800131E0020111E0020611E0020283F0020F7
:10EB58002C1E0020E01E0020903A0020894A1278DE
:10EB6800002A78D1884A1278002A74D1874A127804
:10EB7800002A56D1864B1A78012A08D9002E6AD065
:10EB8800844B1A78012A65D9013A1A7062E012D1C9
:10EB9800814B197811B1013919705CE0B8F1000F97
:10EBA80003D002211970904655E0002E53D003215E
:10EBB800197016464FE0B9F1010F4CD9774BA9F1FE
:10EBC800020220469979D2B211F0B2FBFF2842D056
:10EBD800DBF80030DFF8D091212B3CD01F2B3AD046
:10EBE800013028702046FFF705FB4FF43662624378
:10EBF80029783423013903FB0123694A99F8000075
:10EC0800D31893F804B059468DF81FB0FFF7C6FA29
:10EC1800014618B958464A46FFF7D0FAFAF70EF8EF
:10EC280019E00D2B0BD19DF81F0011F03DFA30B102
:10EC38005C4B1A78012A0ED9013A1A700BE0FF20B2
:10EC4800584911F04FF906E000273E46B84602E061
:10EC5800012700E001262978DFF89891002940F083
:10EC6800CB8099F8003013F0010205D143F001037D
:10EC780089F800304C4B1A6000252046294611F0CF
:10EC8800FBFD30B172236343484AD15C41F0020175
:10EC9800D1540135382DF0D13A356543434E735D73
:10ECA80013F0020F43F3400015D03F4C206810B911
:10ECB8003F4900F0C1BC00203E49F9F7FBFE735DF7
:10ECC80013F00C0F43F3810540F04A85F9F7B6FFBE
:10ECD800256000F045BD314DAB79A3B1012B01D1C1
:10ECE800354906E0022B01D1344902E0032B02D159
:10ECF8003349F9F7DFFEA979204611F055FB0222C6
:10ED080001463048EDE114B920462F4901E02F496A
:10ED18001846F9F7CFFE2E4803786BB92D490A2219
:10ED28002D48F1F70DFE2D49242303FB04135A78CF
:10ED380042F010025A7004E0274829490A22F1F7E4
:10ED4800FFFD284D3821022205F11E00F9F7D8FEF3
:10ED5800204611F04DFB0222014605F11900F9F792
:10ED6800CFFE214B00221A70204B1B7803F0800342
:10ED7800DBB2002B00F0F4841D4B1B88EB8100F004
:10ED8800EFBC00BF131E00201F1E00202B1E0020FA
:10ED9800171E0020111E0020611E00206B1300208A
:10EDA800283F0020E01E00202C1E0020E8550020EF
:10EDB800A9270308CA270308D2280308F328030849
:10EDC80014290308120200200C28030890280308BD
:10EDD800601D002035290308FA010020903A002020
:10EDE80056290308F4010020151E0020883A002047
:10EDF800D9A10308631E002001392046C9B211F0C9
:10EE0800A1FA002800F0F483954B93F800B038235A
:10EE18000BF1FF3B03FB04BB99F800305FFA8BFB57
:10EE280013F0010F03D08F4A1378002B41D08E487E
:10EE3800F9F7E6FD0BEB0B1101F5EA4110228B48BF
:10EE4800BB3102F0C6FF884B11229A71884B1B68B0
:10EE580013B91020874921E0012B02D110208649DF
:10EE68001CE0022B02D11020844917E0052B02D1A7
:10EE78001020834912E01E2B02D1102081490DE099
:10EE88001F2B02D11020804908E0202B02D110202E
:10EE98007E4903E0212B03D17D491020F9F70AFEB2
:10EEA80099F800306F4843F0010389F800300023D7
:10EEB8000370784B1A78002A00F0AB800BEB0B1B21
:10EEC8000BF5EA4909F1BB0910227348494602F0DB
:10EED80080FF00229346704B995C41B10BF1010B06
:10EEE8005FFA8BFB0132BBF1100FF4D107E06A49DE
:10EEF800C2F1100201EB0B002021F1F74BFA654A31
:10EF0800107858450BD90138484402F051FF30B900
:10EF1800604B202118780138484402F03FFFDFF8A1
:10EF280094B19BF8003018460393F9F77FFEDC464E
:10EF3800039BDFF878B110B9432B44D101E0432B90
:10EF480005D100238BF800304FF0200A30E05348F9
:10EF5800534A90F800E053499E450ED1AEF1300E69
:10EF68000A20137800FB0E1E0133DBB213707344C2
:10EF780093F8AD307BB913700DE003709BF8003047
:10EF88004FF0000E82F800E02BB1424803780F2BB7
:10EF980001D80133037040238BF8003013789CF8B4
:10EFA80000200A20303A00FB0211C91891F8ADA0E0
:10EFB8003849394A08785146013802F800A04844CF
:10EFC80002F0ECFE0FE0384B1B7803F08003DBB255
:10EFD8004BB19BF8003033B92E482F490378FF22F4
:10EFE800CB1803F8012C9BF8003013B12F4A013BD2
:10EFF80013709BF80030012B10D1264A13780F2B81
:10F0080001D801331370264A00238BF8003013709F
:10F0180004E004200C21144AF9F704FD144A13688B
:10F028009346002B48D14FF4366262432978342442
:10F03800013904FB01241E4AA4186178164AC1F359
:10F04800C30109B93F2004E0994201D9DB2000E05F
:10F05800A5200133DBB2907501320A2BF1D17FE391
:10F068001E1E0020151E0020741E00207B1E00207E
:10F078002C1E0020533503083D2A03087F2A030865
:10F08800452B0308EA2B03080B2C03082C2C030838
:10F098004D2C0308131E0020F4010020661D0020DB
:10F0A800921D00205CB30208883A0020691D0020E8
:10F0B800303F00204C1D0020012B15D14FF4366342
:10F0C80063432A783424013A04FB0234AB4BE41836
:10F0D800637813F0070300F0438314215943A848C9
:10F0E8008322F9F70DFD3BE3022B26D1A54A9DF8B3
:10F0F8001F30882101FB03232978A34AD8790139D5
:10F108000623202502F8015950FA03F515F0010FDE
:10F1180010D04FF436656543342606FB01559B4EE7
:10F128007519ED791D4115F0010F01D0DB2500E0BF
:10F13800A5255570013BE4D212E3032B13D14FF4FC
:10F14800366363432A783424013A04FB02348F4B34
:10F158001C19237A13F0010F02D010208C496BE29E
:10F1680010208C4968E2042B13D14FF436636343B3
:10F178002A783424013A04FB0234844B1C19237A7C
:10F1880013F0020F02D01020834955E21020834962
:10F1980052E2052B15D1162700262B783422013B85
:10F1A80053434FF4366202FB0433784A7C49D31840
:10F1B800985DC919013616F075F90237052EECD19C
:10F1C800CEE2991F062900F2FF809DF81F206D4F9F
:10F1D80002EB0210411807EBC101C968714801F13F
:10F1E800100651F804CBB14240F804CBF9D19E1F68
:10F1F800F6B202EB02129219013207EBC202507A00
:10F2080092F80AC0684A29781378904673B94FF47F
:10F21800366363433422013902FB0131634BCA5E12
:10F22800634B024102EA0C021A7011E0022B0FD163
:10F23800604B01391B784FF0000900932046C9B292
:10F2480004223346CDF8049011F0E4FD88F80090CC
:10F2580098F80030012B29D1574BDFF8589193F8D3
:10F2680000A05046F9F7E2FC10B9BAF1430F1AD1E1
:10F278000DF11F005149FFF70BF810B1002389F871
:10F2880000309DF81F30DBF8002003EB03139B18B8
:10F2980007EBC303504699F8001013F8202CFAF72F
:10F2A800DBFC89F8000099F800A003E013B9404B93
:10F2B80093F800A0BAF1090F07D9BAF1630F8CBF10
:10F2C8004FF003094FF0020901E04FF001099DF8E2
:10F2D8001F3003EB03139E1907EBC607FB685A7B25
:10F2E800E02A02D12E4A202151779A7BE02A02D1C6
:10F2F8002B4A20219177DA7BE02A02D1284A202163
:10F30800D17798F800200ABB4FF436626243297817
:10F318003424013904FB0124184AA418A27812F0F5
:10F32800080F1BD05A7BE02A02D11D4A3F21517792
:10F338009A7BE02A02D11A4A3F219177DB7BE02BA6
:10F3480040F00E82164B3F22DA7709E21C4B1B78FD
:10F3580003F08003DBB2002B40F002820DF11F00A6
:10F368001649FEF76FFF18B15046FEF755FFF7E153
:10F3780014485146C9EB00004A46B2E6303F002027
:10F388000F020020840D002013020020283F0020D7
:10F39800E22A0308032B0308A82B0308872B03087A
:10F3A800F401002004020020621E00202D3F0020EE
:10F3B800121E0020701E00204C1D00202C1E002054
:10F3C800883A002014020020A3F10D02042A31D843
:10F3D8009DF81F30D6B2222202FB0363984A02EB43
:10F3E80083035F6C3846F1F725FA3946024695489B
:10F3F800F1F7A6FA944B1B786BB1944B1B7803F08A
:10F408008003DBB21BB1924820210222EDE0914B30
:10F418008F4819780CE04FF4366363432A78342414
:10F42800013A04FB02348C4B89481C19A619717CDB
:10F43800822256E6123B0B2B00F292819DF81F2088
:10F44800DBB2222101FB02317D4A163152F821201C
:10F458007C4902F110008A4652F804CB824241F8F6
:10F4680004CBF9D1DFF83092DFF830B22FB199F838
:10F478000020012A15D1013209E096B199F800203F
:10F48800012A07D97549097803290AD1013A89F867
:10F49800002006E005D171490978032908BF8BF8D7
:10F4A800002099F800209AB94FF4B6614C432A78A5
:10F4B8001A21013A01FB0244674AE318083302EBB8
:10F4C80043039A798BF80020DA79644B1A7047E184
:10F4D800634C202104F118000822F0F75BFFB8F113
:10F4E800000F00D1AEB15D4D2B78012B01D15D4AE3
:10F4F80001E04BB95C4A136823615368CAF80430C9
:10F50800B8F1000F21D00BE0022B0CBF574A584A24
:10F51800F1E7584A136823615368CAF8043019E1BF
:10F528009BF800004E4A3121002350FA03F515F0EC
:10F53800010F01D0117701E02D2515770133013135
:10F548000132042BC9B2F0D12FE0002E00F0028165
:10F55800202108224848F0F71DFF3D489BF800107D
:10F568008222F9F7CDFA394B1B7803F08003DBB21E
:10F578001BB199F80030012B02D82B78032B21D12D
:10F58800202102223248F0F705FF1BE050FA03F56C
:10F5980015F0010F01D0117701E02D251577013302
:10F5A80001310132042BC9B2F0D1284B1B7803F08A
:10F5B8008003DBB233B199F80030012B02D9E4188B
:10F5C8002023A376214B1B7803F08003DBB2002BAA
:10F5D80000F0C68099F80030012B40F0C180002F60
:10F5E80040F0BE80174820210822F0F7D3FEB7E08C
:10F5F80099F80030214D13F0010F04BF43F00103C7
:10F6080089F800302E78002E4AD12D210A221C4874
:10F61800F0F7C0FE04201B49F9F74CFA1A4B1B7887
:10F62800012B02D11020194906E0022B02D110202B
:10F63800174901E017491020F9F73CFA90E000BF9C
:10F64800840D0020040200202B1E0020883A002090
:10F6580012020020E01E0020283F0020611E00202A
:10F66800F40100208D340308AE340308CF340308B6
:10F67800F0340308093403080C0200201F1E002080
:10F68800441E00207C360308151E0020662B030844
:10F69800242B0308452B0308171E0020111E0020E9
:10F6A800314B1C782046F9F7C1FA304B304A002814
:10F6B8002AD0304F30493878A04216D130380C78EB
:10F6C8002E4E00EB80073C19345D04B90C700F789E
:10F6D80000EB8000C4190137FFB2C0190F70315C0C
:10F6E800345D59B92448017008E001200870197880
:10F6F8003C7019B1092E9CBF36182E702978511804
:10F7080001F8014C40211970197811B117480139D5
:10F7180001701978012909D12978092902D81848CE
:10F728000131017000211970134B19701168154BC4
:10F73800C3F816105168C3F81A101289DA83124AEE
:10F74800127802F08002D2B252B12A789B18202295
:10F758005A7505E09BF800000A4A3121002315E795
:10F7680009B0BDE8F08F00BF4C1D0020691D0020C6
:10F77800441E0020661D0020921D00205CB3020874
:10F788001F1E0020F4010020883A002010B5002335
:10F7980086B004468DF8143011B118460C4901E0C2
:10F7A80008460C49F9F786F9217810220139C9B2BF
:10F7B80001EB011101F5C241483101A802F009FB32
:10F7C8001020014601AAFDF7EDFD06B010BD00BFEF
:10F7D80074140308B61403080B4B1B78442B06D08B
:10F7E800552B037801D013B17047013B01E0037832
:10F7F8000133037003780BB9203302E0212B01D1C8
:10F80800203B0370FFF7C2BF4C1D00202DE9F74FC6
:10F81800DFF8CC91DFF8D8A199F80030554643F0CD
:10F82800010389F800309AF80130644C23F07F0313
:10F838009B46D3B100206249F9F73CF961482A2177
:10F84800F0F726FE18B121788222F9F759F92278C3
:10F85800002A40F0AF802B6862F3CF332B605A4BFD
:10F868001A7842F003021A70A4E0574F23703B78CD
:10F878003E4603F00202D2B20192DFF87881002AF4
:10F8880044D013F001092BD058465049F9F712F922
:10F8980098F80030232B0CD14D4B4E4A4E481A6035
:10F8A8000121FFF773FF3B7803F0FE036BF341037D
:10F8B8003B7098F800302A2B7CD1337803F0FE0394
:10F8C8006FF3410333702B6843F400432B600F231D
:10F8D8002370414B187803B0BDE8F04F0FF068B8BB
:10F8E80048463E49F9F7E6F898F80030232B61D1ED
:10F8F800374B384A38481A600121FFF747FF3B78F1
:10F9080069F3000369F341033B7053E00EF0A1FF74
:10F91800054600282FD001212F48FFF75DFF98F8F2
:10F928000030532B12D13B78019A03F0F10362F3B4
:10F9380000033B70DAF8003043F40043CAF80030A3
:10F948000F232370244B18780FF032F898F8003002
:10F95800232B2FD13378002203F0FD036FF300032C
:10F9680033701D4B1A70F9F769F91D4A137843F083
:10F978000603137014E01B49F9F79CF898F8003057
:10F98800232B17D13B7865F3410365F300033B70E4
:10F99800F9F754F999F8003043F0060389F8003074
:10F9A800114A1378013BDBB21370104A52F8232036
:10F9B800074B1A6003B0BDE8F08F00BF5259002012
:10F9C800F8140308F4010020DF3C0020191503088F
:10F9D800841D002000B502081E1E00203A150308E9
:10F9E800631E00205B150308431E0020501E0020E4
:10F9F800883A00204C1D00202DE9FF41364C374D38
:10FA0800237843F001032370297801F00401C9B277
:10FA180011B93348FFF7E0FE2B7803F00402D2B2A5
:10FA280032B1304A12781AB92C4A43F008031370DD
:10FA38002D4E3378232B26D12B782A4A6FF3C30314
:10FA4800002113F004082B70284F117009D0234AA5
:10FA580061F382031370264B21483B60FFF796FE43
:10FA680011E0F9F7EBF82378224A43F006032370F4
:10FA78001378013BDBB213701F4A52F823303B6006
:10FA8800174B83F800803378532B23D12B78042429
:10FA9800144A03F0F403234314702B70104B0B2209
:10FAA8001D781649013DEDB202FB05F000F5CA408C
:10FAB800883002F088F900201149F8F7FBFFFF238E
:10FAC800002100930135162022460B46019102952C
:10FAD80002F0ECF9BDE8FF81631E0020DF3C002046
:10FAE8001E1E0020525900204C1D0020841D00209D
:10FAF8001CB50208431E0020501E0020D43C0020E4
:10FB0800D71403082DE9F041984B04469A7812F06F
:10FB1800010F00F017811B88002B40F01381944DD2
:10FB280095F820303F2B40F2D780012C14D1914B0F
:10FB38001B7803F00203DBB2002B00F0C48095F8B9
:10FB480020208B4B402A03D1013283F82020FBE090
:10FB5800482283F82020B6E0022C03D1482385F8F8
:10FB68002030B0E0844E337803F02002D2B28AB15C
:10FB780095F82020402A0DD1032C0BD07F4B804ACA
:10FB880003F1100153F8040B8B4242F8040BF9D12E
:10FB9800412395E003F01003DBB28BB195F82030D8
:10FBA800412B0DD1032C0BD0764B754A03F1100174
:10FBB80053F8040B8B4242F8040BF9D142237FE03F
:10FBC800F37813F0010F0FD095F82020422A0BD1BB
:10FBD8006D4B6B4A03F1100153F8040B8B4242F84A
:10FBE800040BF9D143236BE003F00202D2B27AB1DD
:10FBF80095F82020432A0BD1644B614A03F1100188
:10FC080053F8040B8B4242F8040BF9D1442357E014
:10FC180003F00402D2B27AB195F82020442A0BD11D
:10FC28005B4B574A03F1100153F8040B8B4242F81F
:10FC3800040BF9D1452343E003F00803DBB28BB191
:10FC480095F82030452B0DD1032C0BD0514B4C4A45
:10FC580003F1100153F8040B8B4242F8040BF9D15D
:10FC680046232DE00FF08AFCA0B14B4B1B788BB1DB
:10FC780095F82030462B0DD1032C0BD0474B404A2A
:10FC880003F1100153F8040B8B4242F8040BF9D12D
:10FC9800472315E0F37803F04003DBB29BB195F8F6
:10FCA8002030472B0FD1032C0DD03D4B344A03F1A4
:10FCB800100153F8040B8B4242F8040BF9D1482386
:10FCC80085F8203078E095F820300133DBB2472BF7
:10FCD80085F820307FF629AF95F82060472E04D9A3
:10FCE800234B002683F8206001E00136F6B206F1C6
:10FCF8004007FFB212E02B48314615F0B8FB08B1B7
:10FD0800032C04D1284B9B5D23B1032C02D185F829
:10FD180020600FE00136F6B2BE4203D03F2EEAD98A
:10FD2800402E07D1214B1E221A70402385F820301F
:10FD3800BDE8F08195F820001149652246F6156363
:10FD4800F8F704FE012C37D1194B0D4A03F11001C5
:10FD580053F8040B8B4242F8040BF9D1044B93F887
:10FD680020303F2B3CD9002012493EE0741E002071
:10FD7800F4010020181A0020883A0020AC1B030860
:10FD88007B1E0020CD1B0308EE1B03080F1C030875
:10FD9800301C0308511C03081C3F0020721C030878
:10FDA800B41C0308AE1A0020641A0020201E00208C
:10FDB800AC7E03086A1B0308104BD87800F02000BB
:10FDC800C0B220B1022C06D000200D490DE0032C52
:10FDD80001D10C4909E00C4B93F820303F2B02D895
:10FDE80000200A4901E00A490020F8F763FE1020C4
:10FDF800084A0146BDE8F041F8F714BE883A0020E9
:10FE0800851203088B1B0308F4010020281B030834
:10FE1800931C0308741E002010B5F8F70FFF084B59
:10FE28001B7803F00403DBB22BB106490020BDE8C0
:10FE38001040F8F73FBE0220BDE81040FFF762BE51
:10FE4800181A00205A19030870B5224B06461B7869
:10FE5800214CF3B9257819E02048294615F007FB0D
:10FE680078B123689D4202D9FF2E02D007E0FF2E09
:10FE780002D19D4208D202E036B91DB913B92560F6
:10FE880012E00EB9013500E0AD19EDB23F2DE3D90E
:10FE98000AE0013B2021124810222360F0F77AFA89
:10FEA80000201049F8F706FE0F48F8F7A9FD46F6B6
:10FEB800156320780D496522F8F748FD084D21683B
:10FEC80005F1100001310222F8F71AFE2D23AB7458
:10FED80070BD00BF131E00202C1E00208A1D0020AC
:10FEE800F4010020285D0308741E00207B1E0020FA
:10FEF800F8B5594BF02259481A700378044613F0A4
:10FF08000E051DD1564A43F00203156000F8013B67
:10FF180015F052FA2C46534BE35C1BB1524821466C
:10FF280015F08FFA0134402CF5D1504B01221A708C
:10FF380010F072FB4E4B1A7842F001021A70F8BDAD
:10FF480013F00C0543D12E464748294615F08FFA81
:10FF580008B10136F6B20135402DF5D11EB9237826
:10FF680043F0040331E0002542482946EFB215F07A
:10FF78007EFA68B13B4BEB5C53B13F4B01371F70C6
:10FF88000020FFF761FF237843F00803237002E0A5
:10FF98000135402DE8D1394D3A212846F0F778FA55
:10FFA80038B1401BC0B20130281831460222F8F798
:10FFB800A7FD334B1B78532B4CD12F4B00201870C7
:10FFC800FFF742FF237843F008032370F8BD6FF36F
:10FFD8004103037003F00403DBB2294D23B1002071
:10FFE8002849F8F767FD0EE02B78552B01D1FF2043
:08FFF80002E0442B02D10120BC
:020000040801F1
:10000000FFF726FF13200D21214AF8F70FFD2B786B
:10001000232B23D12478134E04F00204F4B9154B9A
:100020001C7010F0FDFA337803F0FB0364F3C30394
:1000300033700D4B1C60F8F705FE0F4B1A7842F039
:1000400006021A70134A1378013BDBB21370124A8E
:1000500052F82320114B1A60094B1C70F8BD00BFE9
:100060006F1E0020891D00202C1E0020B02C0020B7
:100070008A1D0020B0140020631E0020191A0020E1
:10008000131E0020F40100204C1D00206E6E03089A
:10009000741E0020431E0020501E0020841D0020DE
:1000A00070B505460C4616463BB1400000F536409B
:1000B00039304018114601F075FE054B292202FB2C
:1000C0000535F3092C1906F07F066370E67070BDE4
:1000D000A53B002038B510B3A0F14103DBB2432BA0
:1000E0001FD9C50900F07F040BD0052C19D90021B8
:1000F000601E0A460BF0D4FAD0F1010038BF002090
:1001000038BD082C0FD9601EC0B229462A460AF015
:1001100015FF50B9202C8CBF0020012038BD0120D4
:1001200038BD002038BD284638BD284638BD0000FF
:10013000F7B5604F604C387831234000237400F5E8
:100140003640013323763930053B6374637601F022
:1001500033FEC0B220F07F0200F07F01D2B28DF8F2
:1001600004108DF8002004F1120359B9534A04F128
:1001700015001188927861829A7020210222F0F78E
:100180000DF90CE0D20904EB8202526A10886082F9
:10019000927804F115009A700222F8F7B5FC3878CD
:1001A000400000F536403A3001F006FEC0B220F0C3
:1001B0007F0300F07F01DBB28DF805108DF8013070
:1001C0003F4851B93D4B20311A889B786283837038
:1001D00002220330F0F7E2F80BE0DB0904EB8303C3
:1001E0005B6A1A8862839B78022283700330F8F777
:1001F0008BFC344B1B7813F0010F5AD0324D02A9FF
:100200002A788B1813F8041C13F8086C2F4B1B78F2
:10021000232B04D1002A41D1223B2B703EE02A2B14
:1002200004D1002A3AD0013A2A7037E0552B46EA29
:10023000010611D10DE02B7802AAD318013E13F864
:10024000081CF6B23046C90913F8042CFFF742FF28
:1002500098B9002EEFD121E0442B19D115E02B786D
:1002600002A9CB18013613F8081CF6B23046C909AA
:1002700013F8042CFFF72EFF38B1134B3878197898
:1002800032460123FFF70CFF08E0872EE7D905E08F
:10029000532B03D1533B2B70F9F7C2FC0C4B1B784B
:1002A00003F08003DBB223B12B782022023304F861
:1002B0003320FEBD131E0020F40100206B7A0308DA
:1002C0000E020020631E00201E1E00204C1D002078
:1002D000883A0020024800210922F0F75FB800BFE9
:1002E000311E002070B50A46002405E01B19811A52
:1002F0002A2501345D54E4B20F4D104B295D09B13C
:100300009442F3D1801A001918182021121BF0F71B
:1003100045F80B4B1E7876B1432E07D114B1013C42
:10032000E4B201E0074B1C7000232B553046F8F770
:1003300081FC00B12E5570BD311E0020F40100205B
:100340004C1D0020721E002038B5184C184DA078A6
:1003500000F01000C0B250B91649F8F7AFFBFFF734
:10036000B9FF236843F4801323600F232B702A788E
:100370002AB92368FF2062F31453236038BD0E4866
:10038000C5792DB91C200821FFF7ACFF284638BDE0
:1003900023680A496FF3145308222360F0F77EFAAA
:1003A00000280CBF0120FF2038BD00BF883A002084
:1003B000721E0020BD190308311E0020C4990308D5
:1003C000F0B55C4C85B0667806F01006F6B2002EEB
:1003D0003ED1594B1A78594B013A53F82230584ABA
:1003E000934204D1574B1A7842F0020207E002F11F
:1003F0001C018B4208D1534B1A7842F004020221AF
:1004000061F3C7021A7019E03832934216D1FFF730
:100410009BFF002800F08C8001284A4D06D12B78E4
:10042000022243F0010362F3C70306E03046464967
:10043000F8F744FB2B7866F3C7032B70434B1A780D
:1004400042F001021A70236843F4805323606FE086
:100450003C4D2B7813F0F80606D03D49002005B03E
:10046000BDE8F040F8F72ABB13F0070F41D003F0C6
:100470000202D7B24FB11220314611F013FAFF2316
:1004800000930196029643202AE003F00406F6B298
:10049000A6B13946384611F005FA382102200FF08E
:1004A000C5FD0AF01BFB0EF0FFF9FF230093019737
:1004B00002974420394604223B4614E013F0010F12
:1004C00013D0012143F6206011F0ECF93046F5F726
:1004D000EFFE204B45201E80FF23009301960296DD
:1004E00031460422334601F0E5FC00201A49F8F7B2
:1004F000E5FA2B7803F0FA036FF341032B70174BE7
:100500001B78232B14D123686FF30C332360F8F787
:1005100099FB0E4B1A7842F006021A70064A1378BD
:10052000013BDBB21370054A52F823200C4B1A60D2
:1005300005B0F0BD883A0020431E0020501E002068
:1005400038B50208CC560020DE190308631E0020CF
:100550000A720308621D0020E97103084C1D002087
:10056000841D00201FB50446F5F78EFFA8B14B206F
:1005700002F072F8FF2300930121FF3B0193392021
:1005800004220B460134029401F094FC064B012036
:100590005A7842F004025A7004E0044B188800387C
:1005A00018BF012004B010BDB43C002068590020E1
:1005B000F0B5204E0024337A0546013385B00F464E
:1005C000337210202146012223460094F2F79CF852
:1005D00055B9FF2300934F20294604222B4601954D
:1005E000029701F067FC0EE0012D0CD1FF23009370
:1005F00050202346214604220194029701F05AFC20
:10060000337A013B3372337A052B11D1FA3301214E
:100610000024009327200B4604220194029401F049
:1006200049FC044B1C7205B0BDE8F04001F0E6BF88
:1006300005B0F0BD221E0020074B292202FB00332B
:100640005B7913F0100F05D0044B283ADA711A7158
:1006500009321A72704700BFA53B00206B130020BF
:10066000044B1878A0F1010CDCF1000040EB0C0009
:10067000704700BF801D0020034B1878A0F10202D4
:10068000504240EB02007047801D0020034B187859
:10069000012894BF00200120704700BF801D00206A
:1006A000064B1A7802F0F7026FF304121A70044B2B
:1006B00000221A70034B03321A707047301E00205C
:1006C000721E0020801D002010B5214821490368BA
:1006D0000A789C7B944203D99C8914F0200F18D08F
:1006E0009A8912F0800F01D105E01C3B9A8912F023
:1006F000400FFAD000E01C33036000230B70036846
:100700009B8913F0200F16D0134BDA79114B1A7016
:1007100011E00132D2B20A70986843F60953984248
:1007200009D101E00132D2B2162A03D80B4853B2E4
:100730009840F7D40A700A4A136843F48073136030
:10074000F8F7C4F8074B1A7842F006021A7010BD89
:10075000841D0020131E0020221E00200006008899
:10076000883A0020631E002010B52349234A0B78E5
:10077000D3B11068848914F0200F15D1013BDBB28E
:100780000B70846843F60952944228D104E013B1F7
:10079000013BDBB200E0837B162B03D8184C5AB226
:1007A0009440F4D40B701AE01368988910F0400F4D
:1007B00001D106E01C33988910F0800FFAD0136045
:1007C00002E00E481C3B036013689A7B0A709B8909
:1007D00013F0200F03D00B4BDA79074B1A700A4A3B
:1007E000136843F480731360F8F770F8074B1A78B6
:1007F00042F006021A7010BD131E0020841D002056
:1008000000060088221E0020883A0020631E002077
:10081000074B084A1B68934202D01C32934205D111
:10082000054B1878003818BF01207047002070472A
:10083000841D00208CB50208141A0020074B084ABA
:100840001B68934202D01C32934205D1054B1878A5
:10085000003818BF0120704700207047841D002019
:10086000C4B50208141A002070B50A4C0546E071A0
:1008700000F56A507C3001F09FFA207005F5D840F1
:10088000E93001F099FA60702046BDE87040F5F754
:1008900027BD00BF221E00202DE9F0479A4B86B0ED
:1008A0001A7806460F461C461AB1012A40F0DA8132
:1008B0002FE0964B1A68964B9A4200F0D581F5F7D7
:1008C00063FA944B5B7803F00203DBB253B9924BAB
:1008D0005B7803F08003DBB223B901F0B5FE08B901
:1008E0000AF0FCF88D4B1A686FF310421A6037B9A2
:1008F0008B4B1878F8F79EF9002800F0B581FFF7C8
:10090000E9FC884B3C221A70F7F7E0FF23780133AB
:100910002370844B1B7813B9FFF7C2FEA4E10121B9
:1009200030460AF0FDF8F7F7C5FF00207E49F8F7DA
:10093000C5F806211B20FFF7D5FC7C4B7C491A78B3
:1009400098468A1812F8312C002A00F08D81794AD5
:100950007949137891F80090C3F3C00AC3F30015E6
:1009600003F0F7036FF3041309F00109137017B1D3
:100970000223237000E027700B21062204A801F057
:100980002CFA98F8002004A86949303AEFF72CFCBB
:10099000044610B11227002429E04AF6EB0001F0CA
:1009A0000BFA0028F6D0654D2C72F5F753FB044680
:1009B000002840F05981624A544B21461A60FF23B7
:1009C00000930190029004220820234601F072FA5D
:1009D000012223460E2021460094F1F795FE594B43
:1009E0001A7842F004021A700123AB713CE13946D7
:1009F000062204A801F0F1F998F8002004A84C4957
:100A0000303AEFF7F1FB002840F020812046FFF755
:100A1000A9FD002840F02881DFF82081012188F815
:100A200008002046F5F724FB49EA0A090746F5F7CE
:100A300011FB002840F0BF8038464349EFF7B2FD74
:100A4000C0B901F013FD314BB9F1000F02D115B956
:100A50003E4A24E035B13E4A1A603E4B1A786FF3A5
:100A6000410205E03C4A1A603A4B1A7865F34102AC
:100A70001A70E5E038463949EFF794FD20B1384661
:100A80003749EFF78FFD78B9B9F1000F40F0EC80EE
:100A9000002D40F0E98001F0E9FC324A1B4B1A605E
:100AA0003046FFF7C9FDCBE038462F49EFF77AFD16
:100AB00050B94AF6E900012101F074F9174A1368A8
:100AC00043F400531360DFE738462849EFF76AFD27
:100AD00040B9B9F1000F40F0C780002D40F0C4804C
:100AE000234A0DE038462349EFF75CFD002845D145
:100AF000B9F1000F40F0B880002D40F0B5801E4ADB
:100B0000024B1A609CE000BF801D0020841D002065
:100B10008CB5020872340020C33C0020883A0020C3
:100B20004C1D0020721E002064120308681D002066
:100B3000311E0020301E0020B3640020221E002041
:100B4000FCB502087E26002025A2030848B802084A
:100B5000D0B90208631E0020A8B50208A1A10308AD
:100B600031A40308ECB90208DCA10308DEA10308E4
:100B700024BA0208EEA30308C4B5020838463C496B
:100B8000EFF710FD00285BD101F070FCB9F1000F08
:100B900007D0384A384B1A60384B1A786FF3410245
:100BA00061E0002D60D0364A334B1A60334B1A781F
:100BB00069F3410257E038462D49EFF7F3FC05464B
:100BC00028B901F053FCB9F1000F4DD01EE03846B2
:100BD0002C49EFF7E7FC002846D038462A49EFF7C2
:100BE000E1FC40B9B9F1000F3ED1284A224B88F808
:100BF00007401A6038E038462549EFF7D3FC054630
:100C000060B9B9F1000F16D001F030FC194A1A4B47
:100C10001A601A4B1A7865F3410224E038461D49E0
:100C2000EFF7C0FC20B138461B49EFF7BBFC10B909
:100C3000B9F1000F18D1194A0F4B1A6001F016FCD8
:100C40002046FFF711FE202C0ED105E00134E4B25E
:100C50000737202C7FF4CBAE711C0020C9B2FFF700
:100C6000A7FC01E000221A7006B0BDE8F08700BFC3
:100C7000E0A10308A8B50208841D0020631E00201F
:100C8000D0B90208DEA10308EEA30308C4B5020828
:100C900025A20308A1A10308DCA1030878BA020871
:100CA000034B1B7853FA00F000F00100704700BFBF
:100CB000221E0020034B1B189878003818BF012013
:100CC000704700BF221E0020F8B504460D460E787E
:100CD000FFF7F0FF18B3144A13199F78104600234A
:100CE000021992781A4112F0010F4FF001020DD053
:100CF000BE42297803D09A4042EA010104E09A40BA
:100D0000C2F10F0202EA0101297005E09A40297838
:100D1000C2F10F020A402A700133042BE0D12B7874
:100D200003B92E70F8BD00BF221E002070B57E4BA7
:100D3000044631B11B78532B40F0F580533B0370D0
:100D400070BD1A78302A33D1784B1A795AB1784A63
:100D500078491278292000FB0212527912F0100F04
:100D600001D001221A71744A25781278154012D0E8
:100D70001D7A002D40F0D780E8B2FFF791FF30B127
:100D80000123AB402278C3F10F03134023700135D8
:100D9000042DF1D141E0E8B2FFF782FF20B1012339
:100DA000AB402278134323700135042DF3D134E096
:100DB000A2F13101C9B203293BD85C4E32795AB154
:100DC0005B4A5C491278292000FB0212527912F02A
:100DD000100F01D0012232711D78313DEDB228464D
:100DE000FFF75EFF002800F09E80237853FA05F29B
:100DF00012F0010F0BD0327A002A40F094800132B9
:100E000012FA05F5C5F10F0505EA030304E0012216
:100E100012FA05F545EA0303237000211222474820
:100E2000EFF7BCFA454920461022BDE87040FCF7B8
:100E30008BBA132A0CD0552A18D13D4B3D4A1B784A
:100E4000292101FB03235B7913F0200F03D170BD2F
:100E5000364B01221A7100202146FFF735FF002092
:100E6000FFF728FF00285ED0002054E0142A0CD0A1
:100E70002A2A18D12E4B2F4A1B78292101FB032344
:100E80005B7913F0200F03D170BD284B01221A713A
:100E900001202146FFF718FF0120FFF70BFF002874
:100EA00041D0012037E0152A0CD0232A18D1204B3D
:100EB000204A1B78292101FB03235B7913F0200FC3
:100EC00003D170BD194B01221A7102202146FFF790
:100ED000FBFE0220FFF7EEFE002824D002201AE0DD
:100EE000162A0CD0442A1ED1114B124A1B782921F4
:100EF00001FB03235B7913F0200F03D170BD0B4B73
:100F000001221A7103202146FFF7DEFE0320FFF7BE
:100F1000D1FE40B103200949102246F67973BDE89D
:100F20007040F7F717BD70BD4C1D00206B130020FB
:100F3000161E0020A53B0020221E00204E1D002072
:100F40002DE9F043002387B08DF81730804B1B78D4
:100F5000012B00F07E827F4C227872B17E4B5B7851
:100F6000002B40F076827D4D2B78002B40F0B9802D
:100F7000F7F768FE09232B70B3E0784B19781D460C
:100F8000082900F2AE8076490978232913D11A7016
:100F9000F7F758FE7349744A0B7853B17348013B15
:100FA0000478DBB244F0060404700B70704951F809
:100FB00023301360C1E26D4B1A7812F0010F04D197
:100FC00001210A438DF817101A70F1F7CFFF28B9E5
:100FD0002B781BB90DF11700FCF7B0FDF1F7D4FF2A
:100FE00030B92B78012B03D10DF11700FCF7A6FDCA
:100FF000F1F7D8FF30B92B78022B03D10DF1170090
:10100000FCF79CFDF1F7DAFF30B92B78032B03D105
:101010000DF11700FCF792FDF1F7DEFF48B9F2F78A
:1010200007F830B92B78042B03D10DF11700FCF72A
:1010300085FDF2F731F830B92B78052B03D10DF18E
:101040001700FCF77BFDF2F71BF830B92B78062B65
:1010500003D10DF11700FCF771FDF1F7CBFF30B9AB
:101060002B78072B03D10DF11700FCF767FDF1F783
:10107000CFFF30B92B78082B03D10DF11700FCF707
:101080005DFD9DF81730002B2BD02B78082B23D833
:10109000DFE803F005080D101316191C1F000020CF
:1010A000344901E034490020F7F708FD16E000203C
:1010B0003249F9E700203249F6E700203149F3E7E9
:1010C00000203149F0E700203049EDE700203049A9
:1010D000EAE700202F49E7E7F7F7B4FD2A782E4B1F
:1010E0001A701E4F3B783D46092B40F0BD801F4BC8
:1010F0001B4F1978984611F001015CD1274E12223E
:101100003046EFF74BF90123737415F09FFA10B9CD
:101110002278234B1A70237803B97374737C13B14C
:10112000204B00221A70FCF7EBFC1D48717CFFF786
:10113000FDFD98F8003003F0FD0343F0010388F84B
:101140000030194B1A788AB33A7000221A7032E0D4
:101150006F1E0020141A00206B130020601E002058
:101160004C1D0020431E0020841D0020631E002013
:10117000501E00201E430308FD4203083F4303089E
:101180006043030881430308A2430308C3430308E1
:10119000E443030805440308496400204E1D002071
:1011A000881D002064130020181E002015F04EFA40
:1011B00008B930233B703B78884E13B93379112B33
:1011C0004ED1DFF86892FCF79BFC854899F8111026
:1011D000FFF7ACFD824B1A78984622B1002010210F
:1011E0004A46FCF7E3F8237898F800407D4A24EA61
:1011F000030111707C4A23EA040111703A78A2F1CC
:101200005200C0B2012803D93079744F11280CD193
:10121000002333711CB911B10133009311E1042390
:10122000F3702B7801332B701AE0432A18D1BBB925
:101230007C78ACB96D4BD879F4F7D0FF38B96C49EC
:10124000F7F73CFC0523FB7008332B7004E02046C5
:101250006849F7F733FCFC70674A684B1A606CE129
:101260005F48FCF7C9F868E10A2B31D15D4807F007
:10127000A7F8C6B2594C36B3E378042B02D100204C
:101280005F4903E0022B04D15E490020F7F716FC0A
:1012900002E00BB90433E370314602225A48F7F7F3
:1012A00033FC5A4B1E78232E00F0D3803046F7F7DC
:1012B000C1FC002800F04181312E40F03E812B78A6
:1012C00001332B7002E03B7801333B70042332E0A2
:1012D0000B2B32D1434807F059F8C6B23F4C36B316
:1012E000E378042B02D10020494903E0022B04D10A
:1012F00048490020F7F7E2FB02E00BB90433E37042
:10130000314602224048F7F7FFFB404B1E78232E60
:1013100000F09F803046F7F78DFC002800F00D812B
:10132000312E40F00A812B7801332B7002E03B789C
:1013300001333B700823E370FFE00C2B40F0FD808D
:10134000284807F009F80021C4B2264806F0DAFF61
:10135000002C6DD0214EB3782BB9BE2014F0B0FE16
:10136000B3780133B370F3781C4A092B02D90020FB
:101370001F4915E010D11D4B00241C70D470264B62
:10138000194A1849164801251C7014700C70047015
:101390000095019402949EE0082B04D11F4900207F
:1013A000F7F78CFB11E0062B02D100201C49F7E770
:1013B000042B02D100201B49F2E7022B02D10020AE
:1013C0001949EDE70BB90833D370F378082B3CD8F3
:1013D0000D4821460222F7F797FB36E06B130020F9
:1013E000881D0020711E0020641E0020221E002087
:1013F000723D0308EE3C030894BA0208841D0020E5
:10140000F63D0308173E0308F40100204C1D0020A0
:10141000B43D0308D53D03084D1D00200F3D0308D2
:10142000303D0308513D0308933D03084E1D002045
:10143000012543484349444A2B460095F2F78AFB6D
:101440000095424B01941B7840E0414F3C78232C9F
:1014500002D1FCF77DFB70E02046F7F7EBFB00289C
:101460006BD0303CE4B2631EDBB2012B3C7039D848
:10147000022C364D1ED1E879F4F7B0FE002838D0A2
:101480002F48FCF71FFB002833D1082246F64E01F7
:10149000304800F0A2FC2A492E4813F0A4FF2D4941
:1014A000082246F64E0000F092FC2A492A4813F022
:1014B000B0FF06E0012322482249234A0093F2F7B5
:1014C00049FB01230024009301942B7802932348C5
:1014D0001D49234A1B4BFCF781FAF7F7B3FB214B5D
:1014E0001C602AE0032C28D1184BD879F4F776FE3B
:1014F00010B90C23F37020E015F0A8F870B9044679
:101500000F48214613F0B7FF28B1E02014F0D8FDB2
:10151000204614F011FE0134402CF1D1124A002370
:101520001370F3702B78114A01332B700D4B1A6036
:101530000F4B1A7842F006021A7007B0BDE8F0832C
:10154000071C00204D1D0020711E0020221E0020BF
:101550004C1D0020FC190020591A0020881D002075
:10156000641E0020841D00201E1E002094BA020864
:10157000631E0020194A00231360194A194813708A
:10158000194A1178037001F0F60163F30711117025
:10159000164A1748117863F301011170154A117842
:1015A00063F3C5011170144A1370144A117801F0E5
:1015B000FC0163F382011170114A1168037021F478
:1015C000805163F3CF3111600E4A117801F0F401BC
:1015D00063F3820111700C4A93717047841D0020DF
:1015E000431E00201E1E0020631E0020651D0020DB
:1015F0006E1E0020191E0020211E0020301E00201B
:10160000883A0020DF3C00206B1300202DE9F04FCA
:101610006A4B6B4D1970A0F11103DBB2012B87B03F
:101620000E46287006D8122801D1113800E000209B
:10163000F4F79CFE2B78522B0DD1F1F77DFD28B9E4
:10164000F1F76EFD10B9F1F78FFD20B15D4B1A78FF
:1016500042F008021A705C4B5C4C1B782BB9226874
:101660005B4B9A4201D0FFF785FF2368002B40F0C7
:101670004081584F7B7803F02003DBB273B1564BA7
:1016800093F80080B8F1000F08D14AF6E90041460E
:1016900000F088FB3B6868F34D333B604F4B187894
:1016A00010F01E0002D000204D4907E04D4B93F88A
:1016B00005909846B9F1000F05D04B4907B0BDE839
:1016C000F04FF7F7FBB9494F97F801B0BA46BBF1B5
:1016D000000F2DD0BBF1070F15D94548F7F794F946
:1016E0004449B878652246F61573F7F733F9387828
:1016F000072310F003007B700EBF3F4948463F4967
:10170000F7F7DCF90CE0BBF1020F09D83848437851
:1017100023B1F7F779F987F8019093E202237B7000
:101720001020334A014607B0BDE8F04FF7F77EB905
:10173000334B9A795AB183F806B000F09FFC8E20A3
:10174000594601225B46CDF800B0F0F7DDFF0020DE
:10175000F1F754FE2B4A2C4913782C4843F006032A
:10176000137000230B702A4923600B7088F8013036
:1017700088F80430037029337343264F9146F95C8F
:101780008346C1F3C00111B93046FFF785F829231C
:1017900003FB06777B7913F0100F04D02A78133AF5
:1017A000D2B2032A3AD913F0200F5DD02B78442B04
:1017B00034D031D8232B31D02A2B2EE0161E002016
:1017C0004C1D0020561A00206F1E0020841D002092
:1017D00094BA0208883A0020141A002051590020B7
:1017E000C71203086B130020264403081B1E0020A9
:1017F000741E00207B1E0020CF130308AE130308C5
:10180000221E0020631E0020431E0020181E002000
:10181000131E0020A53B0020552B25D1844B1B789F
:1018200013BB844B1F78FFB943F6DB2000F0C4FAEA
:101830000128014618D188F801001F200591FFF703
:1018400013F899F80030304667F3410389F8003007
:10185000059909F065F9F7F7F5F9774B2360774BB0
:101860001F602B788BF800302B78432B0AD1714BFB
:101870001B783BB90121724B88F801103046236078
:1018800009F04EF928781738C3B2072B27D86D49CD
:10189000FF220BF0EFF89AF800106B4B60F3010198
:1018A0008AF8001001F00301022918D00122032058
:1018B00041B1009001929B7868309B1802930021FF
:1018C000033206E0009001929B786C200133029372
:1018D00004220B4600F0EEFAFF238AF8013098F854
:1018E0000730002B00F0AE8152232B70574B0022A3
:1018F000DA712268524B9A4250D12878A0F1430302
:10190000DAB2122A22D8524A5BB29A401ED5432834
:1019100040F09881464B1B78002B40F0938100F0FB
:10192000AFFD4C4B48B11A7803201109013191FBEE
:10193000F0F000EB4000091A04E01A7811090131B7
:1019400001F0070161F307121A707BE1F7F772F9F2
:10195000002823D03F4F3B7813F0F00108D161F30A
:1019600007133B703C4B21601A7842F008020EE0EE
:10197000102913D100F084FD80B13B7800216FF372
:1019800007133B70344B21601A7842F01002304646
:101990001A7007B0BDE8F04FFEF77EBF2F4B1E2137
:1019A0001A78254F61F346021A702B78232B1CD12D
:1019B0002368BB4219D12A4B292202FB06367379D0
:1019C00013F0100F11D0274B1B7873B1264EF7F789
:1019D00039F9FCF7BDF8F07900F56A507C3000F079
:1019E000EBF93070AA20F1F709FD1A4E337813F0A5
:1019F000010F41D02368BB420BD01C4A934208D050
:101A0000FEF706FF28B9FEF719FF10B9AA30F1F763
:101A1000F5FC2268164B9A4202D10020F1F7EEFC49
:101A20002B78522B40F0D3805322124BC7E000BFDB
:101A3000141A0020801D002078BA0208501E0020D1
:101A40008CB502081D1E00201B1E00206B130020F9
:101A5000002000C0631E0020301E0020E11E002078
:101A6000A53B0020431E0020221E002094BA02083D
:101A7000B0BA02084C1D00202368BB420BD0734A49
:101A8000934208D0FEF7C4FE28B9FEF7D7FE10B97E
:101A9000AA30F1F7B3FC2B78552B1ED1FEF764FE6C
:101AA00033786B4843F0060333708378694F03F053
:101AB0000203DBB24BB1F6F7A7FF23681868FAF709
:101AC00023F93B786FF341033B706348837803F05D
:101AD0000203DBB20BB1F6F797FF2B78442B1ED134
:101AE000FEF7F2FD33785A4843F0060333708378EB
:101AF000584F03F00203DBB24BB1F6F785FF2368C2
:101B00001868FAF701F93B786FF341033B705248CC
:101B1000837803F00203DBB20BB1F6F775FF2B7885
:101B2000522B09D13378002243F0010333704B4B21
:101B30001A704B4B45321A704A4B00271F702B7896
:101B4000232B44D1484B42481F70484B1F70F6F777
:101B50005BFF4148F6F758FF3378454943F00603E9
:101B600033700B783B4A002B2BD0424A013B177055
:101B7000414ADBB20B7052F8233023603F4B1A7896
:101B800012B11F700EF04CFD23683D4A9B689342D2
:101B900002D10AF09DF81AE002F59A718B4203D047
:101BA00002F5E0718B4204D10120014607F0F0F804
:101BB0000DE002F5EE72934209D1324B00221A7009
:101BC00005E0117863F30711117023603AE02E4BA2
:101BD0005B7813B10020F1F711FC23681F7B17F02D
:101BE0000F0702D1FBF782FA1BE0012F02D1F8F7B1
:101BF000C3F916E0022F02D1F9F73CF911E0082FE2
